:020000040800F2
:1000000000C000202D4A0108CD4A0108153401081E
:10001000CD4A0108CD4A0108CD4A01080000000080
:10002000000000000000000000000000CD4A0108B0
:10003000CD4A010800000000CD4A0108077E0008F3
:10004000CD4A0108CD4A0108CD4A0108CD4A010830
:10005000CD4A0108CD4A0108E5C90008E3C90008F6
:10006000CD4A0108CD4A0108CD4A0108CD4A010810
:10007000CD4A0108CD4A0108F9C90008CD4A010856
:100080008D8E0008CD4A0108CD4A0108CD4A0108ED
:10009000CD4A0108CD4A0108CD4A0108E1C900084E
:1000A000CD4A0108C9C50008CD4A0108D9C50008D4
:1000B000B9C50008A9C5000899C50008D967000896
:1000C000DD670008D1670008D5670008CD4A010840
:1000D000CD4A0108F1C90008E7C90008CD4A010866
:1000E000157E0008CD4A0108CD4A0108CD4A010815
:1000F000CD4A0108CD4A0108CD4A0108CD4A010880
:10010000CD4A0108CD4A0108CD4A0108CD4A01086F
:10011000CD4A0108CD4A0108CD4A0108CD4A01085F
:10012000CD4A0108CD4A0108CD4A0108CD4A01084F
:1001300000000000000000000000000000000000BF
:1001400000000000000000000000000000000000AF
:10015000000000000000000000000000000000009F
:10016000000000000000000000000000000000008F
:10017000000000000000000000000000000000007F
:10018000000000000000000000000000000000006F
:10019000000000000000000000000000000000005F
:1001A000000000000000000000000000000000004F
:1001B000000000000000000000000000000000003F
:1001C000000000000000000000000000000000002F
:1001D000000000000000000000000000000000001F
:0401E0005FF8E0F1F3
:1001E8002DE9F04F684B694F9FB03B6000237B605F
:1001F80011F0AAF818B911F0C9F80AF0C3FE0AF00C
:1002080067FF634A634D1378634E43F0010313702D
:1002180000230693079308934FF4E01309932B6880
:10022800B07B43F480332B60AB6943F01003AB61C0
:100238002B6803F400330793069B01330693079B4F
:100248001BB9069BB3F5A06FF2D12B68514913F483
:10025800003301D0022315E00A6842F001020A6067
:1002680006932B6803F002030793069B013306935A
:10027800079B1BB9069BB3F5A06FF2D12B689A07B1
:1002880039D501230893454B45491A6842F01002B5
:100298001A601A6822F003021A601A6842F0020211
:1002A8001A606B686B606B686B606B6843F48063A3
:1002B8006B603C4B1A68043B22F070425A603A4A21
:1002C8001160696821F47C116960596841F0004146
:1002D8005960D96821F40041D9609B681B0449BF63
:1002E800324B4FF4E01313604FF480130993089BCB
:1002F800012B01D117E0FEE7022B18D168B1099B49
:10030800B3F5801F02D14FF4A01305E0099BB3F5A4
:10031800E01F02D14FF40013099309996B680B434E
:1003280043F4803302E06B6843F460136B602B681E
:1003380043F080732B602968164B8C01FBD55968F4
:1003480021F003015960596841F0020159606B6856
:10035800104903F00C03082BF9D14B68DFF854B0AF
:1003680003F00C03042B03D0082B03D00C4B29E01B
:10037800136827E04B684868C3F38343C00303F15D
:10038800020319D40A4A1CE073A70008D800002009
:100398006031002000100240EC11002000200240D3
:1003A80000127A000410014038000020001BB7003A
:1003B80000093D0060000020496812688C0348BFAE
:1003C80052085343CBF800306B68DFF87082C3F3F0
:1003D800031343441A7EDBF800301EACD340CBF83D
:1003E80000307F4A7F4BDFF858A2D360AB69029296
:1003F80043F00103AB616B6A4FF00009BB606B6AA5
:10040800794843F080736B62AB6943F01C03AB61BE
:100418004FF6FF7324F82C3D21468DF84E900FF0CF
:1004280033FE504621460FF02FFE704821460FF04C
:100438002BFE6F4920464B6843F000734B600FF06A
:1004480059F9139B6B49A646B3FBF1F36A49029A23
:100458000B606A4B4FF47A71C3F80090DBF80030F8
:10046800DFF8E0C1B3FBF1F36549013B4B60F023D2
:1004780082F823300723C1F808900B60B36808F1AD
:10048800280BCCF80030BBE80F00AEE80F009BE863
:100498000300AB698EE8030043F00803AB61AB6966
:1004A800042243F00803AB61AB6943F02003AB615E
:1004B8000823CAF810301023CAF81030E246514B0E
:1004C8001A6109F1040154F80900214409F10809E5
:1004D8000FF0DAFDB9F1180FF3D1642007F085FCAD
:1004E800A0224948002116F06CFEEB69002243F077
:1004F8000703EB61AB6943F4006343F00C03AB61A2
:10050800424B4FF0000B03F10C0102F801B001322D
:100518000E2AF5D1FF229A76DA761A775A773C4B6B
:100528003C4A59461A603C483022DAF8005016F026
:1005380048FE5946C5F380190423384ADFF8D8E045
:10054800885C0C224A4302F80E00B9F1000F08D16A
:100558001E3801289FBFFF2003F1FF3302F80E0069
:10056800DBB201310429E8D12D4A2E481370737982
:100578002D4A264913702D4A3A62C03202602C4A2D
:10058800A80602EBC302527848BF01224A62002241
:1005980040F2DC50274921F812000132082AF7D12D
:1005A8000CA800211C22029316F00BFE15F4007B08
:1005B80005F4006A029B47D0AA040BD4BAF1000FD5
:1005C8000AD01D4A96F88601A2F10C01012808BF3D
:1005D8000A4602E0194A00E0174A0292129435E0EE
:1005E80000ED00E00005FA05000801400010014098
:1005F8000000014040420F00681B00206C1B0020D7
:1006080010E000E000140140B01B0020D8000020DA
:10061800C42A0020E0130020C82A00209EC8010830
:10062800A5110020CC1C00201C0A0020001200206C
:10063800D8BD010810110020A0970108949701085F
:10064800000C01409C2D0020CDF808B00E2B03D0E3
:1006580003F0EF03082B02D101238DF8423001206B
:1006680009F002F918B14088003018BF0120C5F31D
:1006780040038DF83630C5F3403300F001008DF8A3
:100688003030C5F3C0338DF835008DF838908DF8CB
:100698003330BAF1000F07D096F886A10AF1FF3E71
:1006A800DEF1000A4AEB0E0AC5F300438DF8393033
:1006B8007B6A1BF1000B18BF4FF0010B003318BF0A
:1006C80001238DF83B30C5F300538DF83C30B6F864
:1006D8004A31B6F84801ADF84030B6F8563105F061
:1006E8000101C5F3C002ADF83E30C5F38043ED0407
:1006F800ADF8460048BFB9488DF8373048BFB0F864
:100708005001B6F8543148BFADF84600B3F5FA7F4A
:10071800ADF8443084BF0023ADF8463096F8D631A2
:10072800AF4887F82830002387F8293043709DF8B0
:1007380042308DF834A0002B8DF831108DF832201E
:100748008DF83AB00CBF0023022301B902B101337E
:1007580008EB8308D8F840304FF00009A3F1020AEB
:100768001A3303934FF6FF733AF802BF9B4500F024
:1007780081819DF835205FFA8BF31AB19A1E012A00
:1007880040F274819DF8382032B196491A0189588F
:10079800954A914200F06A819DF8392032B1914919
:1007A8001A018958904A914200F060819DF83620DC
:1007B80052B18C4A8D4802EB03125168814203D131
:1007C8001289102A00F052819DF8332052B1854ACF
:1007D800864802EB03125168814203D11289022A2A
:1007E80000F044819DF8342052B17E4A804802EBE3
:1007F80003125168814203D11289022A00F036811E
:10080800129A7AB1774D116805EB0315686888422A
:1008180008D129899088884200F02881D2888A42A4
:1008280000F024814FEA1B2BBBF1020F02D19DF887
:10083800302004E0BBF1010F04D19DF83120002ADB
:1008480000F01481674A9DF83C004FEA031802EB58
:100858000805114630B19DF8420018B9043B032B36
:1008680040F2EC80BBF1010F5FFA8BF344D1614E8B
:100878004144FF2391F80DE086F8703086F8713016
:10088800486801F1080309890027ADF84C100221D6
:100898008DF84F1086F8747013A9C6F880508DF83B
:1008A8004EE00592049386F82C7037637763B7633C
:1008B800F76686F8727086F873700FF0E5FB049B94
:1008C800059A997852F808003A4608F02CF9284613
:1008D80039465A460BF0DCFF474BC6F88C70C6F811
:1008E8008430464B2846C6F8883006F1840106F164
:1008F80088020CF015F8B9E0022B4AD15FFA89F2A8
:100908001C2101FB02FC3B4A002602EB0C07354A7E
:100918004FF0010B02EB080191F80DE001F108021C
:100928004868098987F87590ADF84C1087F87660A3
:1009380013A987F87E6087F874B0C7F88050CDF89F
:1009480014C08DF84EE004928DF84F300FF09CFBE8
:10095800244B049A53F808009178324608F0E3F8DB
:10096800284631465A460BF093FF254A214BDDF8BD
:1009780014C0C7F8842003EB0C01224A8431C7F85D
:100988008820C7F88C6028460A1D0BF0C9FFD94497
:100998006CE0032B50D19DF83730164E1A4F3BB1FF
:1009A80096F82A80284608214FF6FF72002337E080
:1009B800BDF8442096F82A80B2F5FA7FBDF8463093
:1009C80028D912492846B1FBF2F2082192B208F060
:1009D800FFF80F4B47F8280027E000BFEC11002074
:1009E8000101002068BA0108000400400008014025
:1009F800000C0140D80000209D8500087D86000875
:100A0800698B000873850008801B002000127A009B
:100A18009D8600086A492846B1FBF2F2012192B28C
:100A280008F0D6F8674B47F82800C36096F82A30D4
:100A3800013386F82A3019E0042B17D1BDF83E207F
:100A48005F4B614E93FBF2F22846BDF8403001211E
:100A580092B296F8297008F0BBF896F8293006EBA0
:100A680087070133C7F8540186F82930039B9A4554
:100A78007FF478AE544E554B96F82920002586F819
:100A88007421534A1D7017789846A7F11702022A55
:100A98001AD8336A0021585903EB050912F072FF7E
:100AA80010B1736A7BBB27E04A4B05EB030E99E84C
:100AB8000F008EE80F0098F8003010350133C02D74
:100AC80088F80030E5D1ECE7434B13F837C003EB67
:100AD800C703D3F8049088F800C0B9F1000FE0D03C
:100AE8006545DEDA3B4A2B0103EB020E4B440FCB84
:100AF80001358EE80F00F3E7384B1A68994612F46F
:100B0800805F26D11FE0364B364A13F8370003EBD7
:100B1800C7035D681070002DEED000238342EBDA26
:100B2800C3EBC3016A18D2F80090DFF8C4C00133E0
:100B380041F80C9001EB0C0E9188AEF804109279F4
:100B48008EF80620EAE707F0EF03082B264B25D19D
:100B580026E098F80030012BF5D9244D05EB031356
:100B680003F1100810354545EDD055F8100C4FF03D
:100B78007C5112F073FD4FF07C5145F8100C55F87C
:100B8800140C12F06BFD4FF07C5145F8140C55F81D
:100B98000C0C12F063FD45F80C0CE3E70E2F08D19E
:100BA8001A78182F42F010021A7023D107F0AAFB06
:100BB80020E01A78192F22F010021A70F5E700BF0A
:100BC80040420F008D860008D8000020671B0020D7
:100BD8001C0A002058090020D8BD01089C2D0020BF
:100BE80028A30108581C0020E019002060090020F3
:100BF800591C002007F06AFBD9F80030BC4F580395
:100C08005EBFBC4B01221A70BB4A4FF48058137860
:100C18004FF0020B43F00403137014238DF84E3089
:100C2800BB69214643F00403ADF84C808DF84FB002
:100C3800B248BB610FF028FAB14AB24B00201A60E3
:100C480007F0ECF8B04BB14D93E80300BB6984E8BA
:100C5800030043F00803BB61139814A90FF014FABA
:100C6800FB69284643F48043FB613B69214643F412
:100C780080433B6118238DF84E304FF42043ADF884
:100C88004C3003238DF84F304FF0040A0FF0FCF975
:100C98004FF48043284621464FF01009ADF84C30F8
:100CA8008DF84EA00FF0F0F928462146ADF84C809B
:100CB8008DF84E900FF0E8F93A69072342F4804224
:100CC8003A613A69012022F480423A61904A1188D7
:100CD80001F4415141F4457141F003011180918BB8
:100CE80021F4006101FA09F121FA09F191831382D3
:100CF800118889B241F040011180C5F81080DFF8F1
:100D08002C820FF0DBFBD8F80040824D04F400433E
:100D180003934A4604F4006328460021049316F01E
:100D280050FA4FF6FF728DF82EB014F002044FF00F
:100D3800000BADF82C208DF82FB00DD01EA921F88E
:100D48004C9D6E480EF07AFE0124072385F800A01A
:100D580085F801B0AC70EB70039B73B102231EA938
:100D680021F84C3D65480EF069FE0123E2182B710D
:100D7800AB7107236C71EB71D4B2049B7BB1022376
:100D88001EA921F84C3D61480EF058FE09230122A6
:100D98002B73AA73631C07226C73EA73DCB27B683B
:100DA8005D4843F440437B607B694FF0000943F0A2
:100DB80001037B61BB69DFF860A143F40073BB6189
:100DC8000EF020FC554B012C1393554B13A914938B
:100DD80094BF4B46802318934FF4807319934FF4B4
:100DE80080631A9320231B9350464FF400531694A4
:100DF8001C93CDF85490CDF85C90CDF874900EF01B
:100E0800E3FBDAF80030474A43F00103CAF8003040
:100E18005368012C23F4702394BF0021012123F48B
:100E2800807343EA0123536091683F4B013C0B40B8
:100E380043F4602343F002039360D36AE4B223F4DB
:100E4800700343EA0454D462012305EB0902917844
:100E580000297DD015F80900591C0928C9B2D27893
:100E6800DFF8C0E011D9A0F10A04DEF80CA004EB09
:100E780044044FF0070C0CFA04FC2AEA0C0CA240BC
:100E88004CEA0202CEF80C200EE0DEF8104000EB2F
:100E9800400C4FF0070A0AFA0CFA24EA0A0402FA8C
:100EA8000CF22243CEF81020062B1E4C0ED8013B24
:100EB800626B03EB83034FF01F0E0EFA03FE22EA68
:100EC8000E0200FA03F31343636340E00C2B2FD8A0
:100ED800073B226B03EB83034FF01F0E0EFA03FE52
:100EE80022EA0E0200FA03F3134323632FE000BF44
:100EF80000100240880E00206031002000080140E8
:100F0800ED74000870310020E4970108000C0140DE
:100F180000380040242B0020080002404C240140E7
:100F2800342B002000240140FDF7F1FF9C2D002008
:100F3800A3F10D02D4F82CC002EB82021F239340C8
:100F48002CEA030E00FA02F34EEA0303E3620B46AF
:100F580009F10409B9F1100F7FF477AFAF4B9A6824
:100F680042F480729A609A6842F001029A609A6824
:100F780042F008029A609968A84A0907FBD4936866
:100F880043F004039360A54B9A6812F00409FAD160
:100F9800A34D9A68B5F85C0142F4A0029A60002853
:100FA80041F0A482B5F95E31002B41F09F82B5F97A
:100FB8006031002B41F09A82D8F800309B031FD58E
:100FC800C82006F012FFAE200FF0E3F908B10FF0C9
:100FD800E5F9944C86F87501C82006F006FF924B97
:100FE80000210C222046C6F8783116F0EAF80223D0
:100FF800E3700CF046F806F0D1FE8C4B0344A36076
:1010080095F86B31B5F864410493894B95F863A161
:101018001B6895F86C81B3F85630B5F80CB0059399
:10102800EB7B844D00210C228348039316F0C9F80A
:1010380014222846002116F0C4F8804A00231370B1
:10104800C6F87C3105F0B4FC30B37D4BB4F5807F35
:101058002B607C4B6B607C4BEB607C4B2B617C4B3F
:1010680001D1002216E0BB2C01D9012212E0612C2B
:1010780001D902220EE0292C01D903220AE0132CFF
:1010880001D9042206E0092C01D9052202E0002C2E
:10109800E7D006221A7062E06E4B93F8825125B9A8
:1010A80005F044FC002800F0A7836B4B00221A804F
:1010B8000DB905F0E5FBB4F5807F00F0A283BB2CE9
:1010C80000F2A183612C00F2A083292C00F29F83F7
:1010D800132C00F29E83092C00F29D83002C14BF70
:1010E800062500255D4A1920138823F040031B04B8
:1010F8001B0C1380138823F038031B041B0C43F0CC
:101108003003138013889BB243F04003138096F892
:10111800801105F0A5FB012006F05CFE29461A2087
:1011280005F09EFB012006F055FE13A805F018FBFC
:101138009DF94E30484A013300F0578313889BB21B
:10114800002B40F057833B4B454A64201A60454AC0
:101158005A60454ADA603D4A1A6106F046FE0123A4
:10116800424A434D2B70136843F001031360002378
:10117800404ABAF1090F00F2B180DFE80AF005AF82
:101188000505818105819AA51370C6F87C3105F0A3
:101198000FFC002875D006210A4613AB682010F012
:1011A80037FE9DF8511001F001029DF84F1001F033
:1011B80001014B0043EA82019DF84D2002F0010332
:1011C8000B430AD05BB2012B01D1002302E0022BB2
:1011D8000ED1012386F8813111E00BAB68200C2178
:1011E800012210F015FE9DF82C3013F00F0303D1E7
:1011F800032006F06FFE02E0042BEAD1E5E70E4B70
:101208001D4A1A601D4A5A6096F88121002A0CBFAF
:101218006F226E221A72032327E300BF00240140C5
:10122800EC1100209029002076130020404B4C0040
:101238002011002050290020682D0020DC07002004
:10124800E1640008116400088B62000890C1793DD0
:1012580000000020D80000208C2D0020003800401D
:101268008962000869670008DD660008DC1900204B
:101278005C00002088310020516500085364000894
:10128800137096F8826136B1644B00221A8036B921
:1012980005F0F6FA03E005F049FB58B1F4E7604BB6
:1012A800604A64201A60604A5A6006F09EFD07236F
:1012B800DBE2137005F090FA38B1594B5B4A1A60BB
:1012C8005B4A5A600823D0E21370554B594A1A609A
:1012D800594A5A6000221A720923C6E2BAF1010F6C
:1012E8003FF652AF1370B8F1040F00F2C181DFE886
:1012F80018F00500CA01680005008C010A2006F0F4
:1013080074FD7720A02101220BAB10F081FD00288D
:1013180057D01E210122772010F0BAFD4FF42F601C
:1013280006F058FD0026A6F160010025C9B2022288
:1013380013AB77208DF84C508DF84D5010F068FDA8
:101348009DF84D309DF84C2043EA02223B4B03F5B3
:10135800C27172520236102EE5D1B3F89221294695
:1013680002F00F0E02F47F42A3F892212B460126C9
:10137800324D21F001002844B0F88401002818BF3C
:10138800002611F0010F03D0C0B24340082002E04C
:1013980083EA1023FAE713F4004F18BF83F4C0530D
:1013A80001384FEA4303F6D101311029E0D142EA6E
:1013B8000E02A5F8922126B9C3F303339E4500F027
:1013C8005B821E4B93F89481B8F1000F41F0AE8018
:1013D800BB691B4E43F01003BB6102234FF4005559
:1013E8008DF84F303046102313A98DF84E30ADF8E4
:1013F8004C500EF049FE4FF48043ADF82C30304687
:1014080028230BA98DF82E300EF03EFE0D4B3561CA
:101418001A68CAB1404606F05DFD17E08C2D002021
:10142800682D0020796200080167000869620008D9
:101438000766000881F200089DF20008D800002025
:10144800001001406C1B0020C04A1A60C04B0127E5
:101458005A69002522F470625A615A6913A842F445
:1014680000725A614FF48043139308238DF851306A
:101478008DF850508DF852700EF0B0FA28230DEB0D
:1014880003004FF0030A8DF828308DF829A08DF855
:101498002A508DF82B7011F039F9142006F0A5FCAC
:1014A8007720D0213A460BAB10F0B2FC002800F0B0
:1014B8009D809DF82C30A74D552B85F8AF31A5F8A8
:1014C800B8A140F09380D1213A460BAB772010F0B9
:1014D8009FFC9DF82C30772003F00F021B0985F83C
:1014E800B02185F8B131162213ABAA2110F090FC77
:1014F8009DF84C209DF84D3043EA0223A5F8983119
:101508009DF84E209DF84F3043EA0223A5F89A3102
:101518009DF850209DF8513043EA0223A5F89C31EC
:101528009DF852209DF8533043EA0223A5F89E31D6
:101538009DF854209DF8553043EA0223A5F8A031C0
:101548009DF856209DF8573043EA0223A5F8A231AA
:101558009DF858209DF8593043EA0223A5F8A43194
:101568009DF85A209DF85B3043EA0223A5F8A6317E
:101578009DF85C209DF85D3043EA0223A5F8A83168
:101588009DF85E209DF85F3043EA0223A5F8AA3152
:101598009DF860209DF8613043EA022341F27072A1
:1015A800A5F8AC316C4B1A8046F678125A806B4A13
:1015B8005A606B4A9A606B4ADA606B4A1A616B4AE6
:1015C8005A6195F8943143B904F08AFE42F6E06016
:1015D80006F000FCB368C3F38038654B012283F83A
:1015E80002805C4B83F8942100F0A0BF614A136825
:1015F80023F480431360604B544A1968914204BF36
:1016080000221A604FF400537361524D95F8BC6183
:10161800002E40F04381142006F0E7FB05F2BD13CD
:101628007620D021012210F0F3FB95F8BD31582B1C
:1016380029D105F5E07388211822762010F0E8FBFF
:1016480031227620F42110F023FC01234B4A85F83F
:10165800BC31414B9A604A4A1E805A6045F6D812FE
:101668005A80484ADA60484A1A61484A5A6115E17C
:10167800B8F1010F07D0464B464A83F80280136839
:1016880043F004031360434D2B689E0702D5424B79
:101698001B689847039BE4B22E4E404A4BB32B6815
:1016A8004CB940F2596113F0020F40F2712318BF90
:1016B8000B467D2108E09C0759BF4FF47A73194601
:1016C8004FF4FA634FF47A719B4505DBBBF57A6FEB
:1016D800A8BF4FF47A6B00E09B464B1E5B44B3FBFC
:1016E800F1F3013BDBB203FB011186F88031116095
:1016F80005E09DF80C30C2F800B086F88031284F1C
:10170800B8463B689847049C264F0023022C3B7040
:1017180004D0032C4ED0002C40F0C38000221EAB16
:1017280003F82C2DC6F8DC211E200A21012210F016
:101738006FFB00283ED09DF84C30482B3AD11A4B0D
:101748001A4A1A601A4A5A600223AEE04162000837
:1017580000000140D800002070060020E96200085F
:10176800DD630008C3620008916300086561000832
:1017780000000020000401406C1B0020616100088B
:1017880063610008B962000845630008FD5E00084F
:101798005C000020DC190020682D0020002E0020AD
:1017A80050290020893100204C060020F50001084E
:1017B80055FD00084FF0000A1EAB03F82CAD0C20B5
:1017C8005146012210F024FB002800F0B3869DF852
:1017D8004C30482B06D1524B524A1A60524A5A6032
:1017E800032362E0504600F0A5BE9DF94C3001335A
:1017F8007FF4A4AC0023138004F0EEFF4B4B60B9D8
:101808002BE000256EE401256CE402256AE403253B
:1018180068E4042566E4052564E4454ABB2C1A609F
:10182800444A5A60444ADA60444A1A61444B01D92E
:1018380001220EE0612C01D902220AE0292C01D9EB
:10184800032206E0132C01D9042202E0092C02D954
:1018580005225A7083E40622FBE73A4A1A603A4A9C
:101868005A603A4A9A6008237AE4394A6B701368D6
:1018780043F00203136036E542F21072354B4FF025
:1018880003081A805A80344A5A60344A9A60344AA3
:10189800DA60344A1A61344A5A61ECE64FF00408B7
:1018A800E9E6012C07D91C462EE7304AD3702B688D
:1018B80043F008032B602E4C94F858310BB12D4A95
:1018C800137094F859310BB12B4A137094F85A31AC
:1018D80003B13B702B68DFF8ACA013F0080F53D0AE
:1018E800BDF914204FF0640B92FBFBF738460492C5
:1018F80011F060FE049A03900BFB172000B211F060
:1019080059FE1E4911F0AAFE039B0146184611F024
:101918009DFD1B4911F0A2FECAF8000037E000BF88
:101928004C06002065FE0008D1FD00085029002063
:1019380065660008C9650008A565000890C1793D7D
:101948000000002087F20008ABF2000883F20008CC
:10195800DC19002070060020AF620008356300081B
:10196800A562000825630008415D00085C000020AE
:10197800EC110020DC070020883100208988883C91
:1019880000002041D81C00200023CAF80030B74AC4
:101998000A27137843F002031370B54B10225A61DB
:1019A80008221A61DFF8C8A21920DAF80C30013FC2
:1019B80083F01003CAF80C30DAF80C3083F008030F
:1019C800CAF80C3006F011FA012006F027FA19209F
:1019D80006F00BFA002006F021FA17F0FF07E1D114
:1019E80008231027CAF81030CAF810702B68180797
:1019F80009D5A04BCAF814701B6898479E4B012262
:101A0800CAF810701A709D4B9D4F1B68187B11F017
:101A1800D1FD9C4911F022FE09F090F982463888E0
:101A280011F0C8FD514611F019FE15F0D7FD964B7F
:101A38001880388811F0BEFD0146944811F0C2FEA6
:101A4800934911F0BFFE934B8E491860D8F81000E7
:101A580011F004FE904911F001FE904F904BFF21C8
:101A680018601B22384615F0ACFB00223A702A6831
:101A78008C4B012112F0020F19701FBF79700321DE
:101A88001970022118BFB970510748BF1978384634
:101A980041BF4D1C1D7003257D5412F00A0F0CD058
:101AA8001A780421B954511CC9B205257D54D11C9A
:101AB80002321970D2B20621B9547B4D29688F06BB
:101AC80041BF1A78571C1F70072748BF87540A065A
:101AD80008D51A7809278754971C01321F70D2B28B
:101AE8000A2787546779082F01D00E2F08D11A7852
:101AF80002F1010E83F800E04FF00B0E00F802E04F
:101B08001A7811F4803F4FF00C0C00F802C002F173
:101B1800010E1CBFDFF88CC102325FFA8EFE83F81B
:101B280000E01FBF8CF800205C4A4FF00E0C02F852
:101B38000EC04A0748BF1A784FF0120C41BF02F195
:101B4800010E83F800E04FF0100E00F802E01A785A
:101B580011F4806F02F1010E5FFA8EFE83F800E047
:101B680000F802C00ED094F818C2BCF1000F09D0DA
:101B7800DFF830C102328CF80020484A4FF0130CCD
:101B880002F80EC01A7811F4007F4FF0140C00F818
:101B980002C002F1010E1CBFDFF808C102325FFA71
:101BA8008EFE83F800E01FBF8CF800203B4A4FF000
:101BB800150C02F80EC0182F13D11A784FF0160E14
:101BC80000F802E002F1010E5FFA8EFE4FF0170CEA
:101BD80000F80EC002F1030E0232D2B283F800E020
:101BE80087540A0341BF1A78571C1F70192748BF2A
:101BF8008754CF0541BF1A78511C19701A2348BF62
:101C0800835400219822294815F0DBFA0DF0D9FBFE
:101C1800274A284BB4F852111A60274BB4F8980198
:101C28001980264900230B808B7025490A6081B2F0
:101C3800244A22F813100133122BF9D12B68D90446
:101C48005CBFB4F89E1111801B0740F1F28094F834
:101C58009231062B00F2E780DFE803F004363D6896
:101C680083A2A20045F2F05230E000BF60310020AC
:101C7800000C01404C060020640600206808002083
:101C88002C00002035FA8E3C840800200AE81C410C
:101C980000401C4698070020BD378635E910002013
:101CA80064080020E81000209C2D0020202A002035
:101CB80076130020BC0F0020C00F00203431002014
:101CC80028310020D82D002042F6F8227E4B1A80B9
:101CD8000DF000FCA6E042F6F8227B4B1A8011F0CA
:101CE80069FC7A4911F0BAFC794911F0ADFB11F0A1
:101CF800A1FE0023774A42F823000133122BF9D1C1
:101D0800754A764940201160754A137007F086FEBF
:101D1800002800F0888001234FF0070A90F900009E
:101D280040218DE808046F4A6F4B76E042F6F822AE
:101D3800654B40201A806D4A674B1A60684B102229
:101D48001A7007F06BFE00286DD001234FF00008D1
:101D580090F9000040218DE80801654A4FF4E1330D
:101D68005BE042F6F822584B40201A80614A5A4BF1
:101D78001A605B4B08221A7007F050FE002852D0F8
:101D880001234FF0000C90F9000040218DE8081065
:101D9800594A4FF4E13307F01FFDC6F8E0013EE071
:101DA80042F6F821484A062B11804D494FF00C02A3
:101DB800DFF884C1DFF884E1504F514C51480A7074
:101DC8000ED000238CF800308EF800303B701B23B7
:101DD80023704D4B027005221A704FF4E1340BE06A
:101DE80000218CF800108EF8001039700270212143
:101DF800454A2170454C1370454A374B40201A60BC
:101E080007F00CFE78B101234FF0000E90F90000A6
:101E18008DE8084023463F4A402107F0DDFC0030AA
:101E280018BF012028B9082009F07AF83A4A2A4B45
:101E38001A602B682A4A13F4804F1FBF08211170BB
:101E48003648254918BF086042F20101194099B186
:101E580044F620601C499F04088041BF0821117086
:101E68002F481D4948BF0860DC0741BF0C2111708D
:101E78002C48194948BF086011781806A1F10401D7
:101E8800517040F19280284F284CC6F8E471002622
:101E9800314615222648DFF8A88066706660A6607D
:101EA800053F15F08EF93046C8F800700AF0B1F811
:101EB800204B02201B68E36007F0B0FD002841D1E9
:101EC800802009F02DF868E0C4080020CDCCCC3F74
:101ED8000000B04438300020340000207D30010874
:101EE800BC2A002021320108A086010069300108BF
:101EF800753101085530010829310108F8290020F9
:101F08001B2A0020233100201C2A002090D0030027
:101F180089F20008B9F20008D9300108AD3001088B
:101F2800C9300108B9300108E0130020B4070020C7
:101F3800C0020020C02D002024310020F9290020F3
:101F4800D407002046796378C5490C2202FB0312A6
:101F58005278B24204D00133DBB2042BF4D9002307
:101F68006370D8F8003062781B7890F90000002B75
:101F78004FF00C0303FB021314BF032601260022B3
:101F88005B7800960192022107F026FCB54B186099
:101F9800002895D001200AF03CF8B34B1868B34BE1
:101FA80000F5C5721A600AF0DBF82B6813AE13F45B
:101FB800007F65D0AE4AAF4C029B1027236093691F
:101FC800AD4843F001039361029B0AA91B888DF871
:101FD8002A70ADF8283002238DF82B300EF054F813
:101FE8002368A5485B880AA9ADF8283004238DF832
:101FF8002A300EF049F8D4F800E00F219EF8083096
:102008004FF0010803F0030203F0FC0303F18043DF
:1020180003F5803398689200914020EA01019960A5
:10202800996808FA02F20A439A60DEF80430934A83
:102038004FF0000A5361304613938DF850A08DF885
:1020480051708DF852800DF0C9FC23680BA85B7A9B
:102058008DF82EA08DF82C3003238DF82D308DF8B7
:102068002F8010F053FB864B864A1B683C3B13605D
:10207800854A13683B431360844B4FF0FF321A6064
:10208800834B844A844C1360844A803313602B68E2
:102098000027D903277040F1B5800EF05BFD40F2B0
:1020A8002A3CDFF82CB2DFF8C8A14FF001086246DD
:1020B80058463946CDF808C084F8008015F081F8F4
:1020C800DAF81830764843F00403CAF81830402389
:1020D800ADF8283018238DF82B300AA903238DF882
:1020E8002A300DF0ABFCDAF81C306E4943F00203DD
:1020F800CAF81C306C4B6D4C1B68AAF6947AB3FB7B
:10210800F1F32188013B21F45C710904090C218059
:102118009BB21D21A1852385A4F81480238C23F06C
:1021280001031B041B0C2384238CA088218B23F020
:10213800020321F0730109041B04090C1B0C41F074
:10214800600180B243EA0803A0802183A786238424
:10215800238B23F008031B041B0C43F00803238381
:10216800B4F844306FEA43436FEA53439BB2A4F890
:102178004430DAF8A83F43EA0803CAF8A83F5046B3
:102188000DF040FA4A4BDDF808C0139380231893EA
:102198004FF48073CDF850B019934FF0100B4FF4F3
:1021A8000053504631461C9317971A971B971D9753
:1021B800CDF854B0CDF858C00DF006FAA3890BA895
:1021C8009BB243F40073A381DAF8003043F00203B2
:1021D800CAF800308DF82CB08DF82D808DF82E704F
:1021E8008DF82F8010F092FA324B1A68324B43F870
:1021F800292009F10109B9F1200FF5D10DF066FE8A
:102208000DF064FE2B685A0540F193802B4C2C4B43
:10221800D4F828850420C3F8008007F0FFFB0421C8
:10222800C4F82C0507F0D6FB264B84F830050820A7
:10223800C3F8008007F0F2FB234B0821186007F071
:10224800C9FB224F84F83105002138462C2214F0AE
:10225800B8FF8E237B704FF07C0AE0233AE000BF82
:102268005C9801088C2900202011002018100020FB
:1022780000100240B0070020000C0140000401409B
:10228800C02D0020AC070020DC19002040110020E0
:102298001414002040220020890E0020D02900209C
:1022A8000008014000366E01600000200004004074
:1022B80034040040EC9701088A0E0020D800002062
:1022C800D0190020281A0020741A0020F8190020BC
:1022D800D50200204FF07D09FB7087F800A087F831
:1022E8002B90984F2C220021384614F06AFF8A233D
:1022F8007B701020A023FB7087F800A087F82B9034
:10230800C4F8348507F08AFB1021C4F8380507F0B3
:1023180061FB84F83C052020C4F8408507F07EFB6B
:102328002021C4F8440507F055FB84F848050AF055
:102338007FFD854A00241388322023F040031B04C4
:102348001B0C138013884FF4805723F038031B04A9
:102358001B0C138013889BB243F0400313809F2308
:102368008DF82C308DF82D408DF82E408DF82F40AB
:1023780005F03BFD8DF84D40744C042267613046F2
:102388000BA910F007FA27619DF84E209DF84D30F3
:10239800120242EA03429DF84F301A436C4B9A42AC
:1023A8006C4B17D008D86C498A420CD001F51A41F9
:1023B80002318A4209D01CE068498A4205D00131BD
:1023C8008A4207D015E0202200E080221A804FF4CC
:1023D800807202E04FF480721A805A809A881988B5
:1023E80012029A604A43DA605D4A012182F849156F
:1023F80004E000221A805A809A60DA60DC6814B31C
:10240800E40AA0464FF00009A14509DA09EB0407E0
:102418007F10F802314610220DF06CFF0F2807DC00
:102428000AF050F84E4B4FEAC822C3F84C250AE090
:10243800002356F82320013254D10133042BF8D15C
:10244800B8463C46E0E72B68464A13F4002318BF19
:102458000123137005F0A2FC434B1860434B5A79D3
:102468001946052A02BF424B4FF4C8721A80414BE5
:102478004FF47A721A80404BC8221A803F4A137868
:1024880043F0080313703E4A137823F002031370D5
:1024980040F602032A6813406BB13A483A4B186079
:1024A8003A4B032018703A4B012018703948002322
:1024B800038039480380930341BF384B04221A71C3
:1024C800DA7844BF42F00102DA708B6801222B608F
:1024D800334B1A70334A137863F07F0313701FB0BD
:1024E800BDE8F08F07F101092746AAE72E4B002225
:1024F8001A7000B211F05EF82C4911F0AFF8139081
:10250800B5F95E0111F056F8284911F0A7F81490B2
:10251800B5F9600111F04EF8244911F09FF82449EB
:10252800159013A808F014FCFEF746BD4FF00208FA
:10253800FFF7A1B8012C7FF6BEA900243870FFF779
:10254800EDB800BF2D1A002000380040000C0140F3
:1025580018BA20001C000020152020001740EF00AA
:10256800D8000020FC2D0020A4080020EC11002039
:10257800CE0F00208231002080310020E019002099
:102588008B31002068130020C81900202C1A002065
:1025980054000020B8100020BA1000209029002014
:1025A800880E0020603100203C00002035FA8E3C67
:1025B800002B0020954A2DE9F04F1568944C05F53D
:1025C8009C43944E20332360336889B013F4804FC2
:1025D800059205D110F0EAFE10B923790133237171
:1025E8008D4A13784BB18D4909688D4240F2E580D8
:1025F80003F1FF3882F80080DFE09846884B5FFAE5
:1026080088F51F78DFF83892AF4231D9D9F8003011
:10261800072D98BF595D834B88BF29461B688048A2
:102628009847032D1ED8D9F8002005F10E0302EBB8
:1026380083039988DA88A8B14FF47A73401A58430B
:10264800531A90FBF3F040F6C90300F57A709842EC
:1026580005DC40F2EE239842B8BF184601E040F688
:10266800CA0080B204EB4505E88008F10108C5E717
:1026780094F804800325B8FBF5F50F2384F82A3075
:1026880094F82B3005EB4505019394F82C30C5EBF5
:1026980008050393D9F80030DFF8ACA10293EBB238
:1026A80004930025BD4255DA5F4B4FEA450933F8DC
:1026B80015B0019B53B910F079FE28B1039B002B8C
:1026C80008BF4FF0000B01E0DDF804B0029B988AC8
:1026D800584502D8D88A58450ED2E8B210F010FEF4
:1026E800032D8346DFBF94F82AE00120A8402EEA94
:1026F8000000D8BF84F82A0010F058FE18B14B48E3
:1027080029F800B022E0049B94F876002AF813B068
:1027180030B9B8F1020F15D93D4B012083F8760086
:10272800BAF80000BAF802300344BAF804000344C7
:102738003F489BB229F800301BB2032093FBF0F30B
:102748009BB200E05B46394829F8003001350AF1B0
:10275800060AA7E794F82A203648A2F10F014A4250
:102768004A4184F89020344B6AB1344A12685201C5
:1027780009D40268D9689A60521AC82A1DD9012258
:1027880083F8212019E002689868DA605B68121AF9
:102798009A4288BF284B4FF0000184F82B1088BF5D
:1027A80083F821100025BD4207DAE8B210F0A8FD31
:1027B8001E4B23F815000135F5E73368DD0405D510
:1027C8001E4B1B68D80701D410F0F8FB059B1F6847
:1027D8001B4B1A68907A002838D01449137B0138AB
:1027E80031F810001BB1C0F53B60083080B200B270
:1027F800A0F57A70B0F57A7FA8BF4FF47A7020EA16
:10280800E07010F0D7FE0F4955E000BF6C31002092
:10281800100F00209C2D0020303100202C3100208A
:10282800BC2A002034000020160F0020D82D0020DC
:10283800880F0020C02D002034310020E410002033
:102848002831002000007A443E0F00203368190424
:102858003AD5D4F89430934DFB1A002B34DB07F5A6
:102868009C432033C5F894308F4BD27A59798F4BDB
:1028780033F8113095F898109BB293FBF2F30131BD
:1028880001F00F0285F898202A4482F8993003460F
:10289800874A825C0130134410289BB2F8D11BB2DE
:1028A80093FBF0F000B26428A8BF642020EAE0702F
:1028B80010F080FE7F4910F085FF7F4910F0CEFEB2
:1028C80011F0B8F87D4B188033687D4D13F4807F84
:1028D80000F00F817B4BDFF8F0919F4205D999F802
:1028E800022012B9012289F8022099F80220002A50
:1028F80000F0FF80744A95F8008092F82170C8F3C0
:1029080080087A1E57425741704A002F9246116834
:1029180018BF4FF0000BC1F38063019308BF4FF05D
:10292800030B99F82020052A00F2DD80DFE802F089
:10293800034E537988A5B8F1000F3AD0D4F8AC000B
:10294800B4F8B01007F007F9012809D16049614AC5
:1029580009681268C988642000FB0122C9F81020A0
:10296800019B6BB15A4A126812794AB10BF04EFEBC
:10297800032289F820204FF47A72C9F81C20D0E786
:10298800002F40F0B080534AD9F8101010684E4A12
:1029980088420AD902920BF039FE029A032182F882
:1029A800201040F6B831D161BBE7012182F8201030
:1029B800B7E7019B4FF4806013B108F0A1FA01E07A
:1029C80008F08DFA0022C9F810208CE0002F49D1B8
:1029D8000BF01CFEA5E727B1052289F8202001206D
:1029E80000E03846B8F1000F0CD0D4F8AC204FF016
:1029F800020BD189384A1180518091803449096885
:102A08004988D180334A1168D9F81420914202D8F4
:102A1800B8F1000F64D147F23052C9F81C200322E4
:102A280021E02A7842F002022A7010F0C7FA294AF7
:102A3800D9F81C1012680A44C9F81820042212E0B8
:102A4800244A9FB11168D9F8182091424BD9234ADA
:102A580012781AB9DAF80020D30744D42A7822F079
:102A680002022A70052289F820205AE71268D9F84C
:102A78001C100A44C9F8182035E01549154A096898
:102A88001268C988642000FB01224FF48060C9F8ED
:102A98001020002289F8202089F8032008F01FFA66
:102AA8003FE700BF100F0020242B0020342B00200C
:102AB800A90F00200000C84200C07F444411002034
:102AC8008B310020404B4C0034310020E4100020B2
:102AD80088290020C02D0020D82D002018000020B3
:102AE80000287FF41EAFBBF1000F02D0584605F056
:102AF800B3F9934F07F5C570B7F8521107F02BF8E3
:102B08000197834668B90BF073FD8E4B0022C3F81A
:102B180000B0C3F804B0C3F808B08B4B1A605A6011
:102B28009A602B785F0736D53368D80633D5874B3C
:102B38001B78D9062FD4864B1B789BB1019B93F841
:102B4800E231BBF1000F15D17BB1824B1A68D4F882
:102B5800B4309B1A002B08DA10F030FA7E4B83F859
:102B6800B8B018E0BBF1000F0DD1102005F074F9D2
:102B780001230EE03BB1774A4FF47A71126801FBEA
:102B88000323C4F8B43094F8B83023B105F04CF9F5
:102B9800002384F8B830019B93F8E0A193F8E11181
:102BA800B3F89AE1B3F89CC1002318466B4F80082C
:102BB80037F9132001337245C4BF60F07F00C0B2FB
:102BC8006245B8BF40F04000042BB946EED194F8F6
:102BD800B930614A834205D192F8BA30F92B04D84A
:102BE800013300E0002382F8BA30594B84F8B90069
:102BF8001A785B4F9846E2B93B68DA0708D5BBF10B
:102C0800000F16D12B78DB0713D510F029F810E048
:102C18002B7858070DD5504B93F82B304BB1514BAF
:102C2800DB7833B911B110F0C9F902E0BBF1000F3C
:102C3800F9D094F8BA30484A142BDFF83CB140F088
:102C4800AD8098F800301AF1000A18BF4FF0010A59
:102C58006BB392F8B9305F2B11D12B7803F00403D2
:102C680003F0FF0113B110F0A9F908E00B2003915C
:102C7800029205F0F1F8029A039982F8BA10BAF1B3
:102C8800000F14D094F8B9307D2B10D12B7803F0B5
:102C9800040303F0FF0213B110F090F907E00B20D2
:102CA800029205F0D9F82C4B029A83F8BA202B78B7
:102CB80003F0040303F0FF01002B6FD194F8B9303F
:102CC800254A572B15D1284B4FF47A721A8033684E
:102CD800190601D509F094FA244B1B685A0742BF1C
:102CE800234A0A21118013F0080357D1214A13807F
:102CF80054E03068400717D55A2B15D192F8BB30ED
:102D08002BB1012382F8BB1082F8BC3046E092F860
:102D1800BD3083F0010382F8BD300BB10C2000E018
:102D28000D2005F099F839E05D2B00F018855B2B34
:102D380000F017855E2B21D1032000F013BD00BFE2
:102D4800EC110020C81A0020441B0020E0190020C4
:102D580018000020C02D0020100F0020D82D0020C2
:102D6800E41000203431002082310020DC190020DA
:102D780080310020DC11002020110020562B01D1C9
:102D880008F06AFB98F80030002B00F0018594F8F1
:102D9800B9306F2B40F0F6840FF062FF33685807A4
:102DA80036D594F8BD30B64A93B12B7859070FD56C
:102DB800019BB9F90610B3F89A31994208DD3B68CE
:102DC80013F0010302BF3221A2F8C01082F8BD300F
:102DD8003B68DA030DD594F8C220A94B2AB993F8B9
:102DE800BB2012B93222A3F8C020012384F8C230D4
:102DF8000EE094F8BB30A24A53B12B7803F00403D9
:102E080003F0FF0123B9012382F8BB1082F8BC301C
:102E1800DBF8009000233B6009F17B0809F1CB0A3D
:102E280098F8002098F8013018F8010C9A420BD253
:102E3800414606F05BFE38B118F8022C012303FA6C
:102E480002F23B6813433B6008F10408D045E7D120
:102E58008C4B1B7853B18C4B8C4F1A68984612F0E8
:102E6800020FDFF8409240F032832AE309F1CA07E3
:102E780009F589783A787B7817F8010C9A4225D2B7
:102E8800394606F033FE08B397F804E00C21BB7806
:102E980001FB0E417E4A013B03EB43031344D1F887
:102EA800C82097F803909A4275480FD0C1F8C830E7
:102EB800002390F8F420C1F8CC30012303FA0EF374
:102EC80022EA030381F8C49080F8F43006374745B6
:102ED800D0D1704BDFF8D0A1D3F800806E4B4FF003
:102EE800000B1B68029394F82B300393DAF8003038
:102EF800002B00F0DD8293F80090B9F1000F00F08C
:102F0800D782DAF8042002998A1A002A0CDB01F524
:102F1800FA72CAF8042094F8F410012202FA0BF2AB
:102F280021EA020284F8F420039A002A00F0C08201
:102F38001AF8042C59780432D2B2002940F0798268
:102F4800564931F91210564AB2F8982102F1C800D0
:102F5800814201DD9F7814E0C83A914202DA9978FB
:102F68004F420EE094F8F420012303FA0BF322EA0F
:102F7800030384F8F430029B03F5FA73CAF80430AB
:102F880096E294F8F43043FA0BF3DB0700F19082F1
:102F9800002FCCBF0220012004F084FF09F1FF328A
:102FA800374B132A00F27C82DFE812F0140023006A
:102FB8003200440061008000E5004A01AF01E401ED
:102FC80013027A02440055008000E5004A01B70068
:102FD8001C01810198F8001040460F44FA2FA8BF41
:102FE800FA2727EAE77788F8007006F065FD0120E0
:102FF8001EE098F8011040460F44642FA8BF6427CC
:1030080027EAE77788F8017006F056FD02200FE0FE
:1030180098F8031040460F44642FA8BF642727EA96
:10302800E77788F80370D3F8F81006F0FDFC032062
:103038003946CBE198F805100D2039446429A8BF1A
:10304800642121EAE17188F8051004F093FEB9F1D2
:103058000D0F00F0258298F804100E2039446429D9
:10306800A8BF642121EAE17188F80410AEE198F85C
:1030780006100520394481F3080188F80610A5E1F7
:10308800100F00208C310020E4100020DC190020F3
:10309800A099010848110020C02D0020D82D00203B
:1030A800EC110020A41A0020D80F0020D3F8FC301F
:1030B8001A78022A22D13846049310F07BFAA949DB
:1030C80010F080FB049B596A059310F0BFF90021AA
:1030D800049010F061FC059B48B9049AA249104677
:1030E80010F078FC049A059B10B19F4A00E000227A
:1030F8005A620F20114604F029FE0AE099780F2041
:103108003944C829A8BFC82121EAE171997004F09F
:1031180031FEB9F10F0F00F0C381944BD3F8FC9046
:1031280099F80030022B1AD1384610F043FA8D492D
:1031380010F048FBD9F8201010F088F90021074654
:1031480010F02AFC30B93846874910F043FC10B11A
:10315800854F00E00027C9F82070122059E199F83E
:10316800011012203944C829A8BFC82121EAE171F9
:1031780089F801102AE1D3F8FC301A78022A22D102
:103188003846049310F016FA774910F01BFB049B9D
:10319800196B059310F05AF90021049010F0FCFB0C
:1031A800059B48B9049A7049104610F013FC049A1C
:1031B800059B10B16C4A00E000221A6310201146EA
:1031C80004F0C4FD0AE0197B10203944C829A8BFBF
:1031D800C82121EAE171197304F0CCFDB9F1100F8F
:1031E80000F05E81614BD3F8FC9099F80030022B17
:1031F8001AD1384610F0DEF95B4910F0E3FAD9F835
:103208002C1010F023F90021074610F0C5FB30B947
:103218003846554910F0DEFB10B1534F00E0002747
:10322800C9F82C701320F4E099F80B1013203944D6
:10323800C829A8BFC82121EAE17189F80B10C5E0A7
:10324800D3F8FC301A78022A22D13846049310F0B9
:10325800B1F9474910F0B6FA049BD96B059310F001
:10326800F5F80021049010F097FB059B48B9049AE3
:103278003D49104610F0AEFB049A059B10B13A4A3E
:1032880000E00022DA631120114604F05FFD0AE035
:10329800997D11203944C829A8BFC82121EAE171C4
:1032A800997504F067FDB9F1110F00F0F9802F4B03
:1032B800D3F8FC9099F80030022B1AD1384610F058
:1032C80079F92B4910F07EFAD9F8381010F0BEF8C9
:1032D8000021074610F060FB30B93846224910F04B
:1032E80079FB10B1204F00E00027C9F8387014208E
:1032F8008FE099F8151014203944C829A8BFC821AF
:1033080021EAE17189F8151060E0D3F8FC9099F88A
:103318000030022B1AD1384610F04CF9114910F040
:1033280051FAD9F8281010F091F80021074610F04A
:1033380033FB30B938460C4910F04CFB10B10A4F3A
:1033480000E00027C9F82870092062E099F8031006
:1033580009203944C829A8BFC82121EAE17189F8A0
:10336800031033E0000020410000C842100F002085
:1033780000007A44D3F8FC9099F80030022B1AD157
:10338800384610F017F9B44910F01CFAD9F834107F
:1033980010F05CF80021074610F0FEFA30B9384604
:1033A800AD4910F017FB10B1AB4F00E00027C9F88A
:1033B80034700A202DE099F80D100A203944C829E4
:1033C800A8BFC82121EAE17189F80D1004F0D2FCE8
:1033D80066E0D3F8FC9099F80030022B1DD13846EE
:1033E80010F0E8F89D4910F0EDF9D9F8401010F008
:1033F8002DF80021074610F0CFFA30B93846964923
:1034080010F0E8FA10B1944F00E00027C9F84070B6
:103418000B20394604F09AFC42E099F817100B206B
:103428003944C829A8BFC82121EAE17189F81710D1
:10343800CCE7012934D19878894B33F91230B3F5A8
:10344800617F05DB40F633029342A8BF134601E0D3
:103458004FF46173B9F10C0F22D14FF4966292FBCD
:10346800F0F0A3F5617393FBF0F37E4ADFB21378B3
:10347800BB4215D0042F34BF3B4602231370019A78
:1034880009FB0323784A03F2B27313600DF039FF86
:103498004846394604F06EFC781CC0B204F002FDC0
:1034A80094F8F420012303FA0BF3134384F8F4305F
:1034B8000BF1010BBBF1040F0AF10C0A7FF416ADF6
:1034C800C9E43368D80510D5684BDB786BB13B6825
:1034D80099070AD5B9F8003013F0010A0AD10BF0A0
:1034E80087F8012007F00CFD04E0012007F0F7FC45
:1034F800012300E00023D8F8002052070DD563B15E
:10350800012007F0ECFCB9F800309B0708D40BF059
:103518006FF8022007F0F4FC02E0022007F0DFFC5D
:10352800B9F80030524A13F0030F4FF0100114BFDE
:10353800516111613A6812F00A0F27D0D8F80020BB
:10354800D00609D559070AD4042007F0D9FC494BFD
:103558001B88A4F8003102E0042007F0C0FCD8F86A
:1035680000309A0607D5B9F800305B0606D440202B
:1035780007F0C6FC02E0402007F0B1FCD8F80030A4
:10358800580642BF3B4B1B88A4F802313B6899069A
:1035980009D4D8F800301A0540F1B0804FF4807093
:1035A80007F0AEFCAEE0344B1B789B076ED5334B6F
:1035B8001B78042B6AD9D8F8003013F4007A0FD09E
:1035C800B9F80030DF063AD4102007F099FC202023
:1035D80007F085FC2A48011D08F07CFD02232AE03B
:1035E800B9F8007007F01007BFB22FB1102007F02C
:1035F80076FC012784F804A1D8F80030580512D5C4
:10360800D4F808311F495A89B1F90030002BB8BFE6
:103618005B42934207DAB1F90230002BB8BF5B4234
:103628009342C0F20881B9F80030990608D52020E5
:1036380007F055FC002384F80431012700E0002737
:1036480094F80C319BBB0E2004F006FC0E4B0122B3
:1036580083F80C212BE000BF0000C84200007A4428
:10366800D82D0020482D002048110020343100209A
:10367800000C0140DC110020E0190020E6190020B0
:1036880050110020E4110020100F0020B9F800307C
:1036980003F03003002B3FF47CAF102007F01FFC31
:1036A800202007F01CFC002384F8043102E0002FDE
:1036B8003FF46FAF002214466B4B002023F8140030
:1036C8006A4B191D03F10A0721F814000021D15192
:1036D80017447860B96023F8140003F132075A33AD
:1036E800D151D150174413447860B960586099603B
:1036F8001432002C7FF44DAF0124DDE74FF48070C5
:1037080007F0EDFB5A4B5A791C46082A01D00E2ABD
:1037180002D1402007F0E3FB33685A0540F1A1804D
:1037280094F818321BB92B7813F0040F03E0D8F87B
:10373800003013F4002F0BD04E4B00221A703C209F
:103748000BF010FF002800F08C800EF0E5FCF6E787
:1037580009F06EFB09B0BDE8F04F0BF032BE012056
:1037680000E002205FFA80F8019A08F1FF3382F83E
:10377800B03707F007FC07F0ABFC404604F092FBBB
:10378800FFF70CBBBAF1000F02D07E2B3FF404AB5D
:1037980094F8B930972B06D1374B4FF4C872A3F879
:1037A800BE20FFF7FBBAA72B06D1344A137843F0A3
:1037B80004031370FFF7F2BA0022BB2B079201D162
:1037C800022303E0B72B04D14FF6FE73ADF81E3089
:1037D80009E0BE2B01D1022303E0BD2B1AD14FF61D
:1037E800FE73ADF81C30DBF80030BDF81C10B3F8E0
:1037F80058200A44A3F85820BDF81E10B3F85A20E0
:103808000A44A3F85A2007F027FE002384F8BA30A8
:10381800FFF7C4BA792B04D1194AD37823F00103EE
:1038280006E07A2B7FF4BAAA154AD37843F001034D
:10383800D370FFF7B3BAB9F800309B063FF500AF75
:10384800202007F05DFB0F4B0F481A685B68011DCD
:103858004360026008F03EFC074B012783F80471BF
:10386800EEE609B0BDE8F08F843100201E1000207C
:10387800EC110020C12A0020100F0020E0190020C0
:1038880090290020E819002058110020B54B2DE997
:10389800F04FB3F90610B44B85B01F6801937A89CD
:1038A80091420EDBB1F5FA6FFC79BFBF8B1A634307
:1038B800A2F5FA6493FBF4F4ACBFC4F16404643475
:1038C80000E06424A94BAA4AB3F898B193F962318D
:1038D80012689BB2029215460393002240F2E6302A
:1038E800A04B4FEA420C33F912E0CBEB0E0303F284
:1038F800F316864203D8002BB8BF5B4201E04FF4B1
:10390800FA73022A2ED0029E96F811611EB1B342B4
:10391800CCBF9B1B0023642093FBF0F8954E6FF0FF
:10392800630A36F818900AFB083A08F1010836F9D4
:1039380018600FFA89F8C8EB060606FB0AF696FB2C
:10394800F0F68D484E4420F80C60BE183679642095
:1039580073438A4E93FBF6F364339BB2634393FB42
:10396800F0F02CE0029890F812611EB1B342CCBF7F
:103978009B1B0023642093FBF0F0DFF82C926FF080
:10398800630808FB003A39F91060013039F9100072
:10399800002BA0EB060000FB0AFA9AFBF8FA039842
:1039A800C6EB0A0A0AFB00FA7348B8BF5B42A0F8E4
:1039B80004A0B8794343714893FBF0F064306B7806
:1039C8004FF06408434393FBF8F36D4E022AB35457
:1039D800EB7A6C4E00FB03F393FBF8F3B3546B7D67
:1039E800654E00FB03F090FBF8F0674B9854674B6B
:1039F8000ED1DE4583F802800DDB5C4CB4F89A21C9
:103A0800914214DBB1F5FA6FA8BF4FF4FA610FE0E9
:103A1800DE459C5404DA36F80C305B4226F80C304C
:103A28000132032A05F101057FF458AFE5E7114695
:103A3800891A4FF47A735943C2F5FA62B1FBF2F16D
:103A4800642391FBF3F2DFF874E16FF063073EF84B
:103A5800120007FB021101323EF9122007B2D21BF5
:103A6800514391FBF3F30344F380494B424D1B88C8
:103A78005F063BD5474A484B10881B88181A00B286
:103A88000FF098FD45490FF0E9FD074607F056F994
:103A98008046384607F0DFF80746B5F902000FF010
:103AA80089FD8146B5F900000FF084FD4146824644
:103AB8000FF0D4FD3946834648460FF0CFFD014646
:103AC80058460FF0C1FC0FF08FFF4146288048464A
:103AD8000FF0C4FD3946804650460FF0BFFD014641
:103AE80040460FF0B3FC0FF07FFF68802C4D2B6829
:103AF800980740F19E8045F207212A4B2A4F1A6801
:103B08007B69D31A8B4240F394807A610CF004F9F4
:103B1800264BDFF8AC901A789846032AB9F800309B
:103B280050D10A2B58D90023282088F8003004F0F7
:103B38005CF90CF0F1F81E4B18880CF0D7F81D4B07
:103B48001A68D37890FBF3F0013008281A4BA8BF05
:103B580008201870537980B243433B831379584344
:103B6800788339E0D82D002048110020EC1100207E
:103B7800201100205E220020E41100200CFEFFFF2F
:103B8800501B0020AE100020641B0020A81A002043
:103B9800A41A002012100020DC11002035FA8E3CF7
:103BA8009C2D00206C310020A01000202C1A002031
:103BB8003C2B0020C8190020540000204622002079
:103BC800CC1900200A2B07D803239C4A88F8003018
:103BD800002313703B837B8398F80030984A012BAD
:103BE8000CD002D3022B1BD023E03A8BB9F800305B
:103BF8009A421EDD012388F800300FE0B9F8001062
:103C08007B8B8B4202DD022313700FE08D4B1B8BE5
:103C18000133994202DD002313700AE0082006E010
:103C28007B8BB9F8002001339A42E3DC072004F0CB
:103C380013F92D68290577D5834B824F1A68FB69DC
:103C4800C3EB020845F2072398456DDD7F4BB6F9B3
:103C580006B0D3F800904FF47A7099F80A30FA61F8
:103C6800012B98FBF0F8B4F85211ABF57A7B784E3B
:103C780003D042D3022B20D041E0764B396A5A7BDD
:103C8800754B4FF0080E33F8122091FBFEF392B2F9
:103C9800C91A8B183B6293FBFEF3BA8440F6E442E0
:103CA8009BB25343B9F80820C2EB13335843B9F910
:103CB800063090FBF3F0306021E0684BB9F808A0BB
:103CC8001B78C6F800A05A0719D5654805F043FFC8
:103CD80020B915F0100F18BF4FF0000B0BFB0BF3BA
:103CE800322293FBF2F3B9F906205B445A434FF4AE
:103CF8007A7392FBF3F3534400E000233360336894
:103D0800D7E90A0103FB08F84FF47A7398FBF3F834
:103D180010EB080041EBE8710023C7E90A01514A9A
:103D28000FF0A8FE504B1860504E3368DB0427D5BF
:103D38002F0622D54E4B1B789D071ED54D4B187864
:103D480004281AD900224C4B0521D718951C4FF08E
:103D58000A0E122AD154E9B287F801E004D0B0EB78
:103D6800510F2A46EFD800E014215A18322002F8E1
:103D7800010CFF225A540F2000E00A2004F06CF8CE
:103D88003E4D2A68002A51D03D4B3E4F186839688D
:103D9800984681424AD83C4BDFF8F8901978526827
:103DA800E1B94FF0010A83F800A0B9F80030D35CFC
:103DB80023B3504604F032F8344B83F800A00FF0D8
:103DC80001FBB9F80030CBB92B681B78053B53458C
:103DD80014D803F0E3FF2E4B18600FE04FF0000AF1
:103DE80083F800A0B9F80030D35C3BB1504604F02A
:103DF80015F8264B83F800A00FF0E4FA2B68B9F801
:103E080000205B6823499B5CFE2B02D100230B80BA
:103E18000CE0FF2B02D104F007F807E0D8F8000007
:103E28000A2505FB030301323B600A800B4D2B7802
:103E3800580733D5184B08225A616DE0540000200A
:103E48002C1A0020A01000206C310020C819002076
:103E5800D4190020242B0020342B00208B31002083
:103E680076130020407E0500D8190020E4100020B9
:103E7800E0190020E6190020742D00207C1B00208A
:103E8800C02D0020741B0020701B0020583100201A
:103E9800B82F0020781B0020000C01403268D107A1
:103EA8005CBF43F001032B70984B1B781F075EBF64
:103EB8002B7823F001032B70D60248BF2B78944A45
:103EC80044BF23F001032B70924B1B6813F0040FBF
:103ED80002D09149098851B99049098809B19807D0
:103EE80005D48F4B1B88003318BF012333B102233D
:103EF80013702B7823F001032B7004E02978C9078D
:103F080058BF0223137003F049FF864B1B68C01A81
:103F1800002801DB0FF056FA08F08AFF824B1E7862
:103F28009846002E00F0AB80804E3368002B00F0DE
:103F3800F186306804F024F8002800F0EB867B4B0B
:103F48007B4C186804F019F8092801D03F2850D193
:103F58004FF0000A5746D4F80090764DB9F1000F9B
:103F680005D0754829684A4613F078F910B9AA4669
:103F780007B92F46714B10359D42EFD3C7B1D7F81B
:103F880000E0DAF800C023681EF803501CF80300AC
:103F9800A8420DD15A1C684938B92D2B05D8644D53
:103FA8002A602025CD54885402E0CD542260EAE7E7
:103FB80023680BB1574511D061480EF09DF957455C
:103FC80007D857F8100B0EF097F909200EF08CF966
:103FD800F5E75C480EF090F94FF000092368994521
:103FE800A7D2554B13F809000EF07EF909F1010923
:103FF800F4E72368002B40F07286042840F0B0866E
:104008004D480AF071FC00F085BED9F80000DFF8D1
:1040180044A103F0B5FF40B3DAF8000003F0ADFFA8
:10402800DBF80030024693F84810002935D12428DF
:1040380040F09280012283F84820DBF80030DFF856
:1040480010A193F84820062ADFD193F8490000F020
:1040580013FF8146002800F0AA803B6898790EF08B
:1040680098F83B68002283F84820374B93F835309E
:10407800002B40F022864C36982E00F04B86334BAE
:10408800F21892F84A100129F5D1314FF3583A60E5
:10409800304ABB4613609146B7E7012904D14D2841
:1040A80014BF00220222C6E7022904D13C2814BF0B
:1040B80000220322BFE703290CD140284FF000015A
:1040C80002D983F84810B8E758711971D9719871F5
:1040D8000422B0E7042906D1997983F849004A40B7
:1040E8009A710522A7E70529A7D158791979884235
:1040F800987906D950409871481C18710B441A7267
:104108009BE790420CBF0622002294E7E0190020AA
:1041180058310020DC19002080310020CE0F00200B
:10412800823100205C3100208C310020642D002079
:10413800CC29002000A101089C290020D0A2010858
:1041480047BC01084CBC0108A0100020202A002010
:10415800841A0020881A00202B78B74958073FF5A1
:104168006CAF232ADAF8003014D1012088F8000057
:10417800B24803910360B24802920363B1480EF05B
:10418800BBF8B1480EF0B8F80399029A0B7843F0DF
:1041980002030B70AD4B1B681B78934201BFAC4AFE
:1041A800AC4B1A60AC4A04BFAC4BDA6045E7DAF8AE
:1041B800002092F849304A2B00F038815CD8332B24
:1041C80000F0A18421D8292B00F03B8409D8252BA5
:1041D80000F01284272B00F01684232B40F0BC85B6
:1041E8003FE22D2B00F03E8407D82B2B40F0B485FE
:1041F8000DF0B2FF607100F05BBD2F2B00F00B8556
:10420800312B00F01D8500F0A7BD3E2B00F0048186
:104218001DD8372B00F0C78404D8352B00F05A82FC
:1042280000F09ABD392B00F0FB833C2B40F09485BD
:10423800DFF82C92D9F800A00DF08EFF8AF8000064
:10424800D9F80030187804F00BF900F031BD432B91
:1042580000F0868406D8412B40F07E854FF0000997
:1042680000F056BC442B00F01F85482B40F07485A5
:1042780008F066F900F01CBDD02B00F0368368D832
:10428800CA2B00F0F5801CD84E2B00F00E8410D8F5
:104298004C2B40F061850DF05FFF84F8D8010DF0DC
:1042A8005BFF84F8D9010DF061FFA4F8DA0100F092
:1042B800FFBCC82B00F08380C92B00F0378300F0C7
:1042C8004BBDCD2B00F01C8304D8CC2B00F02A82E8
:1042D80000F042BDCE2B00F01C83CF2B40F03C8574
:1042E8000DF044FF6FF4AF6283189BB2C62B98BFE2
:1042F800A4F898010DF03AFFA4F844010DF036FF38
:10430800A4F846010DF032FFA4F848010DF02EFF85
:10431800A4F8DA010DF020FF84F8EF010DF01CFF7E
:104328000DF01AFF84F8F0010DF016FF84F88701EC
:104338000DF012FF84F894010DF00EFF484BD3F8EE
:1043480000900DF013FF00EB80004000A9F8560024
:1043580066E3D62B00F04E820AD8D22B19D0C0F0D3
:104368000C83D32B25D0D42B00F04F8200F0F4BC63
:10437800EF2B41D005D8D82B40F0EE844FF0000940
:1043880002E1F22B00F08982FA2B00F0CB8200F0D8
:10439800E3BC2B78590700F18B840DF0DDFE022871
:1043A80084F8B00740F2A7822E4B002283F8B0278A
:1043B800A1E20DF0DBFE2C4B188000F079BC92F8DE
:1043C80005904FEA5909B9F1120F03D90BF0C6F855
:1043D80000F06EBC4FF0000ACA4507D20DF0C6FEC9
:1043E800224B23F81A000AF1010AF5E7144B0122BF
:1043F80083F8342000F05CBCDFF86490D9F800A0A2
:104408000DF0B4FEAAF85A00D9F800900DF0AEFEEF
:10441800A9F8580000F04CBC0DF09EFE84F8E201AB
:104428000DF09AFE84F8E10100F042BC0DF09EFE0A
:10443800A08100F03DBC00BF8B310020642D00201E
:10444800A01000207CBC01084CBC0108C42A002034
:10445800EFBEADDEF04F00200400FA0500ED00E0ED
:1044680020110020EC11002010100020D82D002071
:10447800D64B1A689A461278022A6AD1DAF80030BE
:1044880009F1080B02930DF067FE0FF08FF8D04981
:104498000FF098F9029B43F82B00DAF800B00DF002
:1044A8005BFE09F10A030BEB830B0FF07FF8C94998
:1044B8000FF088F9DAF80030CBF8040002930DF019
:1044C8004BFE0FF073F8C4490FF07CF909F10E0B9D
:1044D800029B09F10109B9F1030F43F82B00CDD173
:1044E800B9F1070FDAF800B01AD10DF035FE0FF068
:1044F8005DF8B7490FF066F9CBF84400DAF800B078
:104508000DF02AFE0FF052F8B1490FF05BF9CBF825
:104518004800DAF800B00DF01FFE8BF84C0012E0EE
:104528000DF01AFECB448BF80100DAF800B00DF05C
:1045380013FECB448BF80B00DAF800B00DF00CFE3C
:10454800CB448BF8150009F10109B9F10A0FC7D15D
:10455800AEE3DAF800B00DF0FFFDCB448BF80100B4
:10456800DAF800B00DF0F8FDCB448BF80B00DAF860
:1045780000B00DF0F1FDCB4409F10109B9F10A0FC2
:104588008BF81500E5D193E3DFF840A209F1080B99
:10459800DAF8003002930DF0E9FD0FF007F88E49C4
:1045A8000FF010F9029B43F82B00DAF800B00DF079
:1045B800DDFD09F10A030BEB830B0EF0F7FF8649CB
:1045C8000FF000F9DAF80030CBF8040002930DF090
:1045D800CDFD0EF0EBFF80490FF0F4F809F10E0B5A
:1045E800029B09F10109B9F1030F43F82B00CBD164
:1045F800B9F1070FDAF800B01AD10DF0B7FD0EF0D7
:10460800D5FF75490FF0DEF8CBF84400DAF800B0B2
:104618000DF0ACFD0EF0CAFF6F490FF0D3F8CBF8E0
:104628004800DAF800B00DF0A1FD8BF84C0012E05C
:104638000DF09CFDCB448BF80100DAF800B00DF0CA
:1046480095FDCB448BF80B00DAF800B00DF08EFD29
:10465800CB448BF8150009F10109B9F10A0FC7D14C
:1046680026E30DF079FD132883463FF6AFAEDFF859
:104678005CA1DAF800900DF06FFD002357490C2279
:1046880002FB0312117A814220D1137809EB8B09BE
:1046980089F879300DF060FD89F87A000DF05CFD3D
:1046A80089F87B000DF058FD4D4A4E4B89F87C0087
:1046B8001A60DAF800004C4B00211860793005F0D8
:1046C80039FA4A4B80F001001870F1E201331C2BD3
:1046D800D4D17BE60DF040FD0B2882463FF676AE3E
:1046E8003A4BD3F800900DF037FD03283FF66EAE35
:1046F800062303FB0A9989F8CE000DF02DFD89F8F1
:10470800C9000DF029FD89F8CA000DF025FD89F8CA
:10471800CB000DF021FD89F8CC000DF01DFD89F8C6
:10472800CD00C5E25379092B7FF650AE019BD3F833
:1047380000900DF011FD019B89F80000D3F800905E
:104748000DF00AFD89F801000DF006FD019B6428B3
:104758001B68A8BF642018710DF0FEFC019B64283B
:104768001B68A8BF642058710DF0F6FC019BFF2858
:104778001B68A8BFFF2098710DF0EEFC019B642810
:10478800D3F8009028BF642089F807000DF0E4FCF6
:10479800019B89F80200D3F800900DF0DDFC019B25
:1047A80089F80300D3F800900DF0E0FC3B68A9F805
:1047B8000A005B790A2B40F27B820D4BD3F80090FC
:1047C8000DF0CAFC89F8080072E200BF2011002031
:1047D800000020410000C84200007A440C9A0108F9
:1047E80030130020081000200C10002018000020B2
:1047F800481100200DF0BAFCCB4B23F8190009F141
:104808000109B9F1080FF5D152E253790F2B7FF462
:10481800DDAD0DF0A1FC072881463FF6D7ADDFF8E6
:1048280034A3DAF800B00DF0A1FC0E2303FB09F95C
:10483800CB44ABF81901DAF800B00DF097FCCB4483
:10484800ABF81B01DAF800B00DF090FCCB44ABF8E4
:104858001D01DAF800B00DF07FFCCB448BF81F0186
:10486800DAF800B00DF078FCCB448BF82001DAF8C8
:1048780000B00DF071FCCB448BF82101DAF800B0E0
:104888000DF06AFCCB448BF82201DAF800A00DF099
:1048980077FCD144C9F823010AE20DF05DFC0F282A
:1048A80081463FF693AD0DF057FCC9EBC909A14409
:1048B80089F8D4000DF050FC89F8D5000DF04CFCB7
:1048C80089F8D6000DF048FC89F8D7000DF044FCB3
:1048D80089F8D8000DF040FC89F8D9000DF03CFCAF
:1048E80089F8DA0003F00EFDE2E12B785B0700F1AE
:1048F800DF810CF04BFD06F045FB06F0E9FBD7E144
:104908002B78580700F1D481884B4FF4C8721A806D
:10491800CEE12B78590700F1CB81854A137843F013
:10492800040328E02B785A07E5D515E20DF014FCAE
:104938007F4B1A7810B142F0020201E022F0020225
:104948001A700DF009FC7B4BDFF80C9218700DF013
:1049580017FCC9F800000DF013FCC9F804000DF0AD
:1049680005FC754B18800DF001FC744B744A1880D7
:10497800137843F0020313709AE10DF0EDFB0290F7
:104988000DF0FEFB83460DF0FBFB82460DF0F8FBB5
:1049980081460DF0EBFB0DF0E9FB0DF0DDFB029B12
:1049A800A3B9684B1020C3F800B0C3F804A006F000
:1049B80096FA5F4A137843F001031370B9F1000FB8
:1049C80000F07681604BC3F8009071E1102B40F045
:1049D8006F815E4BC3F800B0C3F804A0B9F1000FB3
:1049E80002D0594BC3F800905848594B0222011D78
:1049F8001A7007F06FFB5BE1A0600DF0C1FBA368C4
:104A08001843A06054E10DF0B1FBA4F85C010DF06F
:104A1800ADFBA4F85E010DF0A9FBA4F8600147E125
:104A28000DF09AFB84F87C010DF096FB84F8800168
:104A38000DF092FB84F87F010DF08EFB84F8810164
:104A480036E10DF093FBA4F882010DF08FFBA4F87A
:104A580084010DF081FB84F886010DF087FBA4F832
:104A6800880125E10DF078FB84F892010DF07EFBBA
:104A7800A4F89C010DF07AFBA4F898010DF076FBE0
:104A8800A4F89A010DF068FBDAF8003084F8930175
:104A98005B79082B40F20C810DF068FBA4F89E01AD
:104AA8000DF064FBA4F8A00102E192F8059003233D
:104AB800B9FBF3F9B9F1120F3FF688ACDFF89CA007
:104AC8004FF0000BCB4580F0F3800DF045FB8AF8E2
:104AD800A2010DF04BFB40F2ED23984205DD40F6B4
:104AE800CA039842A8BF184601E040F2EE20A0F29F
:104AF800EE20192390FBF3F00BF1010B8AF8A301C8
:104B08000AF1020ADEE70DF027FB84F89401CFE0F2
:104B18000DF022FB04EB090309F10109B9F1080FB3
:104B280083F88A01F4D1C3E04A2D0020CE0F00207B
:104B3800E0190020E6190020E4190020E2190020FD
:104B48004E11002050110020601100205811002043
:104B58001410002020110020E8190020EC1100207A
:104B68000DF0FAFAC4F8089060710DF009FBA3681B
:104B78001843A0600DF0F0FA84F892010DF0F6FAEF
:104B8800A4F85C010DF0F2FAA4F85E010DF0EEFA5B
:104B9800A4F860010DF0EAFAA4F882010DF0E6FA33
:104BA800A4F8840184E053794FF0070AB3FBFAF2C2
:104BB800C2EBC2029A1A12F0FF0F7FF407ACB3FBE4
:104BC800FAFA0AF1FF3A5FFA8AFABAF1FF0F6FD0E0
:104BD8000DF0C2FA5FFA80FB4FFA8BF004F044FE46
:104BE800814600283FF4F2AB80F800B00DF0BEFA21
:104BF800A9F802000DF0B0FA89F804000DF0ACFA3B
:104C080089F805000DF0A8FA89F807000DF0A4FA54
:104C180089F80600D5E7DFF85C9209F1400A0DF043
:104C2800A5FAA9F8A8020DF097FA89F8AA020DF0DA
:104C380093FA09F1040989F8A702D145EFD137E0C1
:104C48000DF08AFA1F2881463FF6C0AB3B685B79B6
:104C5800082B7FF4BBAB0DF089FA09F18A0904EB44
:104C6800890A00F03F00AAF802000DF07FFABAF8AE
:104C78000230800100F4FE501843AAF802000DF03B
:104C88006BFA000104F829000DF066FA14F82930CF
:104C980000F00F00184304F829000DF05DFA8AF8B7
:104CA80001000BF057FF03E05F4B012283F835202A
:104CB80000200DF09DFAFFF7D0B95C4B985903F02E
:104CC80056F918B9322003F090F8F6E703F0DAFA4B
:104CD80006F02EF9564A574BDA60FFF7CCB90C2884
:104CE80040D00A2847D1544D54480DF005FB2846BA
:104CF800232112F09CFA08B1401B20602368002B86
:104D08005CD14D4800213022236012F05AFA98F8FD
:104D1800003053BB4A4B1B689B0614D5494B42498C
:104D28001B688A6B9A1A002A0DDB474A1278042AF4
:104D380009D903F5123303F5F873444A8B63D36832
:104D480083F01003D360424B9B68002B69D0414825
:104D580005B0BDE8F04F18470AF000FCFFF77DB931
:104D68000C2804D13C480DF0C7FA3C480DE07F28D8
:104D780012D1FFF7DEB80D28B5D07F2809D12E4A09
:104D8800013B002136482360D1540DF0B5FAFFF7F6
:104D9800D0B82F2B3FF6CDA8A0F12002D2B25E2AC0
:104DA8003FF6C7A813B920283FF4C3A85A1C2260AD
:104DB800214AD0540DF098FAFFF7BBB85A1EA95CE7
:104DC800202901D113469AE71B4A00212360D154B8
:104DD800244B254DD3F800A0D5F800B0DFF8589043
:104DE800584612F032FA074659463A46484612F0F3
:104DF80035FA1E4A28B919F8073053445B785B071F
:104E080003D010359542E7D306E0954204D2781CCA
:104E1800EB684844984702E015480DF06DFA002306
:104E28006FE705B0BDE8F08FA0100020202A002011
:104E38000400FA0500ED00E09C290020E5CB0108FC
:104E4800DC1900206C310020E6190020000C01401C
:104E580050290020DC10002051BC01084CBC01087E
:104E680078BC01086800002000A10108D0A2010850
:104E78005CBC0108EC1100202DE9F0474B28A0B0DC
:104E8800044600F03B8600F2B480302800F0C68665
:104E980051D8222800F0868423D8032800F06081A6
:104EA80014D8012800F05081022840F022870420FD
:104EB8000DF09EF943200DF06CF94C200DF069F9C6
:104EC80046200DF066F94C2000F04CBE042800F096
:104ED8005181052840F00D871A200DF089F900242A
:104EE80059E1282800F0D88515D8242800F0BF8576
:104EF800262840F0FE86B44C06200DF079F9B4F867
:104F08005C010DF078F9B4F85E010DF074F9B4F8AD
:104F1800600100F0A9BD2C2800F0D1852E2800F0F2
:104F28004C862A2840F0E58601200DF061F9A64B51
:104F3800587900F017BE3D2800F016831ED8362891
:104F480000F021860BD8322800F00686342840F07D
:104F5800D08648200DF04CF9002500F045BC3A28D1
:104F680000F0B5823B2800F01684382840F0C1864E
:104F780004200DF03DF9944C00F07FBD452800F069
:104F8800A58627D8402800F0F085422840F0B18651
:104F98008D4C10200DF02CF960790DF0FAF8A0680E
:104FA8000DF032F994F892010DF0F3F8B4F85C01C1
:104FB8000DF021F9B4F85E010DF01DF9B4F86001A7
:104FC8000DF019F9B4F882010DF015F9B4F884015F
:104FD80000F04ABD472800F05786C0F044864928AB
:104FE80040F0878602200DF003F9774B988900F08E
:104FF8003BBD702800F0EB8258D8692800F0478242
:105008002AD8652800F0FA8015D84D2800F0858543
:10501800642840F06E8607200DF0EAF8E7200DF0CE
:10502800B8F8694B58790DF0B4F800200DF0B1F8D4
:10503800042000F05ABE672800F0AC8100F21A8202
:1050480012200DF0D5F8614B00241B88B3F5806F52
:105058008CBF0825012580E16C2800F02B8217D829
:105068006A2800F087846B2840F0438605200DF0FD
:10507800BFF8574B18880DF0BEF8564B18880DF03E
:10508800BAF8554B93F86E0000F0010000F06ABDC5
:105098006E28514D00F0228200F2718206200DF038
:1050A800A7F8E86D0DF0B0F84C4B0EE2782800F048
:1050B8007E8119D8742800F0B8830BD8722800F0C4
:1050C8001984732840F0158608200DF091F8012402
:1050D80000F049BC762800F06D8400F2EB832F20A5
:1050E8000DF086F83E4C4EE3A42800F0898414D8CD
:1050F8007B2800F0EE82A02840F0FB850C200DF004
:1051080077F8384B18680DF07FF8374B18680DF0B2
:105118007BF8364B186800F0E8BDF12800F0838171
:10512800FE2800F09484F02840F0E3852A4C0420FF
:105138000DF05EF8236CB3F85A000DF05CF8236CA0
:10514800B3F8580000F090BC03200DF051F800208F
:105158000DF01FF820460DF01CF80D2000F002BDE0
:105168000DF046F801200DF014F80A200DF011F8A2
:1051780000F044BC06200DF03BF831200DF009F892
:1051880030200DF006F833200DF003F852200DF012
:1051980000F800F068BC164B185D01340CF0F9FFFC
:1051A8000B2CF8D10024134B185D01340CF0F1FFDF
:1051B800082CF8D10024104B185D01340CF0E9FFDD
:1051C800072CF8D100F093BDEC1100202C00002032
:1051D8005A1A00205C1A0020E0100020D411002088
:1051E800DB990108E8F7FF1FECF7FF1FF0F7FF1F37
:1051F800B4BC0108C0BC0108C9BC0108CA4C0B20DA
:105208000CF0F6FF20880CF0F6FF608880B20CF0F6
:10521800F2FFC64B1B68C3F3C000C3F380028000D3
:1052280040EA4200C3F340021043C3F3401240EA8D
:10523800C20003F0100318430CF0DDFFBC4B1A88C2
:10524800636802F0080103F4475949EA010903F4C5
:10525800804149EA010903F4004149EA010903F4DC
:10526800803149EA010903F4003149EA010903F4EC
:10527800802149EA010903F4002149EA010903F4FC
:10528800801149EA010903F0007349EA0303DFF8D2
:10529800D49212F0010F99F8009018BF4FF002084D
:1052A800C9F3800908BF4FF0000843EA090312F068
:1052B800020F43EA080314BF4FF0040C4FF0000C30
:1052C80012F0040F43EA0C0C14BF4FF0100E4FF00D
:1052D800000E12F0400F14BF202700274CEA0E0ED4
:1052E80012F0100F14BF4FF4007600264EEA07079D
:1052F80012F0200F14BF4FF4806500253E4312F4CE
:10530800807F14BF4FF400600020354312F4007F03
:1053180014BF4FF400110021284312F4806F41EAB2
:10532800000114BF4FF08063002300201943034697
:10533800247AA3420AD27F4A9D5C012202FA05F52B
:105348000D421CBF9A4010430133F2E70CF05CFF9A
:10535800794B93F8B00700F005BC784B33F914008B
:10536800013490FBF5F080B20CF045FF032CF4D12A
:105378006D4CA08C0CF03FFFE08C0CF03CFF208DB6
:105388000CF039FF608D0CF036FFA08D0CF033FF68
:10539800E08D69E310200CF02BFF0024684B185DAA
:1053A80001340CF0F6FE102CF8D100F0A0BC7020EF
:1053B8000CF01EFF00260E2474435B4D01362B6C47
:1053C8002344B3F819010CF016FF2B6C2344B3F8EF
:1053D8001B010CF010FF2B6C2344B3F81D010CF0DB
:1053E8000AFF2B6C234493F81F010CF0D2FE2B6CA0
:1053F800234493F820010CF0CCFE2B6C234493F843
:1054080021010CF0C6FE2B6C234493F822010CF00A
:10541800C0FE2B6C1C44D4F823010CF0F5FE082EBA
:10542800C9D100F064BC70200CF0E2FE424C04F1DB
:10543800700594F8D4000CF0ACFE94F8D5000CF08C
:10544800A8FE94F8D6000CF0A4FE94F8D7000CF04F
:10545800A0FE94F8D8000CF09CFE94F8D9000CF04B
:1054680098FE073494F8D3000CF093FEAC42E0D1D8
:1054780000F03DBC10200CF0BBFE0024314B185D41
:1054880001340CF086FE102CF8D100F030BC2E4D03
:1054980000242878400000F0FE000CF0A9FE2B78CC
:1054A8009C4280F02484294B33F814000CF0A3FEAE
:1054B8000134F4E7264C06200CF09AFE20880CF004
:1054C8009AFE60880CF097FE224B1888CCE20420E4
:1054D8000CF08EFE144B186E00F007BC07200CF081
:1054E80087FE1D4B1888FF28A8BFFF20C0B20CF00C
:1054F80050FE1A4B186880F3100080B20CF07BFE47
:10550800B5F864000CF077FE0B4B93F88721144B29
:10551800186822B10A23584380F3100001E000F311
:105528000F0080B2A0E200BFE0100020DC190020CC
:10553800A41A0020E9100020EC110020CE11002050
:105548001011002024110020BC2A0020D82D002092
:10555800942D0020DC110020CC190020D81900203F
:10556800D41900208B310020BF4C02200CF040FEE3
:1055780094F8E2010CF00DFE94F8E101F2E20B2040
:105588000CF036FEAB6E002618780CF002FEAB6EFF
:1055980058780CF0FEFDAB6EB44C334418790136E4
:1055A8000CF0F7FD032EF6D1A36ED8790CF0F1FDBF
:1055B800A36E98780CF0EDFDA36ED8780CF0E9FD99
:1055C800A36E58890CF017FEA36E187ACAE2A74C8E
:1055D8001E200CF00DFE236C00251B78022B65D1D4
:1055E800236C05F1080253F82200A1490EF036F8A1
:1055F80011F0F4FF80F30800C0B20CF0CAFD236C70
:105608009C4903EB8503D86A0EF028F811F0E6FFF1
:1056180080F30800C0B20CF0BCFD236C05F10E024B
:1056280053F8220094490EF019F811F0D7FF80F3CF
:105638000800C0B201350CF0ACFD032DD0D1072D08
:10564800236C21D1586C8A490EF008F811F0C6FF76
:1056580080F30800C0B20CF09CFD236C8449986C60
:105668000DF0FCFF11F0BAFF80F30800C0B20CF097
:1056780090FD236C93F84C000DF098FF11F0AEFFED
:1056880080F30800C0B20BE02B4458780CF081FD81
:10569800236C2B44D87A0CF07CFD236C2B44587D6A
:1056A80001350CF076FD0A2DC9D120E3236C2B447B
:1056B80058780CF06EFD236C2B44D87A0CF069FDF9
:1056C800236C2B44587D01350CF063FD0A2DEDD178
:1056D8000DE33C200CF08CFD0024644D04F108021D
:1056E8002B6C654953F822000DF0B8FF11F076FFD6
:1056F80080B20CF080FD2B6C5F4903EB8403D86A01
:105708000DF0ACFF11F06AFF80B20CF074FD2B6C49
:1057180004F10E0253F8220057490DF09FFF11F0D3
:105728005DFF013480B20CF066FD032CD5D1072C47
:105738002B6C16D1586C50490DF090FF11F04EFFAC
:1057480080B20CF058FD2B6C4B49986C0DF086FF1D
:1057580011F044FF80B20CF04EFD2B6C93F84C0016
:105768000BE0234458780CF046FD2B6C2344D87A80
:105778000CF041FD2B6C2344587D01340CF03BFDAB
:105788000A2CD4D1B3E214F8010F002800F0AF823C
:105798000CF0FFFCF7E701200CF02AFD334B1B6CE3
:1057A8001878DFE150200CF023FD00252F4B0C2149
:1057B8001C6C324B04EB850494F87920013501FB0D
:1057C800023393F838000CF0E4FC94F87A000CF0FB
:1057D800E0FC94F87B000CF0DCFC94F87C000CF006
:1057E800D8FC142DE2D182E2204B1C6C062303FB6B
:1057F800054494F8CE000CF0CCFC94F8C9000CF0E9
:10580800C8FC94F8CA000CF0C4FC94F8CB000CF067
:10581800C0FC94F8CC000CF0BCFC013594F8CD0029
:105828000CF0B7FC0C2DDFD161E24FF00008012627
:1058380000270E4B1A7A974233DA0933FA5C0024B0
:105848000C2363430D4D05F13001595C914207D19A
:105858002B44586B11F0F9FC82468EB9B14611E021
:1058680001341C2CECD11AE0EC110020E0100020CF
:10587800000020410000C84200007A44DC99010879
:1058880080440CE0D1450ADA0C2303FB04535B6B1C
:1058980013F809000CF07DFC09F10109F2E7013762
:1058A800C7E7002E00F023825FFA88F00CF0A0FC16
:1058B8000026BDE7CC4D0024287A0CF099FC2B7A01
:1058C8009C4280F01482C94B0021E65C0C2202FB4A
:1058D80001F3C74800F13007DA5DB24205D103444D
:1058E80093F838000CF055FC02E001311C29EDD189
:1058F8000134E4E7BF4C16200CF07AFCB4F89801A8
:105908000CF079FCB4F844010CF075FCB4F84601CD
:105918000CF071FCB4F848010CF06DFCB4F8DA0135
:105928000CF069FC94F8EF010CF033FC00200CF04B
:1059380030FC94F8F0010CF02CFC94F887010CF082
:1059480028FC94F894010CF024FC00200CF021FCB5
:10595800A54B0A201B6CB3F9563093FBF0F080B2CC
:105968000CF049FC89E0E0B201340CF012FC092C7F
:10597800F9D1BCE110200CF03BFC9F4B9F4C1878F0
:1059880000F002000CF005FC9D4B18780CF001FCAF
:1059980020680CF039FC60680CF036FC994B1888CC
:1059A8000CF029FC984B18880CF025FC8E4BB3F8AA
:1059B8006C0059E00CF0D0FB074612200CF018FCE4
:1059C800894C17B9266F656F05E0102F19BF0025A0
:1059D8002E46A66FE56F38460CF0DBFB30460CF020
:1059E80013FC28460CF010FCD4F880000CF00CFCDA
:1059F80000200CF000FC00200CF0FDFB0020B1E0C2
:105A0800794D002495F884002E4680000130C0B2FC
:105A18000CF0EEFB95F884000CF0BBFB96F8843094
:105A28009C4280F06481794D285D0CF0B2FB05F151
:105A38001003185D0CF0ADFB05F12003185D30353F
:105A48000CF0A7FB285D0CF0A4FB0134E6E7082066
:105A58000CF0CEFB00200CF0CEFB00200CF0CBFBB2
:105A680000200CF0C8FB00200CF0C5FB3FE104202F
:105A78000CF0BEFB5F4B986837E194F87C010CF0A2
:105A880088FB94F880010CF084FB94F87F010CF0FB
:105A980080FB94F8810165E0564C07200CF0A8FBC8
:105AA800B4F882010CF0A7FBB4F884010CF0A3FB56
:105AB80094F886010CF06DFBB4F88801D4E74D4CDE
:105AC8000C200CF095FB94F892010CF062FBB4F8F2
:105AD8009C010CF090FBB4F898010CF08CFBB4F826
:105AE8009A010CF088FB94F893010CF052FBB4F87F
:105AF8009E010CF080FBB4F8A001B5E73D4C0420F2
:105B08000CF076FB94F8D8010CF043FB94F8D9011B
:105B18000CF03FFBB4F8DA01A6E73D4C3D4D207888
:105B2800002600EB4000C0B20CF062FB237802357F
:105B38009E4280F0DC8015F8020C0CF02AFB15F868
:105B4800010C013600EB800000EB800000F2EE2033
:105B580080B20CF050FBE9E701200CF049FB254B23
:105B680093F894010CF015FBC1E008200CF040FB01
:105B78000024204B234493F88A0101340CF009FBDC
:105B8800082CF6D1B3E0184B1A4C93F8C50004F171
:105B98002005C0EBC000C0B20CF02AFB94F8F60157
:105BA80000231D4AD25C904200F0A5800C33302BB4
:105BB800F7D10834AC42F1D199E040200CF018FB41
:105BC8000C4C04F14005B4F8A8020CF014FB94F84E
:105BD800AA020CF0DEFA043494F8A7020CF0D9FA01
:105BE800AC42F0D183E000BFE0100020E9100020B3
:105BF800DC990108EC110020E0190020E8190020C8
:105C0800E6190020E4190020E2190020651100209F
:105C1800BC2A00208E130020C82A0020E0200CF0A7
:105C2800E7FA424C04F18005B4F82A02043400F083
:105C38003F000CF0E0FAB4F82602C0F386100CF02E
:105C4800DAFA94F8240200090CF0A3FA94F8240272
:105C580000F00F000CF09DFA94F825020CF099FA68
:105C6800AC42E1D143E0324C0D200CF0C1FA0AF00D
:105C78000DFB0CF08EFA20880CF0C6FAE0680CF0E8
:105C8800C3FA06F065FB30E00CF07AFA054684208A
:105C98000CF0AEFA28460CF0B7FA254BDC6805F193
:105CA8008003A3428CBF641B802406F00BFC2846AB
:105CB800224669460AF01EFB05460024AC4216DA65
:105CC8001DF804000CF065FA0134F7E713200CF016
:105CD8008FFA0024174B185D01340CF05AFA0B2C7C
:105CE800F8D100200CF090FA00200CF08DFA012079
:105CF80018E0002016E00CF04CFAB4F8F8010CF0AB
:105D08007AFA94F8FA010CF044FA94F8FB010CF0D2
:105D180040FA94F8FD010CF03CFA94F8FC010CF000
:105D280038FA46E720B0BDE8F08700BFEC11002044
:105D38001C000020B4BC01086B4B6C4A2DE9F04FE5
:105D48005E8914684FEA062AB4EB0A0A9C884FF069
:105D580000054FEA04481C894FF0000BA4FB0A67B2
:105D680065EB0B0B04FB0B77F40944EA476418EB6B
:105D780004065C884FF000094FEAE7154FEAC4387B
:105D8800DC8849EB050787B0CDE90467A4FB0A67FF
:105D980004FB0B77340A44EA076418EB04064FEA5D
:105DA80027259C894FF0000949EB0507CDE90067D5
:105DB800AAFB046704FB0B77F40D44EA472414F5A7
:105DC800FA664FEAE75545F10007B6F5FA6F77F13D
:105DD8000003CDE90267964666DADDE90489A4FB8B
:105DE800046704FB05F34FF0050C07EB4307A6FB1C
:105DF8000C230CFB07335F104FEA3206B8EB06089A
:105E08004FEA920646EA837669EB07099F10DDE9B7
:105E18000023921B63EB0703CDE90023DDE902674A
:105E2800334A4FF0FF33964277EB0303CDE90489F9
:105E380027DA40F6AC520023A4185D4104FB05F3B1
:105E4800A4FB04456FF0060205EB4305664202FB1E
:105E58000566A4FB0223334418EB020649EB03074B
:105E6800CDE904670B26A4FB062306FB0533DDE911
:105E780000455B104FEA3202A41A65EB0305CDE931
:105E88000045DDE902450AFB0BF3AAFB0AAB0BEB65
:105E9800430B4FEADA7242EA4B02A41A4FEAEB7359
:105EA80065EB0305CDE90245DEF80440009B019D42
:105EB800A4FB032304FB05334FEA525848EAC328DE
:105EC8004FEA6359DDE90423B8EB020269EB0303E7
:105ED8009946D30B43EA494300B1036009B1029BD9
:105EE8000B6007B0BDE8F08F5C020020A81100200D
:105EF80024FAFFFF2DE9F04FDFF8589285B00746E6
:105F0800D9F808000E460DF055FB8E4C80462088C7
:105F18000DF04CFB4FF05C51054640460DF09EFBE2
:105F28004FF06451824628460DF098FB01465046D2
:105F38000DF08AFA4FF06251824640460DF08EFB12
:105F48004FF06A51804628460DF088FB01464046CE
:105F58000DF07AFA0546B4F902000DF02BFB014664
:105F680028460DF07BFB5146054650460DF076FB62
:105F78008046B4F904000DF01DFB014640460DF0C3
:105F88006DFB014628460DF061FA80460DF02CFDA8
:105F98006D490546A06140460DF014FCD9F80C3057
:105FA8008046284601930DF005FB4FF07C510DF01B
:105FB80055FB66490DF048FA0546E389B4F90A002D
:105FC80002930DF0F7FA29460DF048FB29460DF02B
:105FD80045FB4FF058510DF041FB8146B4F90800DC
:105FE800B4F810B0B4F80CA00DF0E4FA29460DF09E
:105FF80035FB014648460DF029FA4FF058510DF08F
:106008002DFB4FF060510DF029FB4FF07E510DF044
:106018001DFA8146E0880DF0C9FA014648460DF0A0
:106028001DFB002181460DF0ADFC00287BD12946DF
:1060380028460DF013FB03900FFA8BF00DF0BAFA17
:10604800039B014618460DF009FB4FF060510DF017
:1060580005FB8346BDF908000DF0ACFA0146284659
:106068000DF0FCFA01460DF0F1F9014658460DF025
:10607800EDF94FF07A510DF0F1FA834601980DF0E1
:1060880099FA01464FF093400DF0DEF905460FFAF4
:106098008AF00DF08FFA4FF08F410DF0DFFA0146CC
:1060A80058460DF0D3F94FF066510DF0D7FA014676
:1060B80028460DF0C9F926490DF0D0FA49460DF0E9
:1060C80081FB0546B4F916000DF074FA29460DF067
:1060D800C5FA29460DF0C2FA4FF040510DF0BEFA4C
:1060E8008146B4F914000DF065FA014628460DF012
:1060F800B5FA4FF060510DF0B1FA014648460DF07F
:10610800A5F98146B4F912000DF054FA0146484643
:106118000DF09CF94FF076510DF0A0FA0146284693
:106128000DF094F900E0002017B10DF05DFC386027
:106138002EB140460DF058FC64235843306005B03A
:10614800BDE8F08F980200200000A04500007A47C3
:106158000050C345A8110020704770472DE9F04151
:10616800324C334D62892B8AB4F904809A1A2389F8
:10617800B4F902E05A43B4F91230D613B4F9142032
:10618800DB02324493FBF2F232440A26E2615643C0
:10619800A2F57A6202FB02F3B4F90EC002FB0EFE0E
:1061A80002FB08F2B4F90C801B130CFB03FC03FB85
:1061B80008F31B1403EB62320232E388921002F5F3
:1061C800004253434CF25032B4F920704FEAEE2E9D
:1061D800B4F900400EEBEC2C0CEB8404BC406D6968
:1061E8000234A5EBA4043A4162434FEAD3384EBFC8
:1061F800B2FBF8F35400B4FBF8F340F6DE3448BFC2
:106208005B001A12524362430A4C08365C4324145A
:1062180004EB224202F6CF62361103EB221300B1DF
:10622800036001B10E60BDE8F08100BF700200207C
:10623800A811002043E3FFFF074B1A685969490476
:1062480008D5520441BF4FF480425A61034B0122E2
:1062580048BF1A76704700BF00040140A81100200B
:10626800024B4FF480521A80704700BF2C00002068
:10627800024B4FF480521A80704700BF2C00002058
:106288007047054A537E23B10123037000235376D8
:1062980070470370704700BFA8110020772048217D
:1062A80001220BF0F5BD7720582101220BF0F0BD3B
:1062B8007620F42131220BF0EBBD074B002193F837
:1062C8002020064B9201343219767720F42102F00F
:1062D800FC020BF0DDBD00BF70020020A8110020F9
:1062E800034B00221A767720F4212E220BF0D0BD22
:1062F800A811002007B5002101AB032277200BF07D
:1063080087FD9DF805309DF804001B0243EA004311
:106318009DF80600184303B05DF804FB08B5FFF7C5
:10632800E9FF014B586008BDA811002008B5FFF728
:10633800E1FF014B186008BDA811002007B5F7213F
:106348006B46062276200BF063FD9DF800309DF821
:1063580001101B0343EA01139DF80210094A43EA9E
:106368001113D3609DF803309DF804101B0343EA12
:1063780001139DF8051043EA1113936003B05DF80B
:1063880004FB00BFA81100200F4B13B51B780F4C5E
:106398000BB1237EB3B1032201AB7720F6210BF0BA
:1063A80037FD9DF805309DF804201B0243EA02439F
:1063B8009DF806201343064AB2F92020C2F10802CC
:1063C800D340636102B010BD02000020A811002074
:1063D800700200200A4B13B51B780A4C0BB1237EC0
:1063E80063B1022201AB7720F6210BF011FD9DF875
:1063F80004209DF8053043EA0223238202B010BD31
:1064080002000020A811002013B5062204464321EB
:1064180068206B460BF0FCFCA8B19DF800209DF8A5
:106428000130012043EA022323809DF802209DF8D1
:10643800033043EA022363809DF804209DF8053069
:1064480043EA0223A38002B010BD13B50622044616
:106458003B2168206B460BF0DBFCA8B19DF80020BF
:106468009DF80130012043EA022323809DF8022091
:106478009DF8033043EA022363809DF804209DF8C9
:10648800053043EA0223A38002B010BD0F4B13B5B9
:106498009A7E1C46C2B90E4B1B68ABB11A681AB17A
:1064A8000C49886902438A619A889868ADF8042083
:1064B80002228DF8072004220DEB02018DF8062038
:1064C80009F0E2FD0123A37602B010BDA811002057
:1064D800540200200010024008B5FFF7D7FF6B21D7
:1064E800802268200BF0D4FC642001F07EFC6B2134
:1064F800032268200BF0CCFC0F2001F076FC104B37
:1065080019211A7868200BF0C3FC0F2001F06DFCEC
:106518000C4B1A211A7868200BF0BAFC1B211822A0
:1065280068200BF0B5FC1C21102268200BF0B0FC91
:10653800BDE808406820372100220BF0A9BC00BF45
:10654800580200200000002008B5FFF79FFF074B06
:106558001B7813B1012B03D008BD4FF4006201E092
:106568004FF48052024B1A8008BD00BF5902002028
:106578002C000020F8B50F461646074C4FF48055FE
:10658800656140F080000CF0DFF8384600213246A3
:106598000CF000F92561F8BD000C014013B501228B
:1065A8000DF1070104463820FFF7E4FF052001F04C
:1065B80011FC9DF8073003B10123237002B010BD10
:1065C80013B50446694643200622FFF7D3FF9DF81A
:1065D80000209DF80130012043EA022323809DF822
:1065E80002209DF8033043EA022363809DF80420CB
:1065F8009DF8053043EA0223A38002B010BD13B50D
:10660800044669463B200622FFF7B4FF9DF80020A8
:106618009DF80130012043EA022323809DF80220DF
:106628009DF8033043EA022363809DF804209DF817
:10663800053043EA0223A38002B010BD70B50E46B0
:10664800054C4FF4805565610CF07EF830460CF02F
:106658007BF8256170BD00BF000C014008B58021A2
:106668006B20FFF7EBFF642001F0BFFB00216B20DC
:10667800FFF7E4FF642001F0B8FB6B200121FFF76E
:10668800DDFF1B201821FFF7D9FF1C201021FFF781
:10669800D5FF054B1A201978FFF7D0FFBDE8084051
:1066A80019200021CAE700BF01000020F8B50F46F5
:1066B8001646074C4FF48055656140F080000CF099
:1066C80043F83846002132460CF064F82561F8BDDD
:1066D800000C014013B501220DF1070104463A20D0
:1066E800FFF7E4FF052001F075FB9DF8073003B1C3
:1066F8000123237002B010BD184A13B5138804464D
:1067080023F040031B041B0C138013883B2023F049
:1067180038031B041B0C1380138869469BB243F093
:10672800400313800622FFF7C1FF9DF800209DF863
:106738000130012043EA022323809DF802209DF8BE
:10674800033043EA022363809DF804209DF8053056
:1067580043EA0223A38002B010BD00BF0038004006
:10676800184A13B51388044623F040031B041B0C76
:1067780013801388432023F038031B041B0C138059
:10678800138869469BB243F0400313800622FFF743
:106798008DFF9DF800209DF80130012043EA022377
:1067A80023809DF802209DF8033043EA022363808A
:1067B8009DF804209DF8053043EA0223A38002B027
:1067C80010BD00BF003800400BF0AEB90BF0D4BAD2
:1067D8000BF0AAB90BF0D0BA73B51D4CE37E53BBCE
:1067E8001C4A1D4D93694FF4805643F0080393618A
:1067F80010238DF806302846032301A98DF80730A9
:10680800ADF8046009F040FC144A2E61138823F0A7
:1068180040031B041B0C1380138823F038031B044C
:106828001B0C43F00803138013889BB243F040030A
:1068380013800123E376752001A90122FFF79AFE50
:106848009DF80400A0F170035842584102B070BD91
:10685800A811002000100240000C01400038004040
:1068680070B50E46054C4FF4805565610BF06CFF12
:1068780030460BF069FF256170BD00BF000C014078
:10688800284A08B51388802123F040031B041B0CF9
:10689800138013886B2023F038031B041B0C43F070
:1068A8003003138013889BB243F040031380FFF733
:1068B800D7FF962001F099FA03216820FFF7D0FF4F
:1068C800962001F092FA03216B20FFF7C9FF0120FF
:1068D80001F080FA10216A20FFF7C2FF012001F0C1
:1068E80079FA00216C20FFF7BBFF012001F072FA52
:1068F80000211920FFF7B4FF012001F06BFA1021E5
:106908001C20FFF7ADFF012001F064FA1B201821BD
:10691800FFF7A6FF012001F05DFA034B01221A7070
:1069280008BD00BF003800405A0200201F4A13B5B6
:1069380013886B2023F040031B041B0C138013885F
:10694800802123F038031B041B0C43F03003138011
:10695800138806249BB243F040031380FFF780FF9F
:10696800962001F042FA75200DF107010122FFF788
:106978009DFE9DF80730682B04D0013C14F0FF04FD
:10698800EED10EE00C200DF107010122FFF78EFE7B
:106998009DF80730142B04D3182B04D9543B062B2D
:1069A80001D9002000E0012002B010BD00380040ED
:1069B80007B5232001F019FA6820752101220DF18D
:1069C80007030BF025FA28B19DF80700A0F168032A
:1069D8005842584103B05DF804FB00BF2DE9FF475A
:1069E800CB4C07462378CB4E002B00F0E78132686A
:1069F8006368D31A7C2B40F2E181237A6260013309
:106A080023724FF0000808F12400C14DC0B206F00F
:106A1800C3F905F10A0333F918000CF0CBFDBE4B9E
:106A2800814618880CF0C6FD014648460CF0CAFE9F
:106A3800BA490CF013FE0CF0D7FF08F1010800B2B8
:106A480006F098F9B8F1030FDDD1302006F0A4F96B
:106A5800B5F9100006F08EF906F096F92B7A9A0728
:106A68002CD141F288336A689A4218D9102006F06E
:106A780093F968694FF0640890FBF8F000B206F0EB
:106A880079F9212006F088F9686990FBF8F308FB8A
:106A980013000028B8BF404200B206F06BF914207A
:106AA80006F07AF9B4F9180006F064F91C2006F02B
:106AB80073F9002006F05EF906F066F9237ADFF82C
:106AC80050825B0740F05781022006F065F9D8F83C
:106AD8001C006423323090FBF3F000B206F04AF950
:106AE800B8F926504FF0050A95FBFAF5032006F091
:106AF80053F98B4BADB21B78DFF8389213F0040FC3
:106B08000DD008F5D970394603F025F828B9D9F819
:106B1800003013F0100F18BF002528B205E0D8F890
:106B280004389889B0FBFAF000B206F023F9D9F8D6
:106B380000309F076ED5DFF80092B4F8082899F85E
:106B480000304FF0640808FB02325B00B2FBF3F33D
:106B5800B4F80A7806203F01BFB247EA0327BFB25C
:106B6800C3F303231F4306F017F938B206F002F9FE
:106B7800B4F80A3899F8001001339BB293FBF1F28C
:106B880001FB1233A4F80A38D4F80C38604D9B7B0B
:106B9800012B05D1392006F0FFF8B5F908081AE0ED
:106BA800B5F808586E235D43152795FBF7F53A208D
:106BB800AFB206F0F1F8B7FBF8F528B208FB157587
:106BC80006F0D8F83B2006F0E7F8A8B2451D0A20E1
:106BD80095FBF0F000B206F0CDF8282006F0DCF8BE
:106BE800D4F810380A2093FBF0F000B206F0C2F88F
:106BF800042006F0D1F8D4F804389B8913B109F0C1
:106C08004FF804E0424BD3F8140880F3100000B2A8
:106C180006F0B0F8D4F818383D4F9D0640F1A08032
:106C280097F81C3898071DD5112006F0B5F8B7F865
:106C38001E084FF4F36568433A4B90FBF3F000B23B
:106C480006F098F8192006F0A7F8B7F81E0845438B
:106C5800642095FBF0F595FBF0F300FB135000B2B0
:106C680006F088F894F81C38B4F8205813F0020F8E
:106C780008BF0025012006F08FF828B206F07AF840
:106C8800092006F089F8002006F074F8264B94F8DD
:106C980022581A88B2F5967F0AD91D4B1B7A03F041
:106CA8000F03072B04D842F20F75954228BF1546EB
:106CB800052006F071F8D4F80C385B7B0BB928B2C4
:106CC80016E0A5F120000CF075FC18490CF07AFDCF
:106CD800002105460CF060FE10B94FF07C5101E030
:106CE8004FF03F4128460CF0B1FB0CF07DFE00B29E
:106CF80006F040F894F81C28054B910703D493F844
:106D08002328012A1AD1012384F8233808482EE0C1
:106D1800C4110020C02D00202C00002000007A445F
:106D28008B310020A0860100560000206666E63FF1
:106D3800E81900209C2D002054000020D3F80C589E
:106D4800C04968680CF08AFC0CF04EFEBD49029000
:106D5800A8680CF083FC0CF047FE039002A806E03C
:106D6800B94A02AB92E8030083E80300184606F02C
:106D780023F806F009F8237A282B1FD1B34B0022F9
:106D88001A7233684FF47A70B3FBF0F83C27172077
:106D980006F002F8B8FBF7F5B5FBF7F007FB105063
:106DA800000200B205F0E6FF182005F0F5FF07FB2A
:106DB800158000B205F0DEFF05F0E6FF94F82C38E8
:106DC800A24D002B00F0618100F0E8FFD5F83038C3
:106DD8009F4AC31A9342074640F2C780002385F8AA
:106DE800363885F83838B5F80838DAB21B0A85F825
:106DF800522885F8533885F8482885F84938D5F851
:106E0800602833689A1AD5F86438D97B4FF47A73B6
:106E18004B439A420ED38F4B1B68C5F8603895F8E0
:106E28006838013B012B9FBF102385F836380223B1
:106E380085F83838D4F810280A20D4F8143892FB8A
:106E4800F0F293FBF0F384F85028121284F85128DA
:106E580084F8543894F81C281B1284F8553894F890
:106E680022389207794984F8833803D42D2381F88E
:106E7800843878E0D4F824987748DFF8E8C199FB9B
:106E8800F0FA0CFB0A924FF0060E042B0EFB02F2EE
:106E98008CBF3323322381F88438704BD4F82868A8
:106EA80092FBF3F196FBF0F003FB1122642592FBB1
:106EB800F5F20CFB006C0EFB0CFE84F87528121220
:106EC80084F876289EFBF3F203FB12E393FBF5F3B9
:106ED8000AEB8A0A4FFA81F80AEB8A0A08EB8A0158
:106EE80089B284F8731800EB8000090A84F87418D2
:106EF80000EB800051B201EB800292B284F878284E
:106F0800120A84F8792884F87A38B4F81E281B12F3
:106F180084F87B382423534393FBF5F5B4F896386B
:106F28000A2284F87C381B0A84F87D38B4F82038A3
:106F38004FEAD979B3FBF2F303F5FA739BB284F8FD
:106F48007E381B0A84F87F38B4F89838F60F84F82E
:106F58007058C5F3072584F8729884F8776884F820
:106F6800715884F88538C4F8307894F89A88374D81
:106F7800B8F1000F0DD1D5F8A00801F001F80128EB
:106F880007D90228364E00F05E8203F063FB012326
:106F9800B370D4F8A4282D4D002A76D095F89A68B5
:106FA8003EB140F6B731D5F8AC38FB1A8B4219D848
:106FB8006BE00123D5F8A00885F89A3802F0F9FBB0
:106FC800D5F8B038082193F9000002238DE848006D
:106FD80032464FF4964302F0FFFB85F8B468C5F8D3
:106FE800A00850E095F8A868CEB9D5F8A008C5F86B
:106FF800A46885F89A6802F0DCFBD5F8B038082157
:1070080093F9000001238DE8480032464FF4964377
:1070180002F0E2FBC5F8A00803F01CFB33E0013ED8
:10702800F6B285F8A86895F8B41895F8B538DEB9B9
:107038004A1C013385F8B42885F8B538D5F8A00876
:107048001FE000BF8096184B689B0108C411002000
:107058003F0D0300C02D00208096980040420F008D
:107068002C000020806967FF12F8016B013370184B
:10707800314685F8B408D5F8A008C5F8A42885F8DD
:10708800B53800F080FFC4F8AC7894F8B638A14D54
:10709800F3B1D5F8B838DBB1D5F8BC38C3B1C5F809
:1070A800C0381B689C4AC5F8C438D5F8C83813449A
:1070B800187AFDF7E1FED5F8C03898790BF069F831
:1070C800D5F8C8380133092B88BF0023C5F8C8385C
:1070D800924D94F8CC282E688E4B002A00F0EE8151
:1070E800D3F8D028002A00F0E98193F8D438013B7E
:1070F800012B00F2E381D4F8D008864F00F040FF5E
:10710800E0B1D7F8D00800F038FF97F8D5388046B6
:107118007E2BD5F800900ED102231B2887F8D4388F
:1071280009D1D7F8D00800F02BFF20B90123C7F800
:10713800D89887F8DC3884F8D588DCE7D7F8D828D9
:107148002B689B1A41F6583293421ED9032387F8BD
:10715800D438B3E1724A32F8130010B903464FF439
:1071680003600133B0F5C06FDBB279D01ED9B0F53A
:10717800006F7FD032D9B0F5036F3FD184F8DD3886
:10718800D4F81838634F99063FD494F8DC1894F86B
:10719800DD38002900F054812A68921B012AD9D9C8
:1071A80084F8DD38002384F8DC3887E1B0F5007F07
:1071B80043D007D8B0F5807F49D0B0F5887F00F07C
:1071C8008B80E6E7B0F5806F00F0AE80B0F5826F97
:1071D80000F0F380B0F5047FDBD123E0B0F5E26F77
:1071E80000F08B80B0F5E46F00F08C80B0F5E06FB4
:1071F800CFD184F8DD38B4F90A1087E0B0F5046F10
:1072080074D0B0F5026FC4D103E197F81C389A071F
:10721800BBD5B7F81E1824234B436421123393FBC4
:10722800F1F107E184F8DD383E4B3A4F1B689B07C4
:10723800ABD5B7F808380A21FBE084F8DD38394BBC
:10724800344F1B681905A0D5D7F81018F2E084F858
:10725800DD38D4F818382F4F5A0796D57969E9E000
:1072680084F8DD382F4B2B4F1B681B058DD5D7F8BD
:107278001418DFE0D4F81818264A8F0684F8DD3889
:1072880083D592F81C1888077FF57FAFD90711D5E9
:10729800D2F82838192283EAE371A1EBE37101EBF4
:1072A8005101B1FBF2F1002BACBF41F0004141F0BC
:1072B80040410EE0D2F82438192283EAE371A1EBA9
:1072C800E37101EB5101B1FBF2F1002BB8BF41F0C2
:1072D80080414FF400608BE084F8DD38D4F818382A
:1072E8000C4F5B077FF551AF3969A3E084F8DD38AF
:1072F800B4F91830642159437AE084F8DD38B4F9D8
:107308000C1003E0B4F90E1084F8DD382C2391FB3F
:10731800F3F16DE0C4110020689B0108C02D002026
:10732800B6BD01089C2D002084F8DD3894F8DE38BD
:10733800644A0133DBB2032B88BF012382F8DE38AD
:1073480042F2107394F8DE1859435F4B1B78D80744
:1073580048BF01319A0748BF02315F07B4F8E038E7
:1073680048BF0431D80748BF0A319A0748BF1431CB
:107378001F0648BF2831D80548BF28315A0748BFDB
:1073880064311F0748BFC831980548BF01F5C87167
:107398009A0648BF01F57A71DF0648BF01F5FA6120
:1073A800580648BF01F57A614FF4806003F01EF972
:1073B800444B002283F8DC28E7E6D4F81818DFF8F5
:1073C800048111F0200784F8DD3817D098F81C28BC
:1073D80012F0020F14BF4FF47A71002112F0010F5E
:1073E80014BF4FF4FA6300230B4494F8221819448D
:1073F80003F0FCF8002384F8DC38C6E6334B1B683E
:1074080019067FF5C2AE394603F0F0F888F8DC7843
:10741800BBE684F8DD38D4F818382A4F9A067FF589
:10742800B4AE97F81C389B077FF5AFAEB7F8203895
:107438006421594303F0DAF8002387F8DC38A4E61E
:1074480084F8DD383AE0B37823B1C5F89C7886F83B
:1074580002809EE5D5F89C38FB1AB3F57A6FFFF4E5
:1074680098AD0123D5F8A008B37000F086FD064654
:10747800D5F8A00800F081FD76067FF48AAD8A2849
:1074880002D08E280DD084E5D5F8183898067FF5F7
:1074980080AD95F89A38002B7FF47BAD05F669032B
:1074A80006E095F89A38002B7FF473AD05F634039F
:1074B800C5F8A4382D2385F8A8386AE504B0BDE8D6
:1074C800F08700BFC41100208B3100209C2D0020C4
:1074D800034B4FF4805208B11A6170475A617047E4
:1074E80000080140034B4FF4805208B15A617047BD
:1074F8001A617047000801402DE9F04F89B00593E3
:10750800A04B80461B880492980737D540F2E63294
:10751800129B9D48DC89B0F900301B1B03F2F31560
:10752800954203D8002BB8BF5B4201E04FF4FA73D1
:10753800B0F9022040F2E630121B02F2F314844242
:1075480003D8002AB8BF524201E04FF4FA729342BE
:10755800B8BF13460522C3F5FA7393FBF2F30A2268
:10756800643B534398F81C20D2105343642293FB86
:10757800F2F3134423EAE373DBB200E06423C14669
:107588000193CB1C03930024039B022C13F8016F77
:107598007E4F03934FEA440A05D1B7F904301B36EE
:1075A8005E4376114AE07A4B37F9142033F91430E8
:1075B80003EB4202049B5B429A4203DB049B934227
:1075C800A8BF1346734A32F90A50059A5B1B32F971
:1075D800145003EB050B06F0FBF888B16E4A5846C9
:1075E800155D0BF0E7FF6D490CF0ECF801462846F5
:1075F8000BF006F969490CF031F80CF0F5F98346FF
:10760800604A1288D10714D437F90A501B366E43E2
:1076180093074FEA261611D598F812509DF90420C1
:1076280005FB0BF35343642293FBF2F306EB23169B
:1076380004E098F8085005FB0BF52E11584B04256B
:1076480033F90A30574F93FBF5F5751B99F801602C
:10765800E35D6E435E430293642396FBF3F698F86A
:1076680051B0F611BBF1000F1BD0022C30460CD1E3
:107678000BF0A0FF5FEA5B0304D05B45A8BF5B4645
:107688001A4600E00122484905E00BF093FF5A46EC
:10769800391D01EBC401FB6903F06EF80CF0A4F985
:1076A8000646424B99F80B7019883E4B01FB05F2D0
:1076B80003F1200E5EF82400D21207FB02073C4AB1
:1076C800B7F5001FA8BF4FF40017974203F12C002D
:1076D800B8BF174650F8242040F824504FF6FF70E2
:1076E8000909B0FBF1F1AA1A4A4303F1380103F181
:1076F80044054EF8247051F824E055F8240045F864
:1077080024E098F85050921170444FEA840C7F138B
:10771800104441F824208DB1CDF818C007930BF020
:1077280049FF079B2A4603F1500101EBC401DB69BD
:1077380003F022F80CF058F9DDF818C099F8153064
:10774800F2195843029B013443431846642390FBC3
:10775800F3F0184B0012024423F80A2003F1080240
:107768004CF80260032C03F1140203F120034CF8D7
:1077780002704CF8030009F101097FF405AF09B064
:10778800BDE8F08FA41A0020D82D0020E4110020B5
:1077980084310020942D00207C9B010800002041AA
:1077A80004110020A81A0020BC1A0020E0100020B4
:1077B8000000E0FF101B00202DE9F04F054690F86F
:1077C80050008DB008910592099318B13228A8BFCE
:1077D800322000E001200BF0EDFE0146AA480BF034
:1077E800F1FFAA4B04461888002808BF01200BF0B7
:1077F800E1FEA74906900BF031FF01900199204660
:107808000BF024FE014601980BF0DCFFA14B07901A
:107818001B889A0724D5A049B1F90030B1F90200B4
:1078280083EAE37280EAE071A2EBE372A1EBE07114
:1078380091420C46B8BF1446B4F5E17F12DA914282
:1078480003DD0028D8BF404203E0002BCCBF184618
:1078580058420BF0AFFE91490BF0B4FF064603E027
:10786800002601E04FF07E564FF00009CA46039506
:107878000024630004938A4B33F914000BF09AFE3A
:1078880088490BF0EBFE0CF0AFF80BF093FE86493D
:107898000BF0E4FE804B029033F914000BF08AFEE3
:1078A8007C4B07461B889B077ED001460BF0CEFD1C
:1078B8007E4B804633F914000BF07CFE01464046AF
:1078C8000BF0C4FD0CF090F8059B5B42984203DB7B
:1078D800059B8342A8BF0346754A0499885E099AA6
:1078E8001B1A32F9140018440BF064FE804605F0A8
:1078F8006FFF70B16F4B40466F4914F803900BF05F
:1079080061FF014648460AF07BFF6B490BF0A6FE73
:107918008046287F0BF04AFE68490BF09FFE82469E
:10792800287A0BF043FE014640460BF097FE644967
:107938000BF094FE0CF058F881460AF100400CF068
:1079480053F8814505DB50460CF04EF84845A8BF72
:1079580048460BF02FFEDFF88C910199824640468D
:107968000BF07CFE59F824100BF070FD55494FEAD6
:10797800840B80460CF010F838B9404652490CF098
:1079880029F820B1DFF8408101E0DFF8388149F8B3
:107998000B80A87C0BF00AFE014640460BF05EFE09
:1079A8004A490BF05BFE81463A4BB3F800B01BF036
:1079B800010F40F099803A4B049ADFF82081D35E9A
:1079C800002BB8BF5B42B3F5206F4FEA84030A93DC
:1079D80003DD002348F824302AE03D4938460BF0FF
:1079E8003DFE039B0B9058780BF0E0FD0B9A014687
:1079F80010460BF0E7FE02990BF026FD01990BF0FB
:107A08002DFE58F824100BF021FD324980460BF06A
:107A1800C3FF38B9404630490BF0DCFF20B1DFF82E
:107A2800B88001E0DFF8AC802C4A0A9B42F803805A
:107A3800039BD87A0BF0BAFD284B53F824100BF0AF
:107A48000DFE27490BF00AFE1BF0020F80464DD0B1
:107A5800384651460BF0F8FC014630460BF0FEFD67
:107A6800014650460BF0F2FC4946074640460BF0EB
:107A7800EBFC014630460BF0F1FD014648460BF0A1
:107A8800E5FC804632E000BF83F9223EE01000208A
:107A9800BD378635A41A0020E41100200000E14318
:107AA800041100200000A03ECDCC4C4084310020C1
:107AB800942D00207C9B0108000020410000A0407C
:107AC8006F12033C0000F0C10000F0410AD7A33D4B
:107AD8000000A043000040C300004043441B0020B6
:107AE8000AD7233C3C1B0020C8465746DFF83CB267
:107AF8000BF1A803185D0BF05DFD014602980BF031
:107B0800ADFD89490BF0AAFD014638460BF09CFCF7
:107B180095F85120034642B10BF10401DBF81C3003
:107B280001EBC40102F028FE0346804F029807F1DA
:107B3800AC0B5BF824100A930BF086FC01990BF050
:107B480041FE029B07F1B4024BF8243052F824B0EE
:107B5800029259460BF078FC014607980BF07EFD1F
:107B6800014658460BF072FC029A834642F82400FC
:107B780007F1BC02105D0BF01DFD014658460BF0E5
:107B88006DFD6B490BF06AFD83460A9B414618461A
:107B98000BF05CFC59460BF057FC0FF01FFD049BE3
:107BA80007F16802D0520A9B07F170021846029248
:107BB8000BF01AFF029A07F17C0342F824004046B2
:107BC80002930BF011FF029B07F1880843F8240089
:107BD8000BF100400BF008FF039B48F82400013329
:107BE80003930CB9012444E6089A524B9479B3F9EB
:107BF8000430640028345C434F4B6411B3F904002B
:107C08000BF0D8FC4FF07A510BF028FD0FF0E6FC92
:107C1800201A0BF0CFFC002CB8BF6442322C064669
:107C280002DD0023BB6224E006980BF0DDFE20F0A5
:107C380003000BF0BFFC8046687B0BF0B7FC0146E5
:107C480030460BF00BFD3D49044640460BF0BAFDAB
:107C5800014620460BF002FD0BF0C6FEBB6A184435
:107C6800374B9842A8BF1846364B9842ACBFB8620B
:107C7800BB62BB6A6FF0FF005B13B3F5807FA8BFE0
:107C88004FF480739842B8BF18460BF093FC8046B7
:107C980030460BF0A9FEEB78584380110BF08AFCB4
:107CA80097F8BF300446032B11D9B5F84E60B6F5E6
:107CB800FA7F0CD20BF098FE7342984203DBB04275
:107CC8000346A8BF334618460BF074FC044695F8E3
:107CD800512062B1530803D09A42A8BF1A4600E067
:107CE800012220461849FB6902F046FD0446414638
:107CF80020460BF0ABFB0BF077FE00B20BF05AFC02
:107D08000FF06CFCA7F86C0020460BF06DFEB8670E
:107D180040460BF069FE0023C7F88400C7F890308E
:107D28000DB0BDE8F08F00BFA69B443BA81A002009
:107D3800F7CC9238E41100200411002000803B4564
:107D4800FEFFFF0F020000F0BC1A00201FB5084B11
:107D58001B681B0309D58DF80400039101230D202E
:107D680001A98DF8053002F09DF805B05DF804FB17
:107D78009C2D00201FB5084B1B681B0309D58DF8E7
:107D88000400029100230D2001A98DF8053002F0AE
:107D980089F805B05DF804FB9C2D002010B50A4A4F
:107DA8000A4B11689B6800BF12689142F7D1084AD4
:107DB8004FF47A70D2F8C04000FB04F2D31AB3FB38
:107DC800F4F300FB013010BDC02D002010E000E0EE
:107DD800A81A002038B50446FFF7E0FF0546FFF76C
:107DE800DDFF401BA042FAD338BD10B504462CB1C4
:107DF8004FF47A70FFF7EEFF013CF8E710BD024A36
:107E08001368013313607047C02D0020024BD3F86C
:107E1800C43003B118477047A81A0020014B1B68EB
:107E2800184700BF7031002010B50020FFF7F6FF9B
:107E3800074B00241C700BF0C5FA064B83F8C840AA
:107E4800C3F8CC40A3F8D040C3F8D44010BD00BF5D
:107E580058310020A81A002010B510B9BDE810400C
:107E6800E2E700230C225A430C4C1119125D82429E
:107E780003D00133102BF5D110BD094BD3F8D40032
:107E880018B14A784078824206D20022C3F8D4104A
:107E9800A3F8D020C3F8CC2010BD00BF44AB010824
:107EA800A81A002010B540001428A8BF14200023E9
:107EB800074A022199540B4499181424834201F863
:107EC800014CF5DBFF21D1540F20BDE81040C3E77A
:107ED800742D00202DE9F84381460B26013E37D04A
:107EE8001E4B10225A6108221A6109F101074FF04E
:107EF80032080525194C0120E36883F01003E3607C
:107F0800E36883F00803E360FFF788FF4046FFF764
:107F18006CFFE368002083F01003E360E36883F0FC
:107F28000803E360FFF77AFF4046FFF75EFF45B1BD
:107F3800013DDFD14FF4FA70FFF757FF4FF0FA0811
:107F4800D8E7013FD6D14FF47A70FFF74EFFC5E767
:107F5800034A044BDA60BDE8F88300BF000C014017
:107F68000400FA0500ED00E003685B691847036840
:107F78001B6918470368DB68184703689B6818473C
:107F880003685B68184703681B681847B0F9023034
:107F98002DE9F74F93421CBF0023037090F800A00F
:107FA80004460E469146BAF1000F40F0AB801046E9
:107FB8000BF000FB86490BF051FB86490BF04EFB9A
:107FC8004FF07C510BF04AFB0FF068FB0146054669
:107FD8000BF044FB8049834628460BF03FFB0346E1
:107FE8005846194601930BF031FA4FF07E510BF0C9
:107FF8002DFA01464FF07E500BF0E4FB29468046EF
:108008000BF02CFB29460BF029FB07460146606064
:108018000BF01CFAE7604FF07E572946A0602761F5
:1080280028460BF013FA29460BF018FB4FF0804155
:108038000BF00AFA014640460BF010FB019B606109
:10804800194658460BF000FA39460BF0FFF901467D
:1080580040460BF003FB40F2DC53A046274655464A
:1080680063651023A4F852301823A061A4F8503097
:108078004FF09741D8F810000BF0F0FA0021824633
:108088000BF08AFC28B150464FF07C510BF0DCF91C
:1080980004E050464FF07C510BF0D8F90BF006FD88
:1080A800C7E90E014FF09741D8F804000BF0D6FA53
:1080B800002182460BF070FC28B150464FF07C51ED
:1080C8000BF0C2F904E050464FF07C510BF0BEF9BA
:1080D8000BF0ECFC0135032DC7E9080108F1040891
:1080E80007F10807C4D1A6F2DC531B042367E36732
:1080F8006367C4F88030A367C4F884300123A4F808
:1081080002902370D4F85490B4F95280C9EB060653
:10811800636A06FA08F67343276A4FEAE67B206F1C
:1081280007FB0B332667A7FB0667E26F1F44636CE8
:10813800D4F840C053434FEAE27B0CFB0B3ED4F823
:108148008010C4F88020ACFB02237344B61A67EB96
:108158000307E36AA26A43434FEAE07B02FB0B3E54
:10816800A2FB00237344B6185F41E36C656F4B4371
:108178006067A06C4FEAE17B00FB0B33C4F8841006
:10818800A0FB01011944636B361A05FB03F3206B4E
:108198004FEAE57B00FB0B3367EB0107A0FB05010A
:1081A800801919447941B4F95020A5670BF03AF9C0
:1081B80008F1FF3201239340E067C01841EBE371F7
:1081C80042460BF02FF9484403B0BDE8F08F00BFDA
:1081D8006F12833ADB0F4940F404B53F2DE9F843A9
:1081E8000024254BE0B293F8BF60B0420DD203EBF8
:1081F8008003224AD3F8D83032F810101BB10B286C
:1082080001D8DB6898470134EBE71D4B1B685B031B
:108218002FD500242346E2B2B2422AD2DFF8589082
:108228004FEA840809F1D80757F8242055689D4279
:1082380017D0284604F056FBEFF31283502282F33E
:1082480012882821AA8C01FB009092B20132C0F852
:108258002C21AA8ADBB292B242F00102AA8283F3ED
:10826800118857F8083000221B6801341A802B4601
:10827800D1E7BDE8F88300BFA81A00202411002028
:108288009C2D002008B50E4B1B6813F4805F0D4B26
:1082980014BFD3F8A821D3F8AC2193F8BF10928863
:1082A8000023D8B2884204D2074820F813200133AB
:1082B800F7E7FFF793FFBDE80840322095E500BFD8
:1082C8009C2D0020A81A0020241100200A4B30B54C
:1082D8001A680A4B02F48052D3F8A841D3F8AC517B
:1082E80000230AB1A18800E0A988054820F81310E6
:1082F80001330C2BF5D130BD9C2D0020A81A00208D
:108308004A2D002070B5124D0024214605F2B11007
:10831800702285F8B0410EF054FF2146D5F824327A
:108328000B4A0B4493F9020088B11E6802F2B1149B
:108338000E5108199C88073184809B7970298371B4
:1083480092F8B03103F1010382F8B031E6D170BD83
:10835800A81A0020094B1A680E2303FB0020437A51
:10836800FF2B07D0064A12789A4203D9054A32F8F9
:10837800130000E0808800B2704700BFD4290020B5
:10838800BC2A0020D82D00202DE9F74F304C054697
:10839800D4F82872384602F0D1FC0646384602F076
:1083A8005AFCD4F82C728146384602F0C7FC01907A
:1083B800384602F050FCD5F804A00746314650462E
:1083C8000BF04CF9D5F808808346494640460BF037
:1083D80045F9014658460BF037F8019B2968834652
:1083E80018460BF03BF94946054650460BF036F95E
:1083F80039460BF033F9014628460BF027F8394681
:10840800054640460BF02AF931460BF027F901469C
:1084180028460BF01BF8014658460FF0B7F90D49EE
:108428000BF01CF90C490BF0CDF9D4F830120BF015
:108438000DF80A490BF0C6F90FF0D0F883B21A0408
:1084480044BF00F5B47083B218B203B0BDE8F08F32
:10845800A81A00200000E144DB0F49400000204139
:1084680001380A4B042804D8DFE800F00507090B97
:108478000D00074A08E0074A06E0074A04E0074AF1
:1084880002E0074A00E0074A1A60704758000020D7
:10849800C9DE000801750008E5E100088FDB000867
:1084A800FDD70008C1770008426A806A131A58424B
:1084B800584170474171704743799B070AD5436A11
:1084C8008269D154436A01690133B3FBF1F201FBBC
:1084D800123343627047437913F001031FBFC36827
:1084E80003F1FF32C369006A1DBF181A1040C0B2F9
:1084F80018467047437910B513F0010304460DD0B0
:10850800FFF7E9FF58B1236A6269E168D05C01337B
:10851800B3FBF1F201FB1233236210BD184610BD04
:1085280090F83B3210B57BB990F83A3290F839425E
:10853800A34209D2B0F8401201229A400A430133FB
:10854800A0F84022DBB2F3E710BD8379DB0748BF10
:10855800B1FA81F1D0F8343148BF49095A681B890A
:1085680009B1136170475361704710F80A3C013331
:10857800DBB20A2B84BF10F8131C054A00F80A3C2A
:1085880082BF002322F8113000F80A3C704700BF70
:1085980080300020334A70B5136C9068194440F657
:1085A8008C23081A98429160D060516013463BD9D9
:1085B800127893F9451010468A420BD1111F0829E9
:1085C80008D893F84610182901D8013103E083F838
:1085D800442002E0002183F8461093F944402149E1
:1085E800A24219D191F84740B4B10C310024944209
:1085F80006DA51F8046F1C4D25F814600134F6E7CB
:108608000C2805D01849002421F810400130F7E75C
:10861800164801780131017083F8452000220121B4
:108628001A7083F8471070BD92F84710C9B140F22C
:10863800DA51A0F2EF248C4208D811780B2905D81A
:108648000B1D0131117042F8230070BD002283F820
:108658004720074B03F13002002143F8041F9342DF
:10866800FAD170BD040100208030002034060020BB
:1086780010010020024A136C013319441164704739
:1086880004010020024B53F820301B681980704702
:10869800801B0020074BA1F57A7153F820301A6827
:1086A8001B8959434FF47A7391FBF3F189B2118016
:1086B800704700BF801B00201FB50123ADF80830AC
:1086C800ADF80410002301A9ADF80A30ADF80C305C
:1086D800ADF8062007F06FF805B05DF804FB38B573
:1086E800A0F513746379A579DB0745D594F838327A
:1086F80005F00105F3B1226B1068838DC3F34E03B7
:10870800838494F83C3223B1B4F842320133A4F89C
:108718004232917A6A00FFF7CFFF012384F83B3297
:10872800002384F8393284F83A3284F83832A4F8CD
:10873800403238BD94F83B322046012B04BF94F8F0
:10874800393284F83A32FFF7EBFE94F83B22236B78
:108758003AB9012284F83B221868997A05FA02F29C
:1087680007E0002284F83B2295421868997A08BFEE
:108778000222BDE838409FE738BD10B5A0F5127455
:1087880094F83C22BAB9A36A616A994228D0591C64
:10879800A069A162C35C2069DBB25B0043F400738B
:1087A8008142A4F83E324FF00A0384F83D3228BFD4
:1087B800A262012312E094F93D327BB1B4F83E1273
:1087C80020464B08A4F83E3201F00101FFF7BDFE38
:1087D80094F83D32013B84F83D3201E084F83C32A4
:1087E80094F83832002B4ED194F839320133DBB289
:1087F800092B84F8393203D12046BDE810408FE6B2
:108808000A2B40D194F83B322BB9B4F8403243F0EC
:108818000103A4F840326379D9071CD5B4F84002A3
:10882800820501D4C30705D4B4F844320133A4F84F
:10883800443210E0E36AC0F347000BB198470AE0FE
:10884800E3696269D054E369E1680133B3FBF1F28B
:1088580001FB1233E361012284F8382294F83B22A9
:108868000023012A84F839320DD1A27984F83B32E9
:10887800236B12F0010F1868997A0CBF02220022AC
:10888800BDE8104018E710BDF0B5046D8279A389E2
:10889800467923F4005312F0020F4FEA03434FEADC
:1088A80013430CBF00214FF4005112F0040FA381B1
:1088B80014BF4FF4806E4FF0000E16F0010F87685A
:1088C800054614BF04200020B307238A48BF40F0A0
:1088D80008029BB223F4405343EA01032382A1898F
:1088E80048BF90B289B221F4B05121F00C014EEA90
:1088F800010140EA0102A281A38A87B023F44073F0
:108908001B041B0CA38201A806F0F4FE039B049E23
:10891800254A944218BF1E46A389192272431BB2E6
:10892800002BB4BF7E00BE00B2FBF6F66427B6FB90
:10893800F7F00001010907FB1163A28912B2002AAE
:10894800B7BFD9001A013231B1FBF7F2A7BF3232F3
:10895800B2FBF7F302F007021043A8BF03F00F03BE
:10896800AA79A8BF184380B212F0010F20812B6D9D
:1089780006D00E498B4202BF042001F54841086128
:1089880012F0080F9A8A0BBF22F0080292B2120462
:1089980042F0080208BF120C9A829A8992B242F4F5
:1089A80000529A8107B0F0BD0038014000440040F1
:1089B8002DE9F04F504C4FF4147685B0804691461F
:1089C8001D4606FB0046274608B94C4B02E0012825
:1089D80004D14B4B33631033C6F834314FF414735E
:1089E80003FB08F3474AFC18FA5003226271224637
:1089F80003F59C733B44E162A36100214FF480704E
:108A0800D4F8343134324FF0010B62612162E161F4
:108A1800A162616284F83C1284F83912A4F8421207
:108A2800A4F84412C4F80890A571E060206184F8A5
:108A380038B284F8468258681B890222ADF80C3097
:108A480003A910238DF80E308DF80F20019207F03E
:108A58001BFB236B019A597B58681B898DF80E10F4
:108A680003A9ADF80C308DF80F2007F00DFB304648
:108A78005946FFF76AFD3220FFF7B7F9224BD4F8C1
:108A880034A11B681A46B2FBF9F1B1F5803F03D354
:108A9800012AF8D95208F6E71C4A5046B3FBF2F20D
:108AA80089B2D2B203F0F4FE4FF4147000FB08F060
:108AB800174B07EB000800F512703C180022C8F8A5
:108AC80048325046214603F02BFFD8F8307015F095
:108AD800010F0CBF022200223868B97AFFF7ECFDBB
:108AE8000C4B3846C8F84C32211D002203F018FF01
:108AF800304605B0BDE8F08FDC1C0020A8BA01089C
:108B0800C8BA0108809B01086000002040420F009D
:108B180083870008E786000803460A4690F846025D
:108B2800D96A9B7944E71FB50123ADF808300023C3
:108B3800ADF80C30ADF80A30084BADF804101B78CE
:108B480001A9012B08BF0323ADF8062008BFADF823
:108B58000C3006F030FE05B05DF804FB0001002083
:108B680038B510F80E2C044650F8043C52B90122CE
:108B780000F80E2C20F80C1C997A18680222BDE81F
:108B88003840D0E730F80C2C20F80A1C891A89B232
:108B980020F8081C074A10F80F0C002522F81010BE
:108BA80004F80E5C1868997A2A46FFF7BCFF04F8A7
:108BB800065C38BD80300020044B53F820301BB1D0
:108BC80007289CBF1B681980704700BF2C02002033
:108BD8002DE9F7438E460546DFF8A092114699F82D
:108BE800A0440068164698467246631C89F8A0346B
:108BF80003F0FAFD2B8901A9ADF8043018238DF88C
:108C08000630686802238DF8073007F03DFAAB7A22
:108C180009F2A447240127442A6849460C2B00F28C
:108C2800F680DFE813F00D00F400F400F4005100C2
:108C3800F400F400F4008A00F400F400F400C20028
:108C4800138CDFF83CC223F001031B041B0C1384B4
:108C5800138CB2F804E0108B624520F073004FEAE1
:108C680000404FEA10409BB21FFA8EFE40F07000A1
:108C780014D00CF5006C624510D00CF5406C6245C0
:108C88000CD00CF5806C624508D00CF5806C624500
:108C980004D023F0020343F0030307E023F00E039C
:108CA8002EF4407E43F003034EF4807EA2F804E0E5
:108CB8001083A2F834801384138B23F008031B0459
:108CC8001B0C43F0080336E0138CDFF8B4C123F023
:108CD80010031B041B0C1384138CB2F804E0108BD4
:108CE800624520F4E6404FEA00404FEA10409BB24C
:108CF8001FFA8EFE40F4E04008D00CF5006C624587
:108D080004D023F0200343F0300307E023F0E0030E
:108D18002EF4406E43F030034EF4806EA2F804E067
:108D28001083A2F838801384138B23F400631B0488
:108D38001B0C43F40063138369E0138CDFF840C114
:108D480023F480731B041B0C1384138CB2F804E007
:108D5800908B624520F073004FEA00404FEA1040C4
:108D68009BB21FFA8EFE40F0700008D00CF5006C24
:108D7800624504D023F4007343F4407307E023F4FE
:108D880060632EF4405E43F440734EF4805EA2F8B4
:108D980004E09083A2F83C801384938B23F00803AB
:108DA8001B041B0C43F0080330E0138CDFF8D0C021
:108DB80023F480531B041B0C1384108CB2F804E0BA
:108DC800938B20F4005023F4E6431B0400041B0C8F
:108DD800000C62451FFA8EFE43F4E04340F4405015
:108DE80003D00CF5006C624503D12EF4804E4EF48E
:108DF800804EA2F804E09383A2F840801084938BFD
:108E080023F400631B041B0C43F4006393832B7B44
:108E180043B1B2F844306FEA43436FEA53439BB21D
:108E2800A2F8443013889BB243F001031380AB7A55
:108E38000C2B19D8DFE803F0071818180B181818A6
:108E48000F18181813000B1902F134000AE00B1957
:108E580002F1380006E00B1902F13C0002E00B19A0
:108E680002F14000C3F8A40438460C44A4F8AC64EA
:108E7800C4F8A82403B0BDE8F08300BFDC1C0020C0
:108E8800002C0140084A13689B020BD5074B0021B0
:108E980019704FF6FE730649086803400B604FF4DB
:108EA80000135360704700BF000002408A31002061
:108EB8006C000240F8B504460E46174600252046C9
:108EC80020210EF0B4F90446D0B1013420460EF04A
:108ED80011FAB0F5617F05DB40F634039842A8BF6C
:108EE800184601E04FF46170A0F56170192390FBFA
:108EF800F3F00DB9307000E070703B7801333B70CF
:108F08000DB90125DBE72046F8BD30B505460C460E
:108F1800134629462246BDE83040014801F06CBEA0
:108F2800A8BE01087FB504780646E4B9354B192177
:108F3800186800EB840090F87B5090F879204D4336
:108F480005F5617590F87A30009590F87C004143FA
:108F580001F5617101912C482146013401F04CFE64
:108F6800142CE3D14BE00EF0C5F91328054641DC7B
:108F7800244B701C1C68202100238DF80F300EF044
:108F880056F91E35064670B1013630460EF0B2F974
:108F98001A289FBF04EB850358709DF80F300133E2
:108FA80098BF8DF80F30304620210EF040F9064664
:108FB80070B1013630460EF09DF90D289FBF04EBC5
:108FC800850398709DF80F30013398BF8DF80F30E6
:108FD80004EB85043046E11C0DF10F02FFF76AFF30
:108FE8009DF80F30042B0AD0601C002104220EF0DB
:108FF800E8F804E0054800211322FFF786FF04B0D3
:1090080070BD00BF20110020C7BE0108DCBE0108EA
:10901800014809F071B900BFE2BE01082DE9F0432B
:1090280004788FB00546002C59D17B4B00211422BF
:1090380009A807AED3F800800EF0C3F8072230461F
:1090480000210EF0BEF800231A46A70005A80593D4
:1090580008EB070583807149B5F802E031F813C0C1
:109068001CEA0E0F0AD00E310DF1380C595C02F1D2
:10907800010E624402F81C1C5FFA8EF20133072BC2
:10908800E9D100210B46664AB5F802E011F802C0A2
:109098001CEA0E0F0AD006320DF1380C8A5C03F177
:1090A800010E634403F8242C5FFA8EF3013106297C
:1090B800E9D118F807308DE841006A7859490292D9
:1090C80009A81A0903F00F0301F081FD214656484B
:1090D80009AA013401F090FD202CA6D198E00EF0E9
:1090E80009F91F28044600F3868028462021E4B2A7
:1090F8000EF09DF81F2C02D9FFF78AFF88E0464B37
:10910800451C1B68002103EB8404204604220EF052
:1091180058F80027454B09AE304600210A2217F8B7
:1091280003905FFA87F80EF04CF8002315F8012B2E
:1091380032B10A2B04D04A4502D0F2540133F5E784
:109148004A455ED108F1FF33032B09D8DFE803F065
:109158001005023F0DF1230134E00DF123011EE05B
:1091680030460EF0C7F82378C0B243EA001006E094
:1091780030460EF0BFF8237800F00F001843207037
:1091880031E00133062B0AD0244800F11B069E5D0E
:109198009642F6D103445A7D63881343638011F8DD
:1091A800012F02B30023EFE70133072B0AD01B4836
:1091B80000F10E069E5D9642F6D130F813206388C2
:1091C8001343638011F8012F6AB10023EFE730469B
:1091D8000EF090F80F2804DC30460EF08BF8607023
:1091E80001E0002363700137052F93D1012407F0B4
:1091F800B1FC6CB980E70E4800211F22FFF785FEFD
:1092080006E02046002104220DF0DBFF0024EEE7F3
:109218000FB0BDE8F08300BF40220020989B0108F2
:10922800AD9B0108F0BE0108FFBE0108B99B01080B
:10923800DCBE0108F8B50478064674B9304D2146FD
:10924800B5F8C621B5F8C8312E48013401F0D4FC70
:10925800042C05F10405F2D1F8BD2B490DF0BAFF35
:10926800A8B9274B4FF47A714FF4FA62A3F8C611E4
:10927800A3F8C821A3F8CA11A3F8CC21A3F8CE11EA
:10928800A3F8D021A3F8D211A3F8D421F8BD304611
:109298000EF030F8032805462BD8304620210DF073
:1092A800C6FF044630B1013420460EF023F80126EB
:1092B800074600E00646204620210DF0B8FF10B909
:1092C800BDE8F840A4E601300EF014F8012EF7D1FD
:1092D80040F2DC53A7F2EE229A42F1D8A0F2EE2235
:1092E8009A42EDD8064B703503EB8503DF80188171
:1092F800F8BD064800210322BDE8F84005E600BF96
:10930800EC1100200BBF01081EBF01080DCE01089B
:109318002DE9FF4104780546002C34D16D4808F04A
:10932800EBFF6D4D686900210AF02CFB002840F026
:10933800CE802146694801F05FFC6869694601F002
:10934800E1FA0146664801F057FCA869694601F050
:10935800D9FA0146624801F04FFCE869694601F014
:10936800D1FA01465E4801F047FC286A694601F0D7
:10937800C9FA013401465B4801F03EFC0C2C05F1AA
:109388001005CFD1A3E0584905220DF067FF38B981
:10939800514B002203441030C0285A61F8D196E09E
:1093A8002846524904220DF059FF04462846002C4D
:1093B8003FD120210DF03BFF002800F08880451C9C
:1093C80028460DF042FF0746494B53F824601EB962
:1093D800484808F091FF7AE028463146FAB20DF085
:1093E8003DFF01340028EFD13B4B0021C21810305B
:1093F800C02851619E46F7D13F4B03EBC402D2F817
:1094080004C09846BCF1000F04D131463B4801F036
:10941800F3FB53E0002718F834309F42F5DA3B019C
:109428000EEB0305143563440FCB013785E80F00B5
:10943800F1E70DF05FFF0B28064643DC28462021A4
:109448000DF0F5FE054648B10135284601F0C4F98E
:10945800214B012403EB0613586100E0044628461B
:1094680020210DF0E4FE054640B10135284601F003
:10947800B3F9194B013403EB0613986128462021F0
:109488000DF0D5FE054640B10135284601F0A4F996
:10949800114B013403EB0613D861284620210DF047
:1094A800C6FE10B9FFF7B4FD11E0013001F094F9E0
:1094B800094B032C03EB06163062F3D11048FFF773
:1094C80027FF04E00F4801210C22FFF71EFD04B01E
:1094D800BDE8F08124BF0108EC1100203FBF01085E
:1094E80045BF010827CB01081EBF010849BF010875
:1094F800A0B901084EBF0108D8BD01085DBF010829
:109508007BBC0108DCBE0108F0B5047887B00646CC
:1095180014BB514B19201968062303FB041191F859
:10952800CA5091F8CE20454305F5617591F8C930C8
:10953800009591F8CB50C831684300F561700190EF
:10954800087902904979454803912146013401F090
:1095580053FB0C2CDDD17CE00DF0CCFE0B2804462F
:1095680072DC3D4B701C1D68202100238DF81730DC
:109578000DF05DFE064680B1013630460DF0BAFEAC
:1095880003289FBF062303FB045383F8CE009DF8EE
:1095980017309CBF01338DF81730304620210DF06D
:1095A80046FE074680B1013738460DF0A3FE0D2868
:1095B8009FBF062303FB045383F8C9009DF81730A7
:1095C8009CBF01338DF8173006266643A919384623
:1095D800CA310DF11702FFF76DFC20210DF027FEAF
:1095E800074670B1013738460DF084FE14289FBF36
:1095F8009DF817307619013386F8CC0098BF8DF89E
:109608001730384620210DF012FE78B101300DF0E8
:1096180071FE0D289FBF062303FB045383F8CD007A
:109628009DF817309CBF01338DF817309DF817301F
:10963800062B0ED0062202FB04500021C9300DF083
:10964800C0FDFFF7E5FC04E0054800210B22FFF709
:109658005CFC07B0F0BD00BF2011002069BF010805
:10966800DCBE01082DE9F347047807464CB92046CB
:1096780001A909F0E3FA0134FFF7F4FF122CF6D13F
:109688007FE00DF037FEC5B2112D75D83E4C05F1BF
:10969800D00604EB4603781C202193F802800DF0D5
:1096A800C6FD3A4F034630B9A8F10202D2F10008CC
:1096B80048EB020848E007F1260800F1010A59784A
:1096C80040460DF0B4FD68B1032D8CBF0323002381
:1096D800C8EB0000C0B23B44184490F82A90B9F196
:1096E800030F02D1FFF794FC4BE0A9F10203D3F179
:1096F800000850464FF0200148EB03080DF097FD95
:10970800D8B1B8F1000FEDD001300DF0F3FD40F203
:10971800ED2380B2984205DD40F6CA039842A8BFFF
:10972800184601E040F2EE20A0F2EE20192290FB4C
:10973800F2F004EB4603D87002E0B8F1000FD1D183
:1097480004EB460383F8029004EB4604A3781F4415
:1097580097F82620B8F1000F09D0E17819234B4378
:109768000B48294603F2EE2301F046FA09E02946A0
:10977800084801F041FA04E0074800211122FFF7E8
:10978800C4FB02B0BDE8F087EC110020989B0108EB
:1097980089BF01089BBF01080DCE010810B504461A
:1097A8002046FEF7E4FB18B90A20FEF71EFBF7E790
:1097B80010BD002207490C2303FB0213596881429C
:1097C80004D10022C2621A725A6070470132042A18
:1097D800F0D17047C82A00202DE9F743064689468C
:1097E8009DF8288011461A469DF82C3000250C203B
:1097F80068431A4FC419C057B04202D1207A20B129
:1098080026E00135042DF2D122E0012E0AD003DC36
:10981800F6B90093124807E01E2E0AD01F2E17D162
:10982800012006E00F480093434603F0FDF8044684
:1098380005E0FFF7BDF841460446FEF795FB4CB13D
:109848000C2303FB0575267185F808906C6001E010
:10985800002000E0204603B0BDE8F083C82A0020BD
:10986800003801400044004010B5084B0022196838
:1098780001EBC20393F90240844201D1981C10BD48
:109888000132042AF4D1002010BD00BFC42A0020F0
:10989800F0B5027887B08AB94A4C04F1200694F8EA
:1098A800F6210023484950B2595681426ED00C33F4
:1098B800302BF7D10834B442F1D181E00022049270
:1098C8000592451C0DF016FDC4B260B2FFF7CCFF3F
:1098D800074618B18DF81040012400E004462846D8
:1098E80020210DF0A4FC054638B1013528460DF0BD
:1098F80001FD0134ADF81200E4B20026284620210B
:109908000DF095FCB0B3451C28460DF0F3FC002281
:109918002E495FFA82FE51F82230834204D0013288
:10992800082AF5D1002300E0734651F8232082422B
:1099380020D1022E0FD0032E12D05A1E012ED2B2E1
:1099480004D0042A13D88DF814300EE0042A0ED857
:109958008DF8153009E0052B09D88DF8173004E08B
:109968009A1E052A03D88DF816300134E4B2013660
:10997800042EC3D1052C04D807B0BDE8F040FFF78A
:1099880047BB04AB03CB3860796019E094F8FB015E
:109998000E4B94F8FA5153F82000B4F8F8210090CF
:1099A80094F8FD0153F82000019094F8FC0153F855
:1099B800200053F825300290054801F01DF979E799
:1099C80007B0F0BDEC110020C82A0020B8A4010897
:1099D800AABF010838B1438811EA030003D08B42BB
:1099E8000CBF01200220704730B50A4B0A491C6899
:1099F8000A79032A0AD81346551C04EBC303EAB2B2
:109A08009D882842F5D00A71981C30BD0A71002043
:109A180030BD00BFC42A002040220020014B002294
:109A28001A71E1E7402200202DE9F047877890F885
:109A380003C0BBB2C7F1640E03EB83065C42C3F1FB
:109A480078001C4D5FFA8EFE7600CCF16408A4B253
:109A580080B2A3B20FFA83F9B9F1000F04DC002B2E
:109A680014BF3B46012300E0734609FB09F25B4340
:109A780002FB0CF292FBF3F3434403FB09F30A22C3
:109A880093FBF2F333449BB225F8023FB1F8009000
:109A98004A880A34C9EB020A1AB202FB0AF24FF4E6
:109AA8007A7392FBF3F3A4B24B4484422B80D0D157
:109AB800BDE8F0874422002010B5447800780022E1
:109AC80040F6C41102FB02F3193B634303F6C413C7
:109AD8005343434393FBF1F3034921F81230013216
:109AE800072AEDD110BD00BF5E220020104B0430C4
:109AF80033F91000B0F5617F05DB40F63303984277
:109B0800A8BF184601E04FF461700A7819235A4338
:109B180002F28332824208DA4A78534303F28333EB
:109B28008342B4BF0020012070470020704700BF67
:109B3800D82D002010B500F1500302788A4203D1D5
:109B48008478C278944204D304309842F5D1002036
:109B580010BD012010BD0B4B1B6813F4805F0A4B2E
:109B6800B3F9063005D0C089421A934207DD08448C
:109B780000E0008A8342B4BF002001207047012022
:109B8800704700BF9C2D0020D82D0020344B354A4B
:109B98001B68126810B51A60334A11685960516819
:109BA80092689960DA60314A11681961516892685F
:109BB80059619A612E4A1168D9615168926819628F
:109BC8005A622C4A11881985518859859188D288FA
:109BD8009985DA85284A1188198651885986928884
:109BE8009A86264A1188D9865188928819871946F3
:109BF80021F83A2F224A10780022824206DA214CB4
:109C080034F81240013221F8024FF6E71E4A128852
:109C1800A3F864201D4A1288A3F866201C4A1188FC
:109C2800A3F86C1051889288A3F86E10A3F87020DE
:109C3800184A3B2112689A66174A126892FBF1F299
:109C4800B2F5967FC8BF4FF0FF325A67134A1288A1
:109C5800A3F87820124A5289A3F85E2010BD00BFED
:109C6800202E00206C310020181B0020241B00200F
:109C7800301B0020E411002004110020CE11002028
:109C8800671B0020241100203C2B0020C41000205A
:109C98000A110020D81100200400002044110020DF
:109CA800101100202DE9F84305460E460D4B0024FF
:109CB80093E88003B44213DA7B1933F9140008EBF4
:109CC800050333F9142009EB050333F91430013483
:109CD8001344022293FBF2F3C01A07F094FEE9E75B
:109CE800BDE8F883202E002070B5472006F0E2FC7E
:109CF800174B1B681B0307D5164B174A5B68106880
:109D08001B68C01A07F06FFE144E154C154D3078BD
:109D180007F069FE23682868C01A07F074FE6368B4
:109D28006868C01A07F06FFE0F4B188807F05BFED3
:109D38000E4B188807F057FE0D4B188807F053FE96
:109D4800337823742B68A3606B68E36070BD00BF31
:109D5800A42F0020202E00206C310020E6190020BE
:109D68000C2E0020E8190020E4190020E219002038
:109D78004C1100207FB5264C264E274D2749284AEE
:109D8800284B20B128480088B0F5805F31D2308850
:109D980091F820101278ADF8040028781C4D1B7833
:109DA8008DF806008DF807108DF8082001A82946BF
:109DB80006228DF809300DF0E9F930B30198BDF8A5
:109DC80008302860AB80532006F074FC208807F028
:109DD8000AFEA07807F007FEE37801A8019323792B
:109DE80002936379039307F063FD0F4B00221A80F7
:109DF8000BE0308891F820102080127828781B78A2
:109E0800A070E17022716371DDE704B070BD00BF1E
:109E18006C220020A41A0020E01900203431002010
:109E28003B0F0020A00F0020C42F0020A0F17D03CD
:109E3800012B70B504460D460A4E05D830687D21C1
:109E4800FEF7A1F884F0200430682146FEF79BF85D
:109E580035B12B881C4404EB142404F0FF042C8037
:109E680070BD00BF941A00200A4A1388013313807A
:109E7800094A136801331360084A138801339BB2F7
:109E8800202B01BF00231380054A138808BF013324
:109E980013807047C42F0020AC2F0020B02F002063
:109EA800B22F002038B53A4B05461B780C46083BC4
:109EB800012B6BD8452006F0FDFB284606F0FAFB7F
:109EC8000C2D23D004D80A2D0AD014D835B138BDAA
:109ED8000E2D4BD02ED3FF2D50D038BD206849E031
:109EE800207806F0E7FB62796378002A14BF8020A7
:109EF8000020184300E0207806F0DCFBA07806F08C
:109F0800D9FBE07806F0D6FB20793BE0B4F90000F5
:109F180007F05EFDA07806F0CDFBE07806F0CAFBFE
:109F2800B4F9040007F054FDB4F90600BDE8384060
:109F380007F04EBD637820788BB180F0800006F082
:109F4800B9FBA468E0B206F0B5FBC4F3072006F03D
:109F5800B1FBC4F3074006F0ADFB200E12E006F09B
:109F6800A9FB6068BDE8384007F04DBD206807F0E0
:109F78003AFD6068BDE8384007F035BD054807F090
:109F880046FD0020BDE8384006F094BB38BD00BF50
:109F9800FC2D0020C9BF01082DE9F04FBE4B8BB046
:109FA8001A880193BD4F002A40F0A98042F20103AC
:109FB800B7F8D607BA4EC21A50425041FFF7DAFE38
:109FC800FFF7E4FD34684920254606F073FBB54BDE
:109FD80004F11C09186807F006FD55F8040B07F092
:109FE80002FD284605F0E0F904F1100005F0DCF95F
:109FF8004FF01008AC4D01232A6803FA08F3134206
:10A0080003D0D9F8000007F0FEFC08F10108B8F108
:10A01800130F09F10409EDD104F1280005F0B4F992
:10A02800B7F84431B4F92E00C01A07F0DCFC2B68ED
:10A03800DB0408D59D4BB4F864001B88181AC0F3DC
:10A048000D0007F0D0FC2B68980403D5B4F866001F
:10A0580007F0C9FC2B68590503D504F16C0005F01D
:10A0680093F92B681A0502D5A06E07F0CCFC2B6873
:10A078005B0402D5606F07F0C6FC2B68180403D593
:10A08800B4F8780007F0AFFCA04604F1300005F002
:10A098007BF904F1360005F077F9B7F8443138F95F
:10A0A8003C0F0127C01A07F09EFC814B1B789F428A
:10A0B80008DA38F9020FB4F93C300137C01A07F052
:10A0C800A2FCF2E72B68990505D5B4F95E00A0F269
:10A0D800DC5007F098FC326876487260B260121A59
:10A0E8009110754A4A43531C032293FBF2F202EB88
:10A0F80042029A1A7C2303FB02033360D6E16F4BBA
:10A108006F4A1B6811688B4206D00AA941F8203DA6
:10A1180000201360FFF7C6FE019B97F8D6171B882F
:10A1280097F8D7070B44013BB3FBF0F200FB12335F
:10A138008B4280F086815A4F0120FFF71BFEFFF704
:10A1480025FD50203E687D6806F0B4FABA683B6881
:10A1580010681B687A680344106806F11C0BA3EBAF
:10A16800400007F050FC6A68736802A89B1A0293C3
:10A17800AA68B36805F11C089B1A0393EA68F36898
:10A1880010249B1A049305F00FF92A69336902A871
:10A198009B1A02936A6973699B1A0393B369AA6944
:10A1A8009B1A049307F084FB3F4901220B68A240E5
:10A1B8001A428A4606D0DBF80000D8F80030C01AE8
:10A1C80007F021FC0134132C0BF1040B08F10408EF
:10A1D800EAD106F1260005F12601002331F9024FE4
:10A1E80030F9022F121B02AC44F823200133042B50
:10A1F800F4D103214FF000094FEA89035FFA83F98C
:10A2080002AB53F821206AB102F108000F2802D8E6
:10A2180049F0010906E08032FF2A94BF49F002099B
:10A2280049F0030911F1FF31E6D24846002406F04F
:10A2380041FAA0460DF1080B09F00302022A16D0D4
:10A24800032A1DD0012A4ED1B8F1000F05D1DBF841
:10A25800004090462401E4B245E0DBF800004FF0EE
:10A26800000800F00F00204306F024FA3BE0B8F1A4
:10A27800000F0CD0DBF80000C0F3031020432CE0E3
:10A28800B8F1000F1ED19BF8010006F013FA9BF8F5
:10A29800000006F00FFA26E0B02F0020EC11002095
:10A2A800202E0020AC2F0020A42F0020A02F00205B
:10A2B800671B00202C2E0020DF7BEFBDB82F00206D
:10A2C800B42F0020DBF80000C0F30330204306F071
:10A2D800F1F9DBF80000C0F3071006F0EBF9DBF842
:10A2E80000402401E4B20BF1040B06AB9B454FEA96
:10A2F8009909A1D1B8F1010F02D1204606F0DAF987
:10A30800DAF8003013F480541FBFB6F86420B5F8AB
:10A3180064100124521A18BF02929A040AD50AAA94
:10A3280002EB8401B5F86600B6F866200134121A0B
:10A3380041F8202C580513D502AA02EB840C06F12B
:10A348006A0E05F16A0000223EF9021F30F9028FF9
:10A35800C8EB01014CF822100132032AF4D103346E
:10A36800190508D50AAA02EB8400A96EB26E013459
:10A37800521A40F8202C5A0408D50AAA02EB840085
:10A38800696F726F0134521A40F8202C18040BD5EB
:10A398000AAB03EB8402B5F87810B6F878300134CC
:10A3A8005B1A42F8203C00E0FCB1012C03D1029872
:10A3B80007F029FB19E0631E002002AA52F82320A7
:10A3C8004000C0B20AB140F00100013BF5D506F0EB
:10A3D80071F94FF0000802AB53F8280008B107F0F4
:10A3E80012FB08F10108A045F5DB30200321FFF737
:10A3F80059FC36200321FFF755FC2F4B3C201978D8
:10A40800FFF750FCDAF80030990506D5B6F95E007A
:10A41800B5F95E30C01A07F0F6FA3A6827487B6843
:10A428007A60121A9110264ABB604A43531C0322D1
:10A4380093FBF2F202EB42029A1A7C2303FB02031B
:10A448003B60204B1B681A0630D51F4C1F4D2268F5
:10A458002B689A420BD162686B689A4207D1019BBC
:10A468001B88102B11D11A4B1B885B060DD1482075
:10A4780006F020F9206807F0C6FA606807F0C3FA0A
:10A4880023682B6063686B600EE0124A0F4B1178EB
:10A498002A7C914208D1104A99681068884203D1F1
:10A4A8005268DB689A4201D0FFF71EFC07F0EEF90C
:10A4B8000BB0BDE8F08F00BF671B00202C2E0020DA
:10A4C800DF7BEFBD9C2D0020501100200C2E0020BA
:10A4D800B22F0020E6190020E81900202DE9F84FD6
:10A4E8000C9EC2EB030B394C0B9B002914BF4FF099
:10A4F800060A4FF0040AF61A6368054601339046C7
:10A5080013D1236853455ED2314A032B98BF29469D
:10A5180052F823202F4807F0E5FA63680022013338
:10A5280063602D4B05469A7113E0002511E02B4A14
:10A538001278954240DA0B9BE3B109FB06F2995C6D
:10A5480001228A40264909680A4213D16368013307
:10A558006360D4F804900A9B1C4F9945E7DB2BD124
:10A568000A2006F0A7F83B6801333B604FF0FF3341
:10A578007B6021E0184A917921B12C2006F09AF8E5
:10A58800013501E00121917109FB0BF3226808EB09
:10A59800030752B958F8030007F039FA97F904107D
:10A5A80005444B1CD2D00F4802E03A440E481179BA
:10A5B80007F098FA0544C9E7206850452CBF0020E9
:10A5C8000120BDE8F88F0020BDE8F88FBC2F0020DF
:10A5D80088A00108D4BF01086C2200206400002074
:10A5E800A42F0020E3BF010819C1010830B585B0C8
:10A5F80004AC002524F8025D0091ADF80600214660
:10A608001020FFF713FC9DF806002146FFF70EFC0B
:10A618009DF807002146FFF709FC9DF80000214638
:10A62800FFF704FC9DF801002146FFF7FFFB9DF8AA
:10A6380002002146FFF7FAFB9DF803002146FFF7C9
:10A64800F5FB9DF80E002946C043C0B2FFF7EEFBAC
:10A6580005B030BD10B5054C2068FDF791FC18B168
:10A668002068FDF78AFCF6E710BD00BF641A0020D9
:10A67800F0B50124B0FBF4F58D4201D34C43F9E762
:10A688000026D4B1B0FBF4F504FB1500B4FBF1F4DB
:10A698001EB9002D01DC002CF3D1092D03F1010EA8
:10A6A800EFB204DD002A14BF3725572500E0302516
:10A6B8003D441D7001367346E3E71C70F0BDF0B5EC
:10A6C8000124B0FBF4F58D4201D34C43F9E7002691
:10A6D800D4B1B0FBF4F504FB1500B4FBF1F41EB9DA
:10A6E800002D01DC002CF3D1092D03F1010EEFB28E
:10A6F80004DD002A14BF3725572500E030253D44E6
:10A708001D7001367346E3E71C70F0BD03685A1CE0
:10A718000260197070472DE9F843089E002B074620
:10A7280088461446334614BF4FF030094FF02009CD
:10A7380013F8012B0AB9254603E0002CFBDD013C88
:10A74800F6E7002D04DD38464946C047013DF8E7E5
:10A75800354624EAE474A01B284415F8011B11B1FE
:10A768003846C047F7E7BDE8F883024B1868FDF79D
:10A778000ABC00BFD0100020F8B507460C46486850
:10A78800002115461E4609F0FDF858B1284608F084
:10A7980011FF104908F062FF01464FF07E5009F0A2
:10A7A80011F860606168304608F050FE0146304696
:10A7B80009F008F8256806462946384608F044FE98
:10A7C8000146304608F04AFF0146284608F03EFE9A
:10A7D8002060F8BDDB0FC9402DE9F041027803463F
:10A7E800202A00F10100F9D0092AF7D02D2A02D138
:10A7F8000346414D04E02B2A08BF03464FF07E551F
:10A808001C460026234614F8012BA2F13007F9B2A2
:10A8180009290DD83949304608F020FF0646384640
:10A8280008F0C8FE0146304608F010FE0646E9E783
:10A838002E2A17D1314F234614F8010B3038C2B2F3
:10A84800092A0FD808F0B6FE394608F0BBFF0146C2
:10A85800304608F0FBFD29490646384608F0FEFE5A
:10A868000746E8E71A7802F0DF02452A39D15A7814
:10A878002D2A02D10233012704E02B2A14BF013309
:10A8880002330027013B002413F8012F303AD1B2DC
:10A89800092903D80A2101FB0424F5E7B4F59A7FB6
:10A8A80028BF4FF49A74A0464FF07E53B8F1070FB3
:10A8B80007D91846124908F0D1FEA8F1080803463E
:10A8C800F4E704F0070434B118460C4908F0C6FE52
:10A8D800013C0346F7E719462FB1304608F072FFEE
:10A8E80004E04FF07E51304608F0B8FE0146284695
:10A8F80008F0B4FEBDE8F081000080BF00002041F0
:10A9080020BCBE4C30B5054687B00C4603A80021D4
:10A918000C220CF056FC2846002109F05BF820B107
:10A928002846284908F092FD03E02846254908F002
:10A938008BFD254908F092FE09F056F8054680EA95
:10A94800E0706946A0EBE57008F078F9002DACBF1F
:10A9580020232D2368468DF80C300CF076FC012856
:10A9680007D130238DF80D308DF80E308DF80F306B
:10A978000CE0022805D130238DF80D308DF80E300B
:10A9880004E0032804BF30238DF80D30694603A87E
:10A998000CF03EFC03A80CF058FC0338C5B22A465C
:10A9A80003A920460CF07CFC002363552046074988
:10A9B8000CF02EFC03AB204659190CF029FC20465C
:10A9C80007B030BD6F12033A00007A4407C001088F
:10A9D80070B50646B6FBF2F40846154614B1204693
:10A9E800FFF7F6FF05FB1464024B1B5D00F8013B03
:10A9F80070BD00BF09C001082DE9F04F81468A46A5
:10AA080016461C4689B000253178002900F0DB8005
:10AA1800252902D00136484674E072784FF00008C4
:10AA2800302A0CBFB278B71CA2F1300312BF4FF026
:10AA3800000BF71C4FF0010B092B19D8A2F13003BA
:10AA4800D9B2092905D80A2202FB083817F8012BC0
:10AA5800F4E7A2F16103052B02D8A2F1570305E040
:10AA6800A2F14103052B03D8A2F137030A2BEADD33
:10AA78006C2A30D13A787E1C642A00F083800BD887
:10AA8800252A3DD003D8002A00F09D80BCE7582A2B
:10AA98000CD0632A19D0B7E7732A22D002D86E2ABD
:10AAA80037D0B1E7752A5CD0782AADD1271D206848
:10AAB800A2F1580462424FF01001624155E02CD9CE
:10AAC800582A32D0632A2AD13E4648462178271D83
:10AAD800D04701350FE0642A63D00ED9732A14D108
:10AAE8003E46236848460093514642460023FFF7F6
:10AAF80012FE271D05443C4686E7252ADFD13E463F
:10AB080048462521D04701357EE70AD86E2A06D166
:10AB18003E46236804341D6076E7002A53D03E463B
:10AB280072E7752A26D0782AF9D1A2F1580304F1E0
:10AB3800040C5A422068CDF80CC04FF010015A415D
:10AB480005ABFFF795FDDDF80CC03E46644605AB46
:10AB580000934846514642465B46FFF7DCFD0544F4
:10AB680052E72068271D0A21002205ABFFF7A7FD41
:10AB78003C46ECE704F1040CCDF80CC020680A212F
:10AB88000022DDE72068271D002808DA2D238DF82C
:10AB9800143040420DF115030A210022E6E705AB07
:10ABA800FAE7206804F1040C00280ADA2D238DF84E
:10ABB800143040420DF11503CDF80CC00A210022D3
:10ABC800BFE705ABF8E7284609B0BDE8F08F0EB43B
:10ABD8000FB505AB53F8042B0190064901A8039360
:10ABE800FFF70AFF019B00221A7004B05DF804EB1E
:10ABF80003B0704715A700080FB413B50B4904AB91
:10AC080008680B4953F8042B09680193FFF7F4FE11
:10AC18000446084B1868FDF7AAF90028F9D0204621
:10AC280002B0BDE8104004B0704700BFDC0000204F
:10AC3800D8000020D010002080EAE073A3EBE07376
:10AC48008B4206DB002801DD401A704702D0084419
:10AC580070470020704770B5044608F0C5FE2030E4
:10AC6800402857D820462C4908F0B4FE28B1204681
:10AC78002A4908F0E9FB0446F4E72046284908F089
:10AC88008BFE28B12046254908F0E0FB0446F4E78E
:10AC98002046244908F09EFE30B12249204608F09B
:10ACA800D3FB01461F480AE020461F4908F074FEFE
:10ACB80040B11C49204608F0C9FB01461A4808F073
:10ACC800C3FB04462146204608F0C8FC054620463A
:10ACD800294608F0C3FC15490646284608F0BEFC7C
:10ACE800134908F0B1FB0146284608F0B7FC1149A2
:10ACF80008F0ACFB0146284608F0B0FC0E4908F005
:10AD0800A3FB0146304608F0A9FC0146204608F09E
:10AD18009DFB70BD002070BDDB0F4940DB0FC940B3
:10AD2800DB0F49C0DB0FC93FDB0FC9BF9A7C2E364A
:10AD3800FAAF4F393587083CA4AA2A3E08B503491B
:10AD480008F084FBBDE8084085E700BFDB0FC93F7A
:10AD58002DE9F04F056885B0814628460C46FFF777
:10AD6800EDFF80462846FFF776FFD9F804500646DF
:10AD78002846FFF7E3FF07462846FFF76CFFD9F898
:10AD8800089005464846FFF7D9FF82464846FFF730
:10AD980062FF41468146504608F060FC41468346C2
:10ADA800484608F05BFC51460190304608F056FCD6
:10ADB80049460290304608F051FC39460390504607
:10ADC80008F04CFC4946206007F1004008F046FCBA
:10ADD80029466060A560029808F040FC0146019889
:10ADE80008F034FB2946E060039808F037FC014678
:10ADF800584608F029FB3946206106F1004008F062
:10AE08002DFC29466061584608F028FC0146039845
:10AE180008F01AFB2946A061019808F01FFC0146BA
:10AE2800029808F013FB4146E061384608F016FC2A
:10AE3800206205B0BDE8F08F2DE9F04107688AB0BF
:10AE4800466885680446084601A9FFF781FF01990D
:10AE5800384608F003FC04998046304608F0FEFBAB
:10AE68000146404608F0F2FA07998046284608F05D
:10AE7800F5FB0146404608F0E9FA02992060384699
:10AE880008F0ECFB05998046304608F0E7FB0146E0
:10AE9800404608F0DBFA08998046284608F0DEFBB1
:10AEA8000146404608F0D2FA03996060384608F037
:10AEB800D5FB06990746304608F0D0FB01463846D0
:10AEC80008F0C4FA09990646284608F0C7FB014667
:10AED800304608F0BBFAA0600AB0BDE8F081074B25
:10AEE80010B51A881C4622EA00009042188002D049
:10AEF8000120FCF7D7FF208810BD00BFA41A00204E
:10AF0800064B10B51A881C4610439042188002D090
:10AF18000120FCF7C7FF208810BD00BFA41A00203D
:10AF2800024A936823EA000090607047EC11002001
:10AF380008B5104B1A780023D9B2914207D20E49AE
:10AF4800002051F82310013309680880F4E7322003
:10AF5800FCF74BFF094B1B685A0309D5084B9B6844
:10AF68005B0305D4BDE8084040F2DC50FCF73DBF68
:10AF780008BD00BF671B0020801B00209C2D0020FF
:10AF8800EC1100202DE9F34108F0FAF94B4A692346
:10AF9800137040F2DC735380BE231371EF2382F8E1
:10AFA800D93700231946164682F8DA37F25C01339E
:10AFB800514040F2DC729342F8D1404B404A83F84A
:10AFC800DA17404B04275A6002F188325A60002091
:10AFD800013F17F0FF075FD03A4B3422DA600024B4
:10AFE80054B100234FF4005056F80480019304F044
:10AFF800D1FB0428ECD11DE04FF4302004F0CAFB4B
:10B008000428E5D12F4D4FF430202B6943F002037B
:10B018002B612D4B6B612B6943F040032B6104F0CE
:10B02800B9FB41F6FD732A69042803EA02032B6180
:10B03800D7D0CDE7234D1FFA88F22B694FF4005083
:10B0480043F001032B6104F1006303F57E331A809A
:10B0580004F0A0FB042814D11C4B4FEA18482344E1
:10B068000193019B4FF40050A3F8008004F092FB79
:10B0780041F6FE732A69042803EA02032B6106D00D
:10B08800A6E741F6FE732A6913402B61A0E740F258
:10B09800DC7304349C42A3D10A4A0428136943F0A0
:10B0A8008003136102D106F04FF910B90520FCF7AF
:10B0B80011FF08F04FF902B0BDE8F081EC11002053
:10B0C800230167450020024000F8030802F803083E
:10B0D8002DE9F04106F038F910B90420FCF7FAFE22
:10B0E800B84C08F04DF9B84940F2DC7220460CF033
:10B0F8005DF894F8B0374FF4CC71022B84BF00236D
:10B1080084F8B03794F8B027B04D01FB02F303F58B
:10B118003A7020442344286093F83C0301FB024220
:10B12800022803F54E7384BF0020187192F83C334F
:10B13800A74A13700C2202FB0343A64A03F2B27318
:10B14800136046F20902A3681A401AB99D4A43F4EB
:10B1580000539360A368DE0703D54FF40050FFF750
:10B16800DFFEA368580409D50820FFF7D9FE4FF47D
:10B178000050FFF7D5FE0120FFF7D2FEA36819079C
:10B1880006D54FF40050FFF7CBFE0120FFF7C8FEAD
:10B19800A3689A0413D54FF40040FFF7C1FE894B0A
:10B1A80093F88631012B03D14FF40060FFF7B8FE06
:10B1B8004FF48030FFF7B4FE4020FFF7B1FEA368DC
:10B1C8005B0603D54FF48030FFF7AAFE94F8E02120
:10B1D8007C4B2AB193F8E42112B1002283F8E421D0
:10B1E8004FF0000C67467C4E7C4B1E6004EB0C0352
:10B1F800B3F8F8E14FEA5E0101F077314FEA9E03B8
:10B2080003F03333C1EB0E00C11A4FEADE0303F03B
:10B218001133CB1A03EB231303F00F32FF2392FBF6
:10B22800F3F31EF00108C3EB032318BF0137A2EBA9
:10B23800030318BFFFB2012B0ADD022B40F0BE80CA
:10B24800B8F1000F00F0BA801EF0BC0F00F0B68015
:10B258000CF1080CBCF1200FC8D1013F012F00F2FE
:10B26800AD8006F04EF8302200215D480BF0A9FFB2
:10B278005C4F5D4BD5F800801F605C4B002108F1E6
:10B288007900C3F80080FEF755FC594B80F00100A7
:10B298001870584B07F126021A60574B07F1D40271
:10B2A8001A6098F80000FDF7DBF82868534B00F5A2
:10B2B800C5721A6000F054FF514B94F8D81107F189
:10B2C80094021A6064224A434E4BC8325A600022E4
:10B2D8009A60DA601A615A619A61DA6183F820200B
:10B2E80083F82120484B2D6807F12C021A60474B40
:10B2F80005F219121A60464B05F289121A60454B7D
:10B3080007F108021A60444BDFF848811F60434B7D
:10B3180007F1A0021A6007F1AA03C8F80030404BF1
:10B32800B4F866011E6008F041F9C8F80800B4F8DE
:10B33800680108F03BF995F85C3008F1040288F8D8
:10B34800043095F87830C8F80C0088F8053094F87F
:10B35800E331286E88F81030324BC8F814501A6060
:10B36800314B05F164021A60304908F077F901465B
:10B378004FF07C5008F026FAB5F816412C4B1860AF
:10B38800204608F017F901462A4808F01BFA2A490E
:10B3980008F064F9294A2A4B15602A4A186005F111
:10B3A80068031360284A05F211151560274A1760CB
:10B3B800274ABDE8F041136007F0CCBF04F042F81B
:10B3C8004FE700BFEC11002000F80308201100200F
:10B3D800482D002048110020761300202831002035
:10B3E800D40F002030130020081000200C1000207B
:10B3F80018000020E0070020000600201810002098
:10B40800882900203431002038080020D429002061
:10B41800400A0020501C0020541C00205409002021
:10B42800180A002068080020A0080020DB0F494007
:10B438009C080020000061444C3D0F44A8070020F0
:10B44800500900209C0700204009002048090020DE
:10B45800940600207422002008B5FFF793FDFFF73B
:10B4680037FEBDE808400120FCF71CBD08B50848B8
:10B478000BF0EBFEC0B209280246054B04DC013094
:10B488002021C0B29954F6E700221A5408BD00BF23
:10B49800D528002008B507480BF0D7FEC0B21428FD
:10B4A800044B04D8421C20211954D0B2F7E70022DB
:10B4B8001A5408BDD52800202DE9F74FFCF76EFC7B
:10B4C800A64C804626686568A768861BF643451B18
:10B4D800C71BED43FF43F60FED0FFF0F2EB93FB922
:10B4E800002D00F08782B9462CE04FF0000929E0D2
:10B4F800B14627E003EB8A0BBBF802301A050ED4DD
:10B5080013F4805F1DBF964A9BF801101268954A94
:10B51800954B14BF52F82120126843F82A20BBF833
:10B528000230D80516D499050AD5904B1B7813F02C
:10B53800040F0CBF8E4A8F4A8B4B126843F82A209F
:10B5480009F10109207B5FFA89FA8B4982450B686A
:10B55800D0D326E0894A5046594605F08BFA884BE5
:10B568001B885A0603D550465946864A16E058079E
:10B5780003D550465946844A10E0190703D550466A
:10B588005946824A0AE09A0703D550465946804AE6
:10B5980004E0DB07D4D5504659467E4A05F06AFADE
:10B5A800CEE7DFF808E20093BEF906307822A3F56B
:10B5B8007A7353434FF47A7293FBF2F3F34603F230
:10B5C8002B13019300225FFA82FE864517D2009B57
:10B5D80003EB820EBEF802E01EF4806F0DD040F23D
:10B5E800671ADFF88491019B39F822E09E449EFB9C
:10B5F800FAFC0AFB1CEE29F822E00132E3E74DB31E
:10B6080008F5C333A0336360637B544A13BB937359
:10B61800614B1B6813F0020F0AD0DFF894E19EF823
:10B6280000E0BEF1000F03D04FF0010E82F80EE0EB
:10B63800DA0506D5594BDB781BB1A37B43F002032F
:10B64800A3734A4B1B7813F0050F02BFA37B43F08B
:10B658000403A37394F80EE0BEF1000F03D13F4B2F
:10B668005B7B002B4FD094F80DC01CF0010FACF1A0
:10B678000C031DD1BCF1030F07D8DFF8E8901EF0CA
:10B68800040F3B4A08BF4A4600E0364AACF1040CB6
:10B69800BCF1070F05D8DFF81CC11EF0010F18BF59
:10B6A8006246DBB2032B0ED81EF0020F3C4B06E0BD
:10B6B800DBB2032B06D82F4B2A4A1EF0020F18BF05
:10B6C8001A4600E0274A4FF0000C5FFA8CF38342D9
:10B6D8000DD20B6803EB8C035B881B0642BFD2F8C4
:10B6E8000090214B43F82C900CF1010CEDE785B14B
:10B6F800BEF1000F08D0637B184A0133DBB2142B6C
:10B7080006D1002304E025B1637B002BF3D100E0D0
:10B718005373002E52D0234A3223B2F90250B2F9A1
:10B728000020002DB8BF6D42002AB8BF524295FBD9
:10B73800F3F592FBF3F2EDB2D3B2AB4238BF2B462E
:10B74800194A13B192FBF3F300E013464344236014
:10B75800E37B024A83BB01232FE000BF8C22002039
:10B76800D029002048BB01088A0E00208B31002018
:10B7780030AB010820AB010840220020A0A001083E
:10B78800A41A0020A6A00108ACA00108B2A00108D4
:10B79800B8A00108BEA001089C2D0020343100206B
:10B7A80038AB0108E4110020400D0300D82D00201B
:10B7B8002C1A002040AB01080023D3738F4D904B07
:10B7C8002D78E27BADB9002F00F00F818D4B267BE1
:10B7D8001A788D4B02F0040293F800C08B4BD2B25A
:10B7E800D3F800E00B680021894D03EB86060F466D
:10B7F800B5E01AB9874A1A61002508E0864AFAE7CF
:10B808000A68AB00D6187688760604D40135EBB200
:10B818008342F5D3D7E7814EB6F90060192E25DDAE
:10B8280012F803E094F814C00EF00F09E1452669F8
:10B838000CDCDFF8CCC19CF815C0BCEB1E1FDEBFCA
:10B84800D6F800C0DFF8D8E143F80EC012F803E0DC
:10B8580094F816C00EF00F09E14533DBDFF8A0C1FC
:10B868009CF815C0BCEB1E1F2CDC26E0193629DA23
:10B8780012F803E094F814C00EF00F09E1452669A8
:10B888000CDCDFF87CC19CF817C0BCEB1E1FA2BF04
:10B89800D6F800C0DFF888E143F80EC012F803E0DC
:10B8A80094F816C00EF00F09E1450BDBDFF850C124
:10B8B8009CF817C0BCEB1E1F04DBD6F800E0584EFE
:10B8C80043F806E0554EB6F90260192E1BDD12F852
:10B8D80003C094F814E00CF00F09F14526690CDC5C
:10B8E800DFF81C9199F81590B9EB1C1FDEBFD6F84C
:10B8F8000090DFF82CC143F80C90D25C02F00F0CDA
:10B90800F4451EDD82E7193680DA12F803C094F890
:10B9180016E00CF00F09F14526690CDBDFF8E09022
:10B9280099F81590B9EB1C1FDEBFD6F80090DFF828
:10B93800F0C043F80C90D25C02F00F0CF445FFF60F
:10B9480065AF94F817E0BEEB121FA2BF3668344A01
:10B958009E505BE75888000504D404330435B3428D
:10B96800F8D122E04AB101EB0C0A06209AFBF0F963
:10B9780000FB19A001280DDC01E057B9012793F855
:10B9880001900EEB89003EF829A090F80290C0784B
:10B9980003E01746002081468246013125F802ACB3
:10B9A80085F800906870C9B2D7E7174A1378013B49
:10B9B80013F0FF0308BF06231370124B1B785B07B5
:10B9C80041BFBBF906304FF47A72A3F57A7303EBE3
:10B9D800C30348BF93FBF2F3124A46BF0133DBB2FD
:10B9E800012392FBF3F34344A36003B0BDE8F04F97
:10B9F80004F06CBA03B0BDE8F08F00BF3B0F002025
:10BA08008C2200208B31002030000020D02900201B
:10BA18008C0E00203CAB010848BB0108E411002053
:10BA28008A0E0020400D030010B507F0C3FD002169
:10BA3800044607F0CFFF08B1204601E004F10040BA
:10BA4800054907F0BFFE054907F008FEFFF776F93C
:10BA5800034B186010BD00BF8096184B35FA8E3C1A
:10BA68004C000020F8B59C4B04461B68187818B1A8
:10BA7800012800F06A819AE2242C984D0CD006D84F
:10BA88000A2C00F0D9800D2C00F0D68048E12A2C31
:10BA980006D02C2C04D043E128706870A87050E1BF
:10BAA8008F4B69782F7800208C4A58542FBB19780F
:10BAB800D770472921D1597850291ED1997847291B
:10BAC80007D1D978472904D11979412901D1012110
:10BAD800D1709978824A522903D1D1784D2900F042
:10BAE800688299787E4A472907D1D178532904D1A9
:10BAF8001279562A04BF0322EA70EA78774E022A9E
:10BB080039D0032A4CD0012A40F08580BA1E072A72
:10BB180000F28180DFE802F004080F131A257F2A5B
:10BB280006F0E0FF686076E01B78532B73D16B68F2
:10BB38005B426B606FE006F0D5FFA8606BE01B7896
:10BB4800572B68D1AB685B42AB6064E01B78302B45
:10BB5800644B1A788CBF42F0020222F002021A707B
:10BB680059E0002007F01EF8287354E0002007F081
:10BB780019F8E8814FE0072F06D0082F4BD1012094
:10BB880007F010F8708246E0012007F00BF841F248
:10BB9800184358434FF47A73B0FBF3F030823AE01D
:10BBA800022F07D0032F0AD1002006F0FBFF4E4BCF
:10BBB800187030E0002006F0F5FF30752BE02AD928
:10BBC8003A1F9210337D0132D2B2013B02EB83035C
:10BBD800DBB2102B1FD8F91EC2F1010201EB820261
:10BBE800D2B2012A0BD0042A11D100205E1E06F021
:10BBF800D9FF3E4B002298553D4B9A5507E03D4AE8
:10BC08005E1E0020935506F0CDFF3B4B98553B4AEE
:10BC1800136801331360314B2A2C18BF9A7807F147
:10BC280001074FF000000CBF012254402F706870CC
:10BC38000CBF5A759C7084E0687D002848D0304B52
:10BC480013F8012D2F495A708B42F9D1244A234CFD
:10BC580013785278402B85BF373B1B011B01DBB2A1
:10BC680098BF03F0F003402A8CBF373A303AD2B27B
:10BC78001344AA78DBB29A4227D121230B702249B8
:10BC8800E0780B68012803F101031E4A0B600AD013
:10BC980002281CD172231370228A1C4B1A80628AD4
:10BCA8001B4B1A8013E0672313700E4B1B789F07FA
:10BCB8000ED5184B62681A60A2685A60227B164B30
:10BCC8001A70E289154B1A8002E03F230B7000209E
:10BCD80000236B7535E000BFD4070020A4220020A4
:10BCE800C82D0020E01900206411002095110020C3
:10BCF800851100206511002075110020EC28002016
:10BD0800D4020020C0020020F8280020E2190020F8
:10BD18004C110020E8190020E6190020E419002041
:10BD28006B78687D0E2B9FBFA54A591C5170A54A98
:10BD380098BFD454A24A18B993785C40947000E034
:10BD48000020003018BF0120F8BD9D4B0022997DCE
:10BD5800082900F22C81DFE801F0050B0F15202BD4
:10BD6800475D6700B52C40F02281DA75012239E081
:10BD7800622C08BF022235E003229A751C765C7695
:10BD88009C7614E104229A755A7E997E2244D2B296
:10BD98005A760A449A76DC7609E105229A755A7E23
:10BDA800997E2244D2B25A760A449A769C83FEE05F
:10BDB80006229A755A7E997E2244D2B25A760A444D
:10BDC8009A769A8B02EB0424A4B2B4F5AC7F82BFB6
:10BDD8007B4A0121D17500229C83DA83002C40F034
:10BDE800E68007229A75E2E05A7E997E2244D2B212
:10BDF8005A760A449A76DA8BB2F5AC7F3EBF704920
:10BE0800891881F820400132998B92B29142DA83E5
:10BE1800E7D9CCE008229A755B7EA34200F0C78080
:10BE2800674B0122DA750DE0674D9A7515F8012DFB
:10BE38006A70664A9542F9D1997E614AA14206D054
:10BE48003F232B70624A536801335360AFE0614867
:10BE5800016801310160D07D10B13E232B70A6E04E
:10BE680021212970D17E062941D004D8022907D082
:10BE7800032923D0F8BD122959D0302967D0F8BD3D
:10BE88005021546A297054494C60946A0C60116BB3
:10BE98004FF47A7491FBF4F1504C218092F87811A8
:10BEA8004F4A19B1117841F0020102E0117821F0EE
:10BEB80002011170012283F8792169E05321297068
:10BEC80092F82510CE0705D592F82420D51E6A428F
:10BED8006A4100E0024602F0010183F87811002A65
:10BEE80056D13F490A7822F002020A7050E04F21E9
:10BEF800297092F82B10CC0705D592F82A20D11E6C
:10BF08004A424A4100E0024602F0010183F87811F2
:10BF180022B933490A7822F002020A7093F84F10C6
:10BF2800304A1170B3F84C102F4A118030E0562176
:10BF3800546B29702D490C8042F21074916B91FB5F
:10BF4800F4F12B4C2180012182F87A1120E049215B
:10BF5800297092F82410274A102988BF10211170DF
:10BF6800254914780022A2420ED20E7A234D565546
:10BF78004E7A234D5655CE7A224D565511F80C6FF0
:10BF8800214D56550132EEE720490A6801320A6010
:10BF980093F879310A4A002B3AD092F87A31BBB338
:10BFA800002182F8791182F87A111846F8BD00202C
:10BFB800F8BD1279432A7FF494AD0222EA7090E525
:10BFC800A4220020C82D0020D4020020C002002096
:10BFD800B4070020F8280020E8190020E419002000
:10BFE800E0190020E619002056000020E219002080
:10BFF8004C11002064110020C4220020651100208B
:10C00800751100208511002095110020EC280020D2
:10C01800F8BD0449044B0968002218705A619961F7
:10C028001A777047C02D0020B4070020F8B5101A01
:10C038000D461F4607F0BEFA0446781B07F0BAFA09
:10C04800174B079E196807F009FB2146054620464D
:10C0580007F004FB29460746284607F0FFFA014681
:10C06800384607F0F3F90BF01DFD0E4907F0F6FA14
:10C0780007F0E0FC069B2946186004F100400BF02D
:10C0880085FB094907F0EAFA084907F0DFF907F0E4
:10C09800ABFC0028BCBF00F50C40A0303060F8BDF8
:10C0A8004C0000202C7D8E3FA00CB34500A00C4610
:10C0B80044F25063984203DDA0F50C40A038704765
:10C0C800034B9842BCBF00F50C40A030704700BF3E
:10C0D800B0B9FFFFF7B50368174C184D23600B681C
:10C0E800174E63600068FFF79FFC95E80300154B47
:10C0F8000196009394E80C00FFF798FF3668124BFE
:10C1080060681E606B68114FC01A07F053FA104B35
:10C11800196807F0A3FA07F067FC2A6823687860B3
:10C128009B1A3B600B4B1E600B4B1B68DA880B4B52
:10C138001A8003B0F0BD00BF4C2C0020E819002085
:10C14800582C0020542C0020942C00205C2C00201B
:10C158004C0000208C2C002018100020882C002077
:10C1680070B50446407907F021FA1E4907F02AFB0A
:10C178001D4D1E4E2860E07B07F018FA194907F09C
:10C1880021FBEE606860A07907F010FA184907F003
:10C1980019FB184D2860207C07F008FA114907F0B0
:10C1A80011FB6860A07E07F001FA134907F00AFB4B
:10C1B800EE60A860E07907F0F9F90D4907F002FB95
:10C1C8000E4D2860607C07F0F1F9064907F0FAFA8D
:10C1D8006860E07E07F0EAF9074907F0F3FAEE60D5
:10C1E800A86070BD0000C842642C00200000FA441A
:10C1F80000002041742C002000007A44982C002074
:10C2080010B50C4C23789B0713D50B4B1B78042BCC
:10C218000FD90A4A0A4B1068526818605A60FFF72B
:10C2280003FC084B1A88084B1A80237843F0010353
:10C23800237010BDE0190020E6190020E81900203D
:10C2480050110020DC110020A82C0020164B13B53B
:10C258001B681B0325D5154B154C1B7815498DF804
:10C268000030154B20681B788DF8013007F0F6F97F
:10C2780007F0E0FB11498DF80200606807F0EEF95D
:10C2880007F0D8FB8DF80300A06807F0D3FB0C4B30
:10C298008DF804001B780A2069468DF80530FDF7F3
:10C2A80001FE02B010BD00BF9C2D00208E2D002085
:10C2B800B02D002000002041AC2D002000007A4461
:10C2C800922D0020054A137883F001031370044A65
:10C2D80000231360034A1360B8E700BF922D0020C3
:10C2E800A82D0020A42D0020094A137818441346CD
:10C2F800C0B210F0800F18BF80381070054A197846
:10C308001378994201BF00231370014A13707047D4
:10C31800AD2C0020AC2C002010B50A4B0A4A1B7823
:10C3280042609C18094A046012789A4225BFD31AC1
:10C338000B60C3F1800300232EBF4B600B604A6083
:10C3480010BD00BFAD2C0020AE2C0020AC2C00206E
:10C358001FB5684602A9FFF7DFFF044B02981B6868
:10C3680003440398184405B05DF804FB2406002034
:10C378002DE9F04F89B00193002382469946029136
:10C388000392039A934205DA029A52F82320013362
:10C398009144F6E7019B4D46002B56D103F076FFFA
:10C3A800002852D101987DE00222404E8DF81C20D1
:10C3B8001A0C4FF480578DF81D2006201A0A8DF8A4
:10C3C8001E208DF81F3003F085FF7761062006F0E8
:10C3D800BBF9374B01223761D0461A707761264680
:10C3E800002007A9042206F0D5F9029F4FF0000BA0
:10C3F800039B9B451EDABC4657F8042B4FEA8B0378
:10C40800002A48D0B24236D332465AF803100020E8
:10C41800CDF814C0049306F0BDF9049BDDF814C0F0
:10C428005AF8032032444AF80320DCF800309E1BF7
:10C43800CCF800601D4B4FF480521A611D4A2D1B29
:10C4480013681C44019B146053B34DB3194B1B680C
:10C45800DCB22A19B2F5807F174A88BFC4F5807408
:10C46800D26898BF2C4693429ED3144A0023137077
:10C47800134A137014E00020D8F8001006F08AF967
:10C4880057F8043CD8F80020F61A1344C8F80030CE
:10C49800002347F8043C0BF1010B08F10408A7E757
:10C4A800C5EB090009B0BDE8F08F00BF000C0140E2
:10C4B80021060020240600201C000020AC2C0020AF
:10C4C800AD2C002030B50B4C0B4D22782B7885B065
:10C4D8009A420CD0684602A9FFF71EFF012368465E
:10C4E80002A90222FFF744FF00232B70237005B036
:10C4F80030BD00BFAD2C0020AC2C002030B50E4D57
:10C508000E4C2A78237885B09A4211D0684602A941
:10C51800FFF702FF002302A902226846FFF728FF5F
:10C52800FFF7E2FE20782B781B1A5842584100E0AA
:10C53800012005B030BD00BFAD2C0020AC2C002080
:10C5480038B50E4C4FF4805545F2082003F0C2FE72
:10C558006561062006F0F8F8094B01222561C7201D
:10C568001A70656106F0F0F8064A00232561137019
:10C57800054A1370054A136038BD00BF000C01401E
:10C5880021060020AC2C0020AD2C00202406002021
:10C598000148024900F0E4B800080040281C0020C7
:10C5A8000148024900F0DCB800040040001C0020EB
:10C5B8004FF08040014900F0D3B800BFD81B0020DD
:10C5C8000148024900F0CCB8002C0140B01B002003
:10C5D8000148024900F0C4B8002C0140B01B0020FB
:10C5E800026D70B515880446ADB2A90613D5036B64
:10C5F8008BB9C36A1BB1908880B298470BE0E16998
:10C60800928840694E1CD2B2E6614254E169E26800
:10C61800914228BFE3612B0613D5636AA26A9A4246
:10C62800236D0AD0511CA069A162825C9A8023699B
:10C63800994206D30023A36270BDDA6822F0800213
:10C64800DA6070BD026B0346C16810B5406942B13B
:10C658001A6C8C1A013A08BF0A46005D1A64C0B207
:10C6680010BD1A6A805C01328A4228BF0022C0B21B
:10C678001A6210BD436B13B190F844007047836A87
:10C68800406A1B1A584258417047036B13B15B68E4
:10C69800016C01E0C369016A8B423CBFC2689B1808
:10C6A800581AC0B27047836A8169426B1944D160D5
:10C6B800416A994297BF0169CB1ACB1A536096BF5A
:10C6C8000023536083624FF0000380F844301368FE
:10C6D80088BF816243F0010313607047436A82692F
:10C6E800D154436A02690133934228BF002343624D
:10C6F800436B1BB11B68DB0705D4D4E7026DD36815
:10C7080043F08003D360704738B50D4B0D4D9968E1
:10C718000D4B1A681C465288114203D0FBF73EFBAA
:10C72800286007E0FBF73AFB2B68984282BFC01AE3
:10C73800064B186023685A68054B5A6138BD00BF1C
:10C74800000C014020240020B00700200400002035
:10C75800000401404171FCF797B88160FCF794B878
:10C768002DE9F04105460E46078A83899BB21F4092
:10C77800002F37D0B7FA87F24FF00043D340DB439E
:10C7880099B21F40A2F11B032982042BF0D8DFE8DD
:10C7980003F0221F1C190300746A24B1013C002312
:10C7A800A4B2736201E0AC8DA4B2D6F82080B8F1CF
:10C7B800000FDDD0D8F80030404621469847D8F819
:10C7C8000480F4E73068A98E08E07068298F05E0D6
:10C7D800B068A98F02E0F068B5F84010036889B224
:10C7E8009847C5E7BDE8F081254B10B55A43254B5E
:10C7F800254C1B680139B3FBF2F20388013AA042C9
:10C8080089B292B29BB212D004F50064A0420ED055
:10C81800B0F1804F0BD0A4F59834A04207D004F5AE
:10C828008064A04203D004F58064A04202D123F0C2
:10C8380070039BB2154CA04206D004F58064A04258
:10C848001CBF23F440739BB203800F4B8185984231
:10C8580002850FD003F5006398420BD003F54063BF
:10C86800984207D003F58063984203D003F58063AC
:10C87800984201D1002303860123838210BD00BFA3
:10C8880040420F0060000020002C014000100040D2
:10C8980073B505460068FFF7A7FF2A6801241388C7
:10C8A80000269BB243F001031380EB7A01A88DF8B0
:10C8B80004308DF805408DF806608DF8074005F0C6
:10C8C80025FFEB7A1B2B0BD1192301A88DF8043017
:10C8D8008DF805408DF806608DF8074005F016FFC5
:10C8E80002B070BD0C4B800A98420CD004D8B0F549
:10C8F800801F0CD101207047084B984205D049335E
:10C90800984206D003E00220704703207047FE20BB
:10C9180070470020704700BF01001000020010009F
:10C928002DE9F84304680746204688469146FFF7F4
:10C93800D9FF03284BD8BA7A9108B8F1000F06D16D
:10C94800A589AEB202258D4026EA0505A5810A23F0
:10C9580003FB00131F4A42F82380043342F8239054
:10C96800B8F1000F07D0BD7AA189AD080223AB400A
:10C978000B439BB2A3812823434303F120011144B5
:10C98800EFF31286502585F3128803F10C051C334A
:10C998001544134455F8047F17B10F602968043112
:10C9A8009D42F7D100230B60F3B283F3118828234B
:10C9B80003FB0020036A23B1A3899BB243F0010360
:10C9C80004E0A38923F001031B041B0CA381BDE829
:10C9D800F88300BFB01B002096E695E694E6014870
:10C9E800FEE500BF242400200048F9E57824002053
:10C9F8000B4B4FF400525A604FF6FE730948D0F8BB
:10CA08008C2011680B401360C26FD0F880309A42B6
:10CA180001D0583047E6012380F89C30704700BFAA
:10CA280000000240202400202DE9F0431E46984BC8
:10CA38008DB09842894690469DF8507057D1954BD5
:10CA4800954A96499A6503F1AC02DA6603F5D672FF
:10CA58001A674FF480725A669A66914AC3F86080E2
:10CA6800C3F88820A2F54842543AC3F8A420C3F872
:10CA7800A020C3F8A800C3F88C108A4B9A6942F426
:10CA880080429A615A6942F001025A6102238DF884
:10CA980003303A074FF40073ADF8003001D51C237A
:10CAA8000FE0B30706D518237F4869468DF8023092
:10CAB80003F0EAFAF5070AD54FF48063ADF80030C1
:10CAC8004823794869468DF8023003F0DDFA0E23D1
:10CAD8008DF804300022012301A88DF805308DF867
:10CAE80006208DF80730714C05F010FE4FE0704BB2
:10CAF800984240F0C880674B674AC3F80C805A6078
:10CB08004FF480725A611A6103F52B729A6103F52A
:10CB18006B72DA61674A5865DA641A65614B3C07DB
:10CB2800DA6942F40032DA615A6942F001025A6164
:10CB38004FF002038DF803304FF00403ADF80030D6
:10CB480001D51C230EE0B00706D5182356486946C0
:10CB58008DF8023003F098FAF10709D50823ADF8EB
:10CB680000304823504869468DF8023003F08CFAAB
:10CB780026238DF804300022012301A88DF8053002
:10CB88008DF806208DF8073005F0C0FD4A4C0025C9
:10CB98000123204684F844302562E561A562656278
:10CBA800C4F82C906671C4F80880A771FBF76CFE76
:10CBB800F20731D5206B002826D0E36C039501934A
:10CBC8004FF480530A9380230693E36805950493F2
:10CBD8002023099363690795029308950B9502F042
:10CBE80011FD01A9206B02F0EFFC226B216D136887
:10CBF80043F0010313608B8A9BB243F040038B829E
:10CC080053689BB2236407E04FF6DF72236D1A80E6
:10CC1800DA6842F02002DA60B3072CD5606B28B3DB
:10CC2800A36C002501934FF480530A938023069345
:10CC38002369029504931023039305950795089596
:10CC480009950B9502F0DEFC606B01A902F0BCFCB3
:10CC5800636B1A6842F002021A60226D5D605D60C3
:10CC6800938A9BB243F08003938204E0226DD368D9
:10CC780043F08003D360226D204693899BB243F42E
:10CC88000053938100E000200DB0BDE8F08300BFA1
:10CC98000038014020240020C4A0010844000240BC
:10CCA800580002400010024000080140782400208B
:10CCB8000044004004440040242400200028114A75
:10CCC800B8BF404290FBF2F330B50F4C3C2504FB53
:10CCD800030068430D4D90FBF2F22D682D7B25B9BA
:10CCE80003EB830303EB830301E0C3EB031302EBC2
:10CCF800830304FB02020B804FF47A7392FBF3F276
:10CD08004A8030BD80969800806967FFD01900205E
:10CD1800022803D0431E584258417047064B1B68EF
:10CD28001B7823B1054B1868C0F3C0407047044B0B
:10CD38001878C0F38000704700060020E410002037
:10CD48008B31002010B50A4C5E280146206805D1B9
:10CD58005D21FBF718F920683E2105E05D2903D124
:10CD6800FBF711F920683D21BDE81040FBF70BB92E
:10CD7800CC28002010B50446C0B2FFF7E3FFC4F387
:10CD88000720BDE81040DDE7024B5E211868FBF77D
:10CD9800FAB800BFCC28002038B50546054C5E21FE
:10CDA8002068FBF7F0F820682946BDE83840FBF713
:10CDB800EAB800BFCC28002013B5044601A90068D2
:10CDC800FFF77CFF1320FFF7E7FFBDF90400FFF72B
:10CDD800D1FF1B20FFF7E0FFBDF90600FFF7CAFFF0
:10CDE8002320FFF7D9FF2368002BB4BF53204E2020
:10CDF800FFF7C0FF01A96068FFF760FF1220FFF787
:10CE0800CBFFBDF90400FFF7B5FF1A20FFF7C4FFF9
:10CE1800BDF90600FFF7AEFF2220FFF7BDFF6368EC
:10CE2800002BB4BF57204520FFF7A4FF02B010BD68
:10CE3800674B73B51878FFF76BFF664D04462B7880
:10CE4800834220D0C8B1644B1B68E3B193F900005A
:10CE580002230093614B04211B6800225B78003396
:10CE680018BF012301934FF41653FCF7B5FC5C4B34
:10CE7800186040B101232B7005E0594E3068FCF76B
:10CE880098FC34602C70574B574D1878FFF740FFCB
:10CE98002B780446834218D088B1544B1B68A3B141
:10CEA8000022012493F9000008214FF496430094CE
:10CEB8000192FCF791FC4E4B186028B905E04C4EE6
:10CEC8003068FCF776FC34602C704A4B4A4D187871
:10CED800FFF71EFF2B78044683422E4643D00028D6
:10CEE80038D0464B1A68002A3DD0D37992F9000011
:10CEF800002B4FF00202424C08BF0223009200228E
:10CF080054F8233001921021FCF766FC3D4B05468E
:10CF1800186040B33C4C94F84A30022B0BD094F87C
:10CF28009620022A01D14C3405E023B1002A04F1ED
:10CF38004C0418BF0024354B1C6044B12046002126
:10CF48004C220AF03EF90223256084F84A30012376
:10CF5800337008E02B4E306805F0DEF83068FCF7D7
:10CF680028FC34602C702A4B2A4D1878FFF7D0FE25
:10CF78002B780446834229D000B3274B1B682BB378
:10CF8800264A93F900001268032352782021002AC8
:10CF98000CBF08220922009301924FF4614300223A
:10CFA800FCF71AFC1E4B186080B11E4A012313704F
:10CFB8002B701D4B1A681D4B1A6007E0184E30681D
:10CFC800FCF7F7FB174B34601C702C7002B070BD77
:10CFD80008060020C411002004060020D0190020F3
:10CFE800CC28002009060020F0190020741A00201F
:10CFF800641A0020140600207A1A00201006002067
:10D00800B8A401087C1A0020202A0020801A0020D9
:10D0180020060020901A00201C0600201806002078
:10D02800941A0020981A0020C02D00209C1A002075
:10D03800642928BF6421F8B501FB00F5642495FB39
:10D04800F4F40646E4B20027FBB2A34204D29F20C0
:10D0580003F07BF90137F7E7B4420BD2142195FBB3
:10D06800F1F5C4EB8410663DC4EB80002844C0B2DF
:10D0780003F06BF90134E4B2B44201D29A20F7E725
:10D08800F8BD2DE9F743FAF789FE924C6368C31A95
:10D09800002BC0F2688300F5433303F5A073636087
:10D0A8008D4B1D78237AC5F38005EB1A18BF012331
:10D0B80025724DB1002B00F05683884B5A789A7030
:10D0C80001225A701A702BE0844A2BB1D37843F0AE
:10D0D8000203D37093785370D67806F0020101F0FA
:10D0E800FF0339B97D498968411A002903DB06F035
:10D0F800010300E0012303F00107784917707BB1B1
:10D10800F2070DD50A7905230132D2B2B2FBF3F347
:10D1180003EB8303D31A724ADBB20B71D35C4B70F7
:10D128006E4EDFF8088233787BB3F37823F002037E
:10D13800F3706C4B0344AE20B36003F02AF908B1D6
:10D1480003F02CF988F80000002800F00C83B020C8
:10D1580003F01FF9402003F01CF9002003F019F92F
:10D16800102003F016F94FF48067013F0020BFB28A
:10D1780003F0E6F8002FF8D1384603F07EF972780C
:10D18800594B53F8220003F0FBF898F80030002BB5
:10D1980000F0E9827378062B00F2B282DFE813F020
:10D1A8000700B002180078006A018701EC014F49B6
:10D1B8004F4A504B5048FDF70AFD012003F05DF936
:10D1C8004D4803F0DDF8022003F057F94B48ACE175
:10D1D8004B4F3B689B0735D5DFF854810A23B8F8D5
:10D1E8000010DFF85091B1FBF3F203FB121399F82A
:10D1F800001092B29BB200913F484249FDF7E7FC0C
:10D20800FEF748F9012003F038F93B4803F0B8F875
:10D218003D4B99F800201868B8F80030067902FBF1
:10D22800163164234B43C17802208E1B5643B3FB4F
:10D23800F6F6F6B203F021F931461520FFF7F8FEAD
:10D24800032600E001263B681F0540F159822F4B59
:10D258002F491F68642397FBF3F2096803FB1273D5
:10D26800009125482B49FDF7B2FCFEF713F930462B
:10D2780003F003F9204803F083F802F011FD074694
:10D28800701C03F0FAF815203946FFF7D1FE37E293
:10D298000120214F03F0F1F8204803F071F83B68B2
:10D2A800980749D51E4A1448B2F90210B2F900305D
:10D2B8000091B2F904201B4901921B4AFDF787FC33
:10D2C800FEF7E8F8022003F0D8F80B4803F058F806
:10D2D800032632E0CC2800208B3100209029002042
:10D2E8002EC00108404B4C00DCA0010833C00108E7
:10D2F8003CC00108C9BC0108D528002043C001086A
:10D308009C2D00204CC00108C8190020D419002009
:10D31800D819002064C00108DC19002079C0010870
:10D32800CE1100208FC001089EC001084D020020C8
:10D33800CC1900205400002002263B68D9071AD5D2
:10D348007B4A7C48B2F90210B2F900300091B2F978
:10D35800042079490192794AFDF739FC06F1010860
:10D36800FEF798F8304603F088F85FFA88F87148B5
:10D3780003F006F846463B681A0718D5704A6D4808
:10D38800B2F90210B2F900300091B2F904206A49EA
:10D3980001926C4AFDF71BFC771CFEF77BF83046C0
:10D3A80003F06BF8FFB2634802F0EAFF3E46664AB4
:10D3B8006149B2F90030B2F902205E480092634A2E
:10D3C800DFF8B091B2F90020771C0192604AFDF7AE
:10D3D800FEFBFEF75FF8304603F04FF8554802F0C1
:10D3E800CFFF5449D9F80000FDF78CFA514809F0ED
:10D3F8002CFFFFB2C1B2092909D84B1CDBB221446A
:10D4080020224A720021E21891721946F3E7DFF8E8
:10D418002481D9F804004144FDF774FAFEF73AF87C
:10D42800384603F02AF8404602F0AAFF4146D9F8E8
:10D438000800FDF767FA404609F007FF0236F6B222
:10D44800C7B2092F09D87B1CDBB2274420227A7285
:10D458000021E21891721F46F3E73E4BB3F9000032
:10D4680006F0A8F808EB0701FDF74CFAFEF712F8EA
:10D47800304657E00026384F3B78B34240F24081AF
:10D488000E2E00F03D817008013002F0F6FF3046A4
:10D4980005F0AEFB3B78B34206D9202002F055FFD9
:10D4A800701CC0B205F0A4FB0236F6B2E3E72B4EBF
:10D4B8002B4996F8B0271F48FDF789FB012002F099
:10D4C800DCFF1C4802F05CFF264B27491F781948EF
:10D4D8003A46FDF77CFB022002F0CFFF154802F028
:10D4E8004FFF0C2303FB0766204996F8B32796F8ED
:10D4F800B2371048FDF76BFBFDF7CCFF032002F0B5
:10D50800BCFF0C4802F03CFF96F8B81796F8B6270F
:10D5180096F8B737074800911549FDF758FBFDF70E
:10D52800B9FF042002F0A9FF024802F029FFE7E052
:10D5380004110020D52800208FC00108A2C00108CE
:10D548000A1100202CD70108942D0020DC1100209E
:10D55800A6C0010884080020BC2A0020EC11002085
:10D56800AAC00108482D0020B6C00108C7C001089C
:10D57800D8C00108780800207C4B1B681B0640F1C6
:10D58800BB80236A616A7A4A8B421CBF536292F855
:10D5980028304FF001011CBF013303F003034FF0A3
:10D5A800000018BF82F8283002F073FF94F8283082
:10D5B800704A0026D05C02F0C8FE0220012102F069
:10D5C80068FF6D4B3620F35C0136C3EBC30393FB56
:10D5D800F0F0C0B2062828BF06206038C0B202F0BA
:10D5E800B4FE102EEDD1654B65491B78654813F0E4
:10D5F800020F654B1A7814BF59234E23FDF7E7FA3B
:10D60800FDF748FF022002F038FF5E4802F0B8FE3E
:10D618005E495F4B4E680A685A4892FBF3F25D49CF
:10D6280096FBF3F3FDF7D3FAFDF734FF032002F07E
:10D6380024FF544802F0A4FE574B58491A88514811
:10D64800FDF7C5FAFDF712FF042002F016FF4D485A
:10D6580002F096FE524B53491A884A48FDF7B7FA2A
:10D66800FDF704FF04210A2002F013FF454802F0E9
:10D6780087FE4D49E26A4348FDF7A9FA4B4EFDF78C
:10D68800F5FE052002F0F9FE3E4802F079FE7268C8
:10D69800B36847493B48FDF79AFAFDF7E7FE0521CD
:10D6A8000A2002F0F6FE374802F06AFE3369F26893
:10D6B8004049D21A3348FDF78AFAFDF7D7FE06200B
:10D6C80002F0DBFE2F4802F05BFEB2683A492D48B3
:10D6D800FDF77DFAFDF7CAFE06210A2002F0D9FE01
:10D6E800284802F04DFE35491522264809F0D8FD94
:10D6F800FDF7BCFE072015E7F37843F00203F3704B
:10D70800002D30D12E4B002193F820301220052B0C
:10D7180097BF2C4A3F259B181D7F02F0BAFE28466A
:10D7280002F013FE1320002102F0B3FE264B1B78F3
:10D73800002B264B18BF72201B7808BF2120002B16
:10D7480018BF522002F001FE1420002102F0A1FEB1
:10D7580094F83050074B585D013505F0030502F089
:10D76800F4FD84F8305003B0BDE8F0839C2D002010
:10D77800CC280020EAC0010895110020E0190020FB
:10D78800EFC00108D5280020E6190020E81900207C
:10D798008096980000C10108E21900200DC1010817
:10D7A8004C11002015C101081CC10108B407002054
:10D7B80023C101082CC1010833C10108C00200209F
:10D7C80034310020DCA001083B0F0020A00F00200E
:10D7D800064B1B7803F0040303F0FF001BB1044B56
:10D7E8001888C0F3C01000F0010070478B3100208A
:10D7F800A41A00202DE9F04F89B00593BE4B0026EE
:10D80800B3F90290B3F90030B9F1000FB8BFC9F10C
:10D818000009002BB8BF5B429945B8BF99468046BE
:10D82800B2463446B9F5FA7F04910392A8BF4FF483
:10D83800FA79019000960296B04D2B88990754D03A
:10D84800AD4B610033F91420AD4B33F9143003EBC1
:10D858004202039B5B429A4203DB039B9342A8BFAD
:10D868001346A84A8F5E059ADB1B32F914001F186D
:10D87800FFF7AEFF90B1A44B384613F804A005F0AB
:10D8880099FEA24905F09EFF0146504604F0B8FFF4
:10D898009E4905F0E3FE06F0A7F8074698F8083019
:10D8A80064227B4393FBF2F398F81C206FF0040A80
:10D8B8000AFB02FA534504DB02EB820A9A45A8BF29
:10D8C8009A4642F21072924B53F824003844904220
:10D8D800A8BF10468F4A9042B8BF104643F82400AC
:10D8E80098F812305843031302932D8805F0030368
:10D8F800012B38D0804B884933F91430A6000093A7
:10D90800019B51F8247093F801E0844B33F914001B
:10D9180080EAE073A3EBE073B3F5206F16DC009A9E
:10D9280050235A4392FBFEF3042290FBF2F0181A9C
:10D938000744B7F57A5F7A4BA8BF4FF47A579F42EE
:10D94800ACBF41F8247041F8243002E0002341F8CC
:10D9580024308B597D2693FBF6F6019BDB7A7343C3
:10D96800402693FBF6F6AA0712D5009A09FB06F59E
:10D9780009FB02F70298C9F5FA7303FB0A7703FB60
:10D9880000534FF4FA7297FBF2F193FBF2F505E0BE
:10D99800EB0755BF354651460099029D5F4B04275A
:10D9A80033F914305F4A93FBF7F3A25C6FF04F072B
:10D9B800534393FBF7F398F851204FEA440BCF18E1
:10D9C80072B13846069205F0F5FD5749574B01EB01
:10D9D800C401069A1B68FCF7CFFE06F005F8074657
:10D9E8004E4B534A3BF803003BF9021003B25B1A53
:10D9F800042193FBF1F102F1040E5EF824302BF8B8
:10DA080002000C3252F8240042F8243098F85020D2
:10DA180018444FEA840C08444EF8241082B1CDF81B
:10DA28001CC0069205F0C6FD4249404B01EBC401FB
:10DA3800069A1B68FCF7A0FE05F0D6FFDDF81CC0AF
:10DA48003D4BDFF810E11B5D7A195843202390FB0A
:10DA5800F3F3D21A2BF80E20384A5B424CF8023006
:10DA6800019B3748374901334CF801504CF8007096
:10DA7800019375460CB90124DEE61F4B0427B3F960
:10DA88000440049B244E9B79D6F808E00F335B00D2
:10DA98006343224C5B11B4F90440002B94FBF7F765
:10DAA800A3EB0707B8BF5B42322B98F80D400BDC9D
:10DAB80004FB07E4244BA342A8BF2346234CA342FC
:10DAC800ACBFB360B46001E00023B36098F80340D2
:10DAD80004FB07F31E4C9B112478032C3DD9B8F89E
:10DAE8004E40B4F5FA7F38D26742BB4234DBA342DA
:10DAF800A8BF234631E000BFE4110020A41A00208B
:10DB080084310020942D00207C9B010800002041D6
:10DB180000290020F0D8FFFFC81A002004110020B7
:10DB280080C1FFFF501B0020AC1A0020C41A00203F
:10DB380008290020F81A0020641B0020301B002050
:10DB4800181B0020241B0020FEFFFF0F020000F01E
:10DB5800671B0020101B00203B46B4686FF0FF06CF
:10DB680044F34F34B4F5807FA8BF4FF48074B442B7
:10DB7800B8BF344683601E190023AE808C60936062
:10DB880009B0BDE8F08F2DE9F04F87B00393B44B8F
:10DB980081461D88029105F00205ADB2019295B14A
:10DBA800B04BB3F90250B3F90030002DB8BF6D4245
:10DBB800002BB8BF5B429D42B8BF1D46B5F5007F3C
:10DBC800A8BF4FF40075CB460026A64BA64933F9EB
:10DBD8001620A64B4FEA460A33F91630520083EA5C
:10DBE800E374A4EBE374B4F5206F4FEA860851F8A8
:10DBF800260011DC042493FBF4F3D31A0344B3F591
:10DC08007A5F9B48A8BF4FF47A538342ACBF41F870
:10DC1800263041F8260002E0002341F8263051F86A
:10DC280008709BF80B30FF119BF801405F438C4B49
:10DC380054431B88BF119B074FEAA41456D08D4B41
:10DC48003AF903301A44019B5B429A4203DB019B79
:10DC58009342A8BF1346884A3AF902209B1A039AAE
:10DC680032F916201A440492FFF7B2FD049A98B1CB
:10DC7800824B10469B5D049305F09CFC804905F09F
:10DC8800A1FD049B0146184604F0BAFD7C4905F045
:10DC9800E5FC05F0A9FE024642F21070794958F8F1
:10DCA800013013448342A8BF034677488342B8BF74
:10DCB800034648F8013099F8081099F81C004A43BF
:10DCC80000EB8000D21141428A4203DB8242A8BFA6
:10DCD8000246114699F81220641A53431B13FF1A7F
:10DCE8006F436C4303EB672701EB64245F4B04220B
:10DCF8003AF9033093FBF2F2644B9B5D534399F876
:10DD08005120A4EBA31472B12046049205F052FCF2
:10DD18005F49604B01EBC601049A1B68FCF72CFDB8
:10DD280005F062FE044651495B4B3AF801003AF9A6
:10DD380003E002B2CEEB02024FF0040E92FBFEF2B9
:10DD48002AF803009E440C3358F80EC058F8030014
:10DD580048F80E206044104499F8502048F803C051
:10DD68008C467AB10591049205F024FC4B49494B45
:10DD780001EBC601049A1B68FCF7FEFC05F034FEB3
:10DD8800DDF814C0464BDFF834E19B5DE2194343EC
:10DD98005B11D21A2AF80E2042484349434A5B4293
:10DDA80048F8004048F8017048F802300BF1010BC0
:10DDB80074460EB9012608E72A4B0427B3F9045024
:10DDC800029B294E9B79D6F808E00F335B006B4322
:10DDD800BCF904505B1195FBF7F7002BA3EB070781
:10DDE800B8BF5B42322B99F80D500BDC05FB07E5F9
:10DDF8002F4BAB42A8BF2B462E4DAB42ACBFB360F6
:10DE0800B56001E00023B36099F8035005FB07F300
:10DE1800294D9B112D78032D0CD9B9F84E50B5F525
:10DE2800FA7F07D26F42BB4203DBAB42A8BF2B4647
:10DE380000E03B46B5686FF0FF0645F34F35B5F592
:10DE4800807FA8BF4FF48075B542B8BF3546836060
:10DE58005E190023A6808D60936007B0BDE8F08F3F
:10DE6800A41A0020E4110020C81A00200411002080
:10DE780080C1FFFF84310020942D00207C9B010885
:10DE88000000204100290020F0D8FFFF501B00208F
:10DE9800AC1A0020C41A00201C290020F81A0020FF
:10DEA800641B0020181B0020241B0020301B0020AE
:10DEB800FEFFFF0F020000F0671B0020101B002070
:10DEC8002DE9F04F89B00593AE4B0027B3F90280D6
:10DED800B3F90030B8F1000FB8BFC8F10008002B43
:10DEE800B8BF5B429845B8BF98468246B946BB461C
:10DEF8003C46B8F5FA7F0492A8BF4FF4FA7802902E
:10DF08000397A14D2B88990757D0022C55D09D4BCC
:10DF1800610033F914209D4B33F9143003EB4202AE
:10DF2800049B5B429A4203DB049B9342A8BF1346BF
:10DF3800974A8E5E059A9B1B32F914001E18FFF74C
:10DF480047FC90B1934B304613F804B005F032FB10
:10DF5800914905F037FC0146584604F051FC8E49BA
:10DF680005F07CFB05F040FD06469AF8083064226F
:10DF7800734393FBF2F39AF81C206FF0040101FB42
:10DF880002FB5B4505DB02EB82029342A8BF134606
:10DF98009B4642F21072814B53F824003044904261
:10DFA800A8BF10467E4A9042B8BF104643F82400E6
:10DFB8009AF81230584303130393298801F0030396
:10DFC800012B01D1022C3DD16E4B764D33F91490C3
:10DFD800029BA00093F801E0734B55F8247033F9C5
:10DFE800146086EAE673A3EBE673B3F5206F1CDCD6
:10DFF800022C14D0502303FB09F292FBFEF30422F7
:10E0080096FBF2F69E1B3744B7F57A5F674BA8BFBD
:10E018004FF47A579F42ACBF2F502B5007E089EA44
:10E02800E973A3EBE973642BE4DD00232B505D4B0C
:10E038007D27C35893FBF7F7029BDB7A7B43402786
:10E0480093FBF7F78A0713D5022C11D008FB07F5C5
:10E0580008FB09F60398C8F5FA7303FB0B6603FB84
:10E0680000534FF4FA7296FBF2F193FBF2F508E0D5
:10E07800CB0704D5022C02D0039D594601E03D464A
:10E08800494663000193484B042633F91430484A43
:10E0980093FBF6F3A25C6FF04F06534393FBF6F342
:10E0A8009AF85120CE18E2B1022C069230460BD1D4
:10E0B80005F080FA069A530803D09A42A8BF1A4678
:10E0C80000E001223B4905E005F074FA3A49069A56
:10E0D80001EBC401394B1B68FCF74EFB05F084FCCF
:10E0E8000646314B019A0198D15A354B0AB2C05EA7
:10E0F8004FEA840C121A042092FBF0F20198C152E4
:10E1080003F10801143351F824E053F8240041F8CE
:10E118002420704410449AF8502043F824E082B137
:10E12800CDF81CC0069205F045FA2649234B01EBB1
:10E13800C401069A1B68FCF71FFB05F055FCDDF8C7
:10E148001CC0214B214A1B5D01995843202390FB99
:10E15800F3F073191B1A8B521D4B40424CF80360A5
:10E168001C4B01344CF803501B4B032C4CF8030098
:10E17800029B03F1010302937FF4C3AE09B0BDE82B
:10E18800F08F00BFE4110020A41A00208431002081
:10E19800942D00207C9B01080000204100290020CC
:10E1A800F0D8FFFFC81A00200411002080C1FFFF2B
:10E1B800501B0020BC1A0020AC1A0020C41A0020F2
:10E1C80030290020F81A0020641B0020101B0020B2
:10E1D800181B0020241B0020301B00202DE9F04FC5
:10E1E80089B005939D4B80461B880C469B0702927D
:10E1F8004DD540F2E631129B994AD889B2F90030E0
:10E208001B1A03F2F3158D4203D8002BB8BF5B42EB
:10E2180001E04FF4FA73B2F90220101A40F2E63224
:10E2280000F2F311914203D80028B8BF404201E040
:10E238004FF4FA7098F84C503DB39842B8BF18465E
:10E24800C0F5FA7005F0B6F9864905F0BBFA4FF04B
:10E258007E5105F0F9F80646642090FBF5F005F0CC
:10E26800A9F90146304605F0F9F94FF07E5105F05D
:10E27800EDF80021074605F08FFB30B938464FF01E
:10E288007E5105F0A7FB20B101E0002701E04FF027
:10E298007E57E31C0393CDF800800024039B022CD7
:10E2A80013F8015F704E039309D1B6F904000A35DB
:10E2B800684305F07FF96D4905F084FA74E036F992
:10E2C800140005F077F98146029805F06FF9654961
:10E2D80005F078FA0146484605F0C0F9644B8146D6
:10E2E80033F9140005F066F90146484605F0AEF822
:10E2F800029B8146584205F05DF9834648465946D7
:10E308004FEA440A05F048FB48B9029805F052F96B
:10E3180083464846594605F05DFB00B9CB46554B48
:10E3280033F90A0005F046F90146584605F08CF81D
:10E33800059B814633F9140005F03CF9014648462F
:10E3480005F084F84C4905F03DFA8146FFF740FA9C
:10E3580028B14A4B4946185D04F052FA81463F4BB2
:10E36800B3F800B01BF0010F05D04846D8F84410A8
:10E3780005F074F918E036F90A001435684305F019
:10E3880019F93A4905F01EFA1BF0020F05460CD0A0
:10E39800D8F84810484605F061F9394605F05EF9A5
:10E3A8000146284605F052F8054663000493344BAD
:10E3B800344E33F9140005F0FDF8334B196E05F0AF
:10E3C8004DF90146284605F03FF8009B8246196A38
:10E3D80005F044F92D4B0546185D05F0EBF80146AC
:10E3E800284605F03BF92A4905F0ECF998F8512040
:10E3F800814692B1022C09D1530803D09A42A8BF92
:10E408001A4600E001224846224902E0224901EB6F
:10E41800C4013368FCF7B0F98146336850461946A1
:10E42800019305F01BF9009BDFF878B0D96A05F075
:10E4380015F9114905F012F95BF8241005F006F8F2
:10E448001649A500064605F0A7FA68BB30461449E8
:10E4580005F0C0FA48B3124E27E000BFA41A002006
:10E46800D82D00200000FA43E411002000004842A3
:10E4780084310020942D0020000020417C9B01085D
:10E4880004110020C41A002000290020A81A002026
:10E498000000C842BC1A0020AC1A002000007AC351
:10E4A80000007A43441B0020444E4BF80560DFF817
:10E4B8003CB1504655F80B1004F0C6FF45F80BA0C8
:10E4C800069001994FF07E5005F07CF9069B0146B5
:10E4D800184605F0C3F882460BF10C03EA580BF115
:10E4E800180B104655F80B100793069204F0AEFF70
:10E4F800514604F0ABFF069A079B45F80B2098F8A5
:10E508005020014645F803A032B12D49019B01EB8B
:10E51800C401FCF731F9014608462A4905F052F9C9
:10E52800009B996B05F09AF8274B8246185D05F019
:10E5380041F80146504605F091F8244905F042F9A2
:10E548002349824605F028FA38B95046214905F092
:10E5580041FA20B1DFF87CA001E0DFF874A0314671
:10E56800484604F073FF514604F070FF09F036F88E
:10E57800194BB0F57A7FA8BF4FF47A709842B8BFAC
:10E588001846049A154B0134D052484605F02CFA27
:10E59800134B5851304605F027FA124B5851504644
:10E5A80005F022FA104B032C5851009B03F1040389
:10E5B80000937FF473AE09B0BDE8F08F00007AC312
:10E5C800F81A002000004040A81A00200000C842A5
:10E5D800000096C30000964318FCFFFF101B0020A4
:10E5E800181B0020241B0020301B00206429002059
:10E5F800044B00221A605A60034B00221A605A60CA
:10E60800704700BF002900203C1B002010B50C4CAF
:10E618000123E3704FF48060022384F82030FCF774
:10E628006FFC084A084BD2F888201B68527864218E
:10E6380001FB0233636123880133238010BD00BFCF
:10E648003431002000290020C02D002038B50024D6
:10E658000B4D6059254403F04FFE696811B1094814
:10E66800FCF7CAFAA96811B10748FCF7C5FA0748C8
:10E67800103403F041FEB4F5E87FE9D138BD00BF9E
:10E6880000A101086CC1010872C10108E5CB0108AD
:10E69800F0B585B0044608F0D8FD082826D1621EDA
:10E6A800E01D1F4912F8013F09681944497801F033
:10E6B8000301022908BF203B82421370F1D125468D
:10E6C80004F1080715F8016B1648314608F0AFFD4C
:10E6D80020B12846314608F0AAFD10B1FAF798FC97
:10E6E8001CE0BD42EED1204600F0D6FE0E4803F0F5
:10E6F80003FE00230D4A04A91A4492F88A210A4409
:10E708000849595C0133082B02F80C1CF2D100238C
:10E71800074801A98DF80C30FCF76EFA05B0F0BD7A
:10E728006800002030D7010878C10108EC110020EA
:10E7380027CB01082A4B2B4C1E6880B52068FBF7B5
:10E748002DF83046FBF72AF8206841798D0703D465
:10E7580041F00201F9F708FC234B08221A61234D06
:10E7680010221A612B689A0341BF06236371E3796B
:10E7780023F0010344BF43F00203E3712068F9F773
:10E78800FFFB90B1184F08237B61164B1868F9F707
:10E79800F4FB8046FDF766F908B102F035FA304619
:10E7A8004146F9F7F0FB08233B613046F9F7E8FBEF
:10E7B80078B10D4F4FF01008C7F814803046D4F8E0
:10E7C8000090F9F7DAFB01464846F9F7DCFBC7F891
:10E7D80010802B689B03D1D5FEF753FCCEE700BF12
:10E7E800642D00208C290020000C01409C2D002065
:10E7F8002DE9F047054608F028FD2F4E0446D6F8C7
:10E80800088090B92D4803F077FD2D4B53F824105C
:10E8180049B10123A34013EA080F02D02948FCF7A5
:10E82800EBF90134F1E7284822E028462749224637
:10E8380008F014FD58B9264803F05EFD254C54F83D
:10E84800041F0029EFD01F48FCF7D6F9F7E72B780B
:10E858004FF000092D2B03BF013504F1FF344FF0B1
:10E86800010A4FF0000A164B53F8297027B91A48C5
:10E87800BDE8F04703F040BD28463946224608F077
:10E88800EDFCA8B9012000FA09F0BAF1000F03D095
:10E89800FCF746FB114803E040EA0800B060104866
:10E8A80003F02AFD3946BDE8F0470E48FCF7A4B945
:10E8B80009F10109D7E700BFEC1100207EC101086A
:10E8C800D0A2010888C10108E5CB01088CC1010864
:10E8D80091C10108CCA201084EBF01089DC10108E1
:10E8E800A6C1010826CB010810B5084803F004FDAD
:10E8F800074B00241C741C64064B1C70F9F7E6FCDB
:10E9080003F0D2FE044B1C6010BD00BFAEC101086D
:10E918008C2900208C310020642D002070B506461B
:10E9280000240B4BE518AA8816420AD0E15809487A
:10E93800FCF762F92846002103F06FFC064803F053
:10E94800DBFC40F6BC4314349C42EAD170BD00BFE6
:10E95800E4AC0108DAC10108E5CB010808B50848AC
:10E96800FCF74AF9FDF7ECFD01F090FC18B96420BA
:10E97800F9F73BFAF8E70348BDE80840FCF73CB96B
:10E98800E4C10108F1C101082DE9FF410A480688E0
:10E9980085684488B0F80480C768FDF7D9FCCDF8CD
:10E9A80000800290019731462A4623460348FCF727
:10E9B80023F904B0BDE8F0811C000020F9C101086A
:10E9C800F0B504788BB005460CB1002436E04B4B0B
:10E9D80019680E2303FB0411B1F91D51B1F919216E
:10E9E800B1F91B31009591F8205101F58C70019512
:10E9F80091F8215101F59071029590F90700039063
:10EA080091F902103E48049121460134FCF7F4F8CC
:10EA1800082CDCD170E02D2B14D1072C1BDC2846E8
:10EA280008F068FC0AAB661C03EB440424F8100CDD
:10EA380015F8013F303B092BFAD934462B78002BC7
:10EA4800E9D104E0A3F13002092A09D8E5E7082C46
:10EA5800BDF8182009D00BB0BDE8F040FAF7D8BAD5
:10EA6800202BF8D101352646E7E7072AF3D840F2EC
:10EA7800DC55BDF81A00214BA0F2EE2189B2A9425B
:10EA88001B68E8D8BDF81C10A1F2EE24A4B2AC4271
:10EA9800E1D8BDF81E6004B237B2A742DBDB0DB285
:10EAA800AF42D8DCA542D6DBBDF8247007F1640478
:10EAB800A4B2C82CCFD8BDF826E00FFA8EF4112CDA
:10EAC800C9DCBDF82050B42DC5D8BDF82240B42CFF
:10EAD800C1D812B24FF00E0C0CFB0233A3F8190187
:10EAE800A3F81B11A3F81D6183F8205183F8214175
:10EAF80083F81F7183F822E10BB0F0BD20110020CC
:10EB080056C20108F0B504468FB0204608F09DFBB8
:10EB1800C5B21DBBAB4803F0EFFBAB4C94F8D61065
:10EB280009B9AA4853E049B294F8D42094F8D530EA
:10EB3800009194F8D710A648019194F9D810073499
:10EB4800029194F9D210039194F8D31004912946B4
:10EB58000135FCF751F8102DE0D1E2E720469D4938
:10EB6800052208F07BFB0546B8B929469A48702269
:10EB780008F027FB2846994B19680E2303FB00135E
:10EB880001300022082883F8232183F8242183F800
:10EB9800252183F82621F0D112E12046904904224C
:10EBA80008F05CFB05462046002D4AD1202108F0DC
:10EBB8003EFB002800F00481461C304608F045FB67
:10EBC8002C460746874B53F824502DB986480FB07A
:10EBD800BDE8F040FCF710B830462946FAB208F014
:10EBE8003DFB01340028EDD1774A164602F1700149
:10EBF800002382F8DA3082F8D63082F8D53082F8ED
:10EC0800D43007328A42F3D1784901EBC40191F834
:10EC18002822934210DAD1F82C72C3EBC302B01841
:10EC28003A44176800F1D401C0F8D47090880133D1
:10EC3800888092798A71E7E729466D48FBF7DCFFFF
:10EC48008FE06C49072208F009FB05462046002D95
:10EC580049D1202108F0EBFA064608F0F6FAC4B2CA
:10EC68006CBB6548FBF7C8FF214664480134FBF7D5
:10EC7800C3FF0E2CF8D15548FBF7BEFF00246048AF
:10EC88002146FBF7B9FF0025544A012311680E22DB
:10EC980002FB0412D2F82321AB401342594B5A49C4
:10ECA8005A4808BF19460135FBF7A6FF0E2DEBD1D0
:10ECB80046480134FBF7A0FF082CE0D180E030463D
:10ECC800534908F01BFB2C4600284CD0022C4FD08F
:10ECD80008F010FB06AB43F824004D49002008F06B
:10ECE8000DFB0134F0E74A4908F008FB002460B145
:10ECF800082C38D008F0FEFA06AB43F82400444943
:10ED0800002008F0FBFA0134F1E7082C2BD1069B10
:10ED18000F2B28D8DDF81CE0BEF1070F23D8089F79
:10ED28000D2F20D8099E06F16402C82A1BD80A9D17
:10ED3800FF2D18D80B98642815D80C99642912D877
:10ED4800884210DA0D9C032C0DD8324AC3EBC3035A
:10ED5800134483F804E05F719E71DD711872597273
:10ED68009C722D4CD1E60FB0BDE8F040FAF750B9CF
:10ED7800069B072B20D807990D291DD80278722ADF
:10ED88000DD06E2A18D1154A0E20126800FB0323F5
:10ED980001228A40D3F8231121EA020209E00F4A2E
:10EDA8000E20126800FB032301228A40D3F82311A6
:10EDB8000A43C3F8232101E0FAF72AF90D4CA4E627
:10EDC8000FB0F0BD7EC20108EC110020E5CB0108B0
:10EDD800A9C201081EBF0108C0120020201100208E
:10EDE80049BF0108A0B901084EBF010800A10108E8
:10EDF8005DBF010876C2010876C10108C5C20108D5
:10EE080019C10108FACF010840CF0108CAC2010898
:10EE1800CEC20108BC1200207BBC01082DE9F743D3
:10EE2800047805468CB9324D95F8AB12B5F8A8228E
:10EE380095F8AA322F48009121460134FBF7DCFEF1
:10EE4800102C05F10405EFD14EE008F053FA0F2815
:10EE5800044636DC2846202108F0E9F9264EE4B2BB
:10EE6800D6F84480451CA4000027284608F042FA3A
:10EE78005FFA87F9B9F1010F83B208D0B9F1020F2F
:10EE88000BD0B3F5B47F24D2726C13530AE0FF2B76
:10EE98001FD8736C2344987004E0FF2B19D8736C47
:10EEA8002344D87028462C2108F0C1F9054608B13A
:10EEB800013502E0B9F1020F0BD10137032FD4D18C
:10EEC80012E00E4800210F2203B0BDE8F043FAF724
:10EED8001CB808EB04000021042208F072F903B002
:10EEE800BDE8F043FAF794B803B0BDE8F08300BF7B
:10EEF800EC110020D0C201088C290020DCBE0108DA
:10EF08002DE9F04FAB498BB0044608F063F9AA49E4
:10EF1800002820460CBF0125072508F05BF9A74902
:10EF28000028204608BF022508F054F9002808BF29
:10EF38000425E90740F1E680A14803F0DDF9002047
:10EF480002F0EAFF9F4CA04803F0D6F99F4803F06F
:10EF5800D3F963799E4A013B52F823109D48FBF789
:10EF68004BFE9D48FBF748FE26460027D6F814803E
:10EF78000021404604F006FD20B19848FBF73CFE0E
:10EF8800002669E039469648D6F818B0D6F81CA08D
:10EF9800D6F82090FBF730FE4046002104F0FCFC38
:10EFA80010B1202003F0A0F906A94046FBF7AAFCFF
:10EFB80001468C48FBF720FE5846002104F0ECFC83
:10EFC80010B1202003F090F906A95846FBF79AFCE7
:10EFD80001468448FBF710FE5046002104F0DCFC93
:10EFE80010B1202003F080F906A95046FBF78AFCEF
:10EFF80001467C48FBF700FE4846002104F0CCFCA3
:10F0080010B1202003F070F906A94846FBF77AFCF6
:10F01800013701467448FBF7EFFD0C2F06F1100687
:10F02800A4D1AAE749B294F8D42094F8D530009135
:10F0380094F8D7106D48019194F9D81007340291CB
:10F0480094F9D210039194F8D31004913146013603
:10F05800FBF7D2FD102E03D094F8D6100029E1D189
:10F06800634803F049F9574B624C9F6854F8041FF2
:10F0780019B16148FBF7C0FDF8E70E465F4B53F83E
:10F0880026404CB10123B3403B4203D05C482146A3
:10F09800FBF7B2FD0136F1E75A4803F02DF9214696
:10F0A800484B0AAA0B4493F88A311344564A8A5C9F
:10F0B8000131082903F8102CF2D1002306A953487E
:10F0C8008DF82030FBF798FD514803F015F95148A9
:10F0D800FAF7DEFB504803F00FF94E48F9F79EFFA8
:10F0E8004E4803F009F94B48FFF798FE4C48FBF7E8
:10F0F80083FD4020FFF712FC4A4803F0FDF845481D
:10F10800FAF7B0FAAA0739D5474803F0F5F847489F
:10F1180003F0F2F83F4802F03FFF454803F0ECF8EF
:10F128003C48F9F7FFFE434803F0E6F83948FAF798
:10F13800EBF94148FBF760FD3648FAF77BF83F48A2
:10F1480003F0DAF83348FFF73BFC00260E27774335
:10F1580000243B4A0123926CA3403A44D2F80A2087
:10F1680013421ED101340E2CF3D10136082EEDD1F5
:10F178002B48FBF741FD8020FFF7D0FB6B0716D526
:10F18800304803F0B9F8304803F0B6F8214802F0E7
:10F19800DDFE2348FBF730FD4FF48070FFF7BEFB20
:10F1A80005E0314622462948FBF726FDDAE70BB091
:10F1B800BDE8F08FE4C201082DC70108EBC20108C1
:10F1C800F1C20108EC110020FFC2010811C30108B7
:10F1D800A0B901081DC3010828C3010835C30108E7
:10F1E80042C3010875C1010827CB01085AC30108A9
:10F1F8004AC30108CCA2010879C30108D0A20108BA
:10F2080087C3010894C3010830D70108A0C30108C7
:10F21800A9C301087BBC0108B8C30108C4C301081D
:10F22800E5CB0108D2C30108DFC30108F2C3010816
:10F2380000C401080AC4010819C4010827C4010848
:10F248008C29002033C4010844C4010856C40108AD
:10F25800084BDA68D10709D4DA68520708D4DB68A2
:10F2680013F0100F14BF03200420704701207047CB
:10F278000220704700200240704701207047704705
:10F2880003788B4286BF024B33F811000020704789
:10F29800D829002008B50021062207F092FF012096
:10F2A80008BD08B50021062207F08BFF012008BD24
:10F2B80070B50546F8F772FD324CA369A061C31A10
:10F2C800B3F5FA5FE36182BF002384F8203084F845
:10F2D800213094F820302BB9A12D02BF294A0121F1
:10F2E80082F8211094F82110264A31B1D118EDB2D4
:10F2F800013381F8225082F8203094F8205094F895
:10F308004330AB423CD11F4B93F84430052B02D01D
:10F31800062B03D02FE0002003F0A6FF94F823303B
:10F328001E2B28D100200246C1B26B1E99421ADA60
:10F33800214491F822300821DBB283EA0206F6075D
:10F3480044BF83F01803C3F3460301F1FF3154BFF0
:10F358005B0843F0800311F0FF01C2F34702ECD1D0
:10F3680001301A46E0E7234493F822309A4202D14A
:10F37800032003F079FF002384F8213084F820303B
:10F3880070BD00BFD829002010B50446B0F90000B0
:10F3980002F039FBB4F9020002F035FBB4F90400BD
:10F3A800BDE8104002F02FBB10B50446006802F01B
:10F3B8002AFB606802F027FBA068BDE8104002F055
:10F3C80022BB2DE9F74F0120FAF728FB002488B368
:10F3D800012C2FD84FF04C0909FB04FA174E06EB05
:10F3E8000A0808F19007BD7815B10134E4B2EEE7D8
:10F3F80090F9003090F804E01846114B03228DE88C
:10F40800240001212A4653F82E30FAF7E5F98346FD
:10F4180060B106F14800504429464A4607F0D1FE3B
:10F4280001231C44C8F848B0BB70E4B20120FAF7C5
:10F43800DBFACCE703B0BDE8F08F00BFD829002085
:10F44800B8A401080021222210B5104807F0B9FE1F
:10F458000F4B002219460F480424105C013283F830
:10F46800F60183F8FB4105200024042A83F8FA01F9
:10F4780083F8FD4183F8FC0103F10803EBD1012374
:10F48800A1F8F831522381F8F43110BDE0130020BF
:10F49800EC1100209EC8010870B50646441E14F8F9
:10F4A800011F89B1094D284607F0C1FE0028F6D092
:10F4B80005F1080398423FBF054B401BC018A31B2A
:10F4C80038BF80F88A31EAE770BD00BF30D701083D
:10F4D800EC11002007B51C4B03F1E402C3F8E0204F
:10F4E8001A4A92F892215AB1012A14D1032183F8B9
:10F4F800E610072183F8E82083F8E7100C2208E0DB
:10F50800022183F8E610032183F8E82083F8E71046
:10F51800072283F8E4200E4A0E4B40201A60FAF7BF
:10F528007DFA70B10122002390F9000040218DE896
:10F538000C00094A4FF4E133FAF74EF9003018BFCE
:10F54800012003B05DF804FBD8290020EC1100204D
:10F558002D30010834000020DD3001080120002191
:10F5680002F028BE174AF0B5164692F8E930D2F8EC
:10F57800ECE0032B10D85C1C0EEBC3039D1CE4B21B
:10F5880008D09A88D10705D5104203D008E0013188
:10F59800042907D12346ECE786F8E9300020F0BDBE
:10F5A8009F7800210C2202FB01F3064D05F1F00CB7
:10F5B8001CF803209742EAD12B4485F8E940D3F898
:10F5C800F400F0BDD82900208A6810B50C6A0368D9
:10F5D80014430A6923F4FF4314434A6923F0700370
:10F5E80014438A691443CA6914434A6A14438A6AE9
:10F5F800224313430360CB6843600B6883604B6806
:10F60800C36010BD4FF6FE73026813400360002309
:10F61800036043608360C360284B984201D1284A45
:10F6280027E0284B984201D1254A2AE0264B9842E8
:10F6380001D1234A2DE0254B984201D1204A30E0E0
:10F64800234B984201D11E4A33E0224B984204D101
:10F658001B4A536843F470032EE01F4B984204D1B1
:10F66800174A536843F0706326E01C4B984204D154
:10F678001B4A536843F00F031EE01A4B984204D10B
:10F68800174A536843F0F00316E0174B984204D129
:10F69800134A536843F470630EE0144B984204D144
:10F6A8000F4A536843F4704306E0114B984204D163
:10F6B8000B4A536843F470235360704708000240B4
:10F6C800000002401C00024030000240440002409A
:10F6D800580002406C0002408000024008040240CA
:10F6E800000402401C04024030040240440402406A
:10F6F80058040240224A10B5536803F00C03042B47
:10F7080003D0082B04D01F4B14E01F4B5B6811E09B
:10F7180053685168C3F38343C90303F1020301D457
:10F728001A4906E0516811F4003F1749496818BFA3
:10F7380049084B4303605368154CC3F30313234430
:10F7480093F820100368CB4043605168C1F302214D
:10F75800214491F8201023FA01F181605168C1F326
:10F76800C221214491F82010CB40C3605268C2F3F3
:10F778008132224492F83020B3FBF2F3036110BDCA
:10F788000010024000127A003400002000093D00F9
:10F79800B8A4010810B50446FFF75AFD012806D1A0
:10F7A8001CB1FFF755FD013CF8E7052010BD002C02
:10F7B80008BF052010BD0A88F0B54B888E88B1F8BF
:10F7C80008E0CC88002A3AD1028C43F0010322F0E9
:10F7D80001021204120C0284058B078CADB225F0CD
:10F7E800F30545EA0E1189B241EA06027A49BFB229
:10F7F800884212D001F5006188420ED0B0F1804FE6
:10F808000BD0A1F59831884207D001F58061884274
:10F8180003D001F58061884202D127F0020701E098
:10F8280027F00A071F4302830784038B23F00C0386
:10F838001B041B0C0383038B9BB21C4344E0042A68
:10F8480044D1028C22F010021204120C0284018BA3
:10F85800058C21F440721205120D42EA0E325E49FF
:10F8680092B242EA06228842ADB292B212D001F5B3
:10F87800006188420ED0B0F1804F0BD0A1F59831CD
:10F88800884207D001F58061884203D001F5806184
:10F89800884207D125F0200141EA03139BB243F0C7
:10F8A800100304E025F0A00143F010030B4302838A
:10F8B8000384038B23F440631B041B0C0383038B17
:10F8C8009BB243EA0424A4B20483F0BD082A028C44
:10F8D8003ED122F480721204120C0284828B3E4DB7
:10F8E80092B222F0F307018C47EA0E1292B2A842B4
:10F8F80089B242EA060212D005F50065A8420ED088
:10F90800B0F1804F0BD0A5F59835A84207D005F582
:10F918008065A84203D005F58065A84207D121F487
:10F92800007141EA03239BB243F4807304E021F49D
:10F93800206143F480730B4382830384838B23F019
:10F948000C031B041B0C8383838B9BB21C4341E079
:10F9580022F480521204120C0284858B018C25F447
:10F9680040752D052D0D45EA062545EA0E321A4D3E
:10F9780089B2A84292B212D005F50065A8420ED00D
:10F98800B0F1804F0BD0A5F59835A84207D005F502
:10F998008065A84203D005F58065A84207D121F407
:10F9A800005141EA03339BB243F4805305E047F624
:10F9B800FF5543F480530D402B4382830384838B8C
:10F9C80023F440631B041B0C8383838B9BB243EAA1
:10F9D8000424A4B28483F0BD002C0140016830B532
:10F9E800CD43154B1C682C401C605A682A405A604D
:10F9F800027902F1804202F58232146821431160D3
:10FA080002689C68D5432C409C60D9682940D9601D
:10FA18004179102909BF996801F180431143996020
:10FA280015BF03F58233D96819680A4316BF0A431C
:10FA3800DA601A6030BD00BF00040140CA78F0B532
:10FA4800D40648BF8C780D8802F00F0348BF2343C3
:10FA580015F0FF0F1DD0016800240126A64006EA14
:10FA68000507B74211D14FEA840E0F2606FA0EF6A3
:10FA780021EA0601282A03FA0EF641EA060101D115
:10FA8800476102E0482A08BF07610134082CE4D125
:10FA98000160FF2D1FD94168002404F108070126E1
:10FAA800BE4006EA0507B74211D14FEA840E0F2679
:10FAB80006FA0EF621EA0601282A03FA0EF641EAAA
:10FAC800060101D1476102E0482A08BF07610134F5
:10FAD800082CE2D14160F0BD0F4B1A6842F00102D8
:10FAE8001A6059680D4A0A405A601A6822F08472EE
:10FAF80022F480321A601A6822F480221A605A6846
:10FB080022F4FE025A604FF41F029A60044B4FF031
:10FB180000629A60704700BF001002400000FFF8C2
:10FB280000ED00E02DE9F8435B4C0368013AC4F8A6
:10FB3800203183880D46A4F82431072A42D8DFE80B
:10FB480002F0040A101822292F35B4F820310B804E
:10FB5800B4F8223113E0B4F822310B80B4F8203124
:10FB680005E0B4F820315B420B80B4F822315B42E7
:10FB780005E0B4F822315B420B80B4F820316B8089
:10FB8800B4F824311DE0B4F820315B420B80B4F89E
:10FB9800223112E0B4F822310B80B4F820310CE0A5
:10FBA800B4F820310B80B4F8223105E0B4F82231E2
:10FBB8005B420B80B4F820315B426B80B4F824318F
:10FBC8005B42AB80354B1B7A002B62D1B5F9000044
:10FBD80003F0F0FC8046B5F9020003F0EBFC0746A1
:10FBE800B5F9040003F0E6FCD4F8281106464046AF
:10FBF80003F034FDD4F834118146384603F02EFD65
:10FC08000146484603F022FCD4F8401181463046AC
:10FC180003F024FD0146484603F018FC07F0DEFC1B
:10FC2800D4F82C112880404603F018FDD4F8381178
:10FC38008146384603F012FD0146484603F006FCAB
:10FC4800D4F844118146304603F008FD0146484681
:10FC580003F0FCFB07F0C2FCD4F830116880404682
:10FC680003F0FCFCD4F83C118046384603F0F6FC5F
:10FC78000146404603F0EAFBD4F8481107463046EF
:10FC880003F0ECFC0146384603F0E0FB07F0A6FC65
:10FC9800A880BDE8F88300BFD829002034000020E0
:10FCA80038B50F4B1B689C890E4B186880F3100001
:10FCB800201A03F07FFC0C4903F0D0FC05462046CF
:10FCC80003F078FC0146284603F07CFD03F08CFE27
:10FCD8006428A8BF642020EAE070C0B238BD00BF25
:10FCE800C8190020D81900200000C84244F6FB714A
:10FCF800084B1A68137803EB431300FB031350787F
:10FD0800C0EB0030B3FBF0F39078B3FBF0F080B2B7
:10FD1800704700BFC819002008B50A480A2290F8A1
:10FD28004D3100EB4303B3F85C1100F5B47089B2B0
:10FD380020F8041CF8F72AF980B2FFF7D7FF024B26
:10FD4800188008BDD8290020CC19002037B50446F2
:10FD580003211E2006226B4602F05AF878BB9DF854
:10FD680001309DF80000174D43EA002000B203F06F
:10FD780021FC296803F072FC03F036FE9DF803307D
:10FD880020809DF8020043EA002000B203F012FC34
:10FD9800A96803F063FC03F027FE9DF80530A080F6
:10FDA8009DF8040043EA002000B203F003FC6968F0
:10FDB80003F054FC03F018FE6080012000E00020EE
:10FDC80003B030BD400000201FB5044602210C20BE
:10FDD80001220DF1070302F01BF808B900203BE0EF
:10FDE8009DF80730DB07F9D50321062202AB0C206A
:10FDF80002F00EF80C20092101220DF1070302F090
:10FE080007F80028EAD09DF8073013F00C0FE5D169
:10FE18009DF809209DF808300C2043EA0223C3EB23
:10FE280083339B009DF80B2023809DF80A300A211C
:10FE380043EA0223C3EB83339B009DF80D206380C4
:10FE48009DF80C3043EA0223C3EB83339B00A38065
:10FE5800012202F01DF8012004B010BD07B50A21E7
:10FE680000220C2002F014F81420F7F7BEFF0A2134
:10FE78000F220C2002F00CF80A20F7F7B6FF01ABAE
:10FE8800102103220C2001F0C3FF0A20F7F7ADFF71
:10FE98000A2100220C2001F0FBFF0A20F7F7A5FF3A
:10FEA8000DF10303022101220C2001F0B1FF0DF135
:10FEB8000303092101220C2001F0AAFF0A210122D3
:10FEC8000C2001F0E5FF03B05DF804FB2DE9F047D5
:10FED800664D2B686649581C0A788E4602F0FF0664
:10FEE8000AB10346F6E737462B60687BAB6895F89E
:10FEF8000C80AA7B39B2202900F09C80DFF880C1F1
:10FF08000CEB8103DC789B783CF82110C3F1FF03EC
:10FF18009BB2002B65D04FF03C0CB1FBFCF9C3F150
:10FF2800FF0363431B12B9F1050F5DD8DFE809F041
:10FF3800030B1A293A4AE01A4143B1FBFCF0DAB242
:10FF48001044C0B251E0B1FBFCF00CFB101189B2B7
:10FF5800DAB2C1F13C01E31A4B43B3FBFCFC204687
:10FF680094442CE0B1FBFCF00CFB1011E21A89B2AE
:10FF78004A43B2FBFCF25FFA83F84244D2B220460D
:10FF880032E0B1FBFCF90CFB191189B2E01AC1F19E
:10FF98003C014843B0FBFCF05FFA83F84044C0B230
:10FFA800224621E0B1FBFCF80CFB1811D8B289B24B
:10FFB800E31A01FB03F2B2FBFCFC224684445FFA1D
:10FFC8008CF412E0B1FBFCF80CFB181189B2D8B222
:10FFD800C1F13C01E31A4B43B3FBFCF20244D2B239
:10FFE80003E02246204600E044464FEA042C4CEA4F
:08FFF800004C4CEA020C172337
:020000040801F1
:100000004FF0010808FA03F806F1170118EA0C0F7F
:10001000A1EB0301DFF8748014BF4FF011094FF01A
:10002000090989B213F1FF3308F80190E8D21836B4
:100030000137B6B2BFB2114BA0465FE7AB600123F8
:100040008EF8003040F22A33AA730D4AE9800D4938
:1000500085F80C806873AE80536000238B840B8816
:100060009BB243F001030B80136843F0010313605C
:10007000BDE8F087C82B00208A310020D42B002057
:100080006C000240000400408A0E0020D5020020CF
:10009000F0B5B1F800E000234EFA03F2D50725D5FC
:1000A0008E784FEAD30CF40648BFCC7806F00F02E6
:1000B00003F0070748BF2243BF0050F82C500F241D
:1000C000BC4025EA0404BA402243282E40F82C20E4
:1000D00005D1C46801229A4024EA020205E0482EB4
:1000E00004D1C46801229A402243C2600133102B1C
:1000F000D2D1F0BD2DE9FF41604B1B689BB11A685E
:100100001AB15F49886902438A619A889868ADF894
:10011000042002228DF8072004220DEB02018DF845
:100120000620FFF7B5FF3220F7F763FE002111220A
:100130001E2001F0B1FE012160221E2001F0ACFE64
:100140006420F7F756FE002402A8FFF703FE2746B7
:1001500026460A25022101221E2001F09DFE3220A2
:10016000F7F747FE02A8FFF7F5FDBDF90820BDF936
:100170000A1014448A42A8BF0A46BDF90C300F4445
:1001800093421E44A8BF134613F5805F09DD3D4A24
:10019000013DD36883F01003D360DBD14FF0010839
:1001A00001E04FF000081E200021122201F074FE31
:1001B0000A25022101221E2001F06EFE3220F7F7EF
:1001C00018FE02A8FFF7C6FDBDF90820BDF90A1008
:1001D000A41A8A42A8BF0A46BDF90C307F1A93427E
:1001E000A6EB0306A8BF134613F5805F07DD254A7B
:1001F000013DD36883F01003D360DAD101E04FF002
:100200000008204603F0DAF901461F4803F0DEFA41
:100210001E4D20F000402860384603F0CFF901461B
:10022000194803F0D3FA20F000406860304603F02C
:10023000C5F90146164803F0C9FA20F00040A8604D
:10024000002170221E2001F027FE012120221E2005
:1002500001F022FE1E200221002201F01DFE64207A
:10026000F7F7C7FDB8F1000F04D14FF07E532B60B4
:100270006B60AB6004B0BDE8F08100BFB402002049
:1002800000100240000C014000406F46400000207A
:1002900001C05E460F4B73B518781C4698B1052314
:1002A0000D4D8DF800304FF4805600238DF801304D
:1002B00001A86E616946022202F070FA2E619DF873
:1002C000050000F0010000F00100207080F0010046
:1002D00002B070BD21060020000C0140064B70B535
:1002E00006461C461D68FFF7D5FF18B923685B1B3F
:1002F000B342F8D970BD00BFC02D0020F7B503236D
:100300008DF80430030C8DF805308DF80700030AD2
:1003100006200F4614468DF80630FFF7DFFF78B150
:10032000084D4FF4805601A904226E61002002F0AE
:1003300035FA38460021224602F030FA20462E6176
:1003400003B0F0BD000C0140024640213C2001F00A
:10035000A3BD70B500EB8000094CA0F1A1059C384D
:1003600025440444074B15F8010F1E787040FFF731
:10037000EBFFA542F6D13046BDE87040E4E700BF90
:10038000ECA401088D31002010B5441E14F8010FB3
:1003900010B1FFF7DEFFF9E710BD024680213C20D7
:1003A00001F07ABD10B5D420FFF7F7FF8020FFF7EA
:1003B000F4FFA820FFF7F1FF3F20FFF7EEFFD32067
:1003C000FFF7EBFF0020FFF7E8FF4020FFF7E5FF16
:1003D0008D20FFF7E2FF1420FFF7DFFFA120FFF7DA
:1003E000DCFFC820FFF7D9FFDA20FFF7D6FF122085
:1003F000FFF7D3FF8120FFF7D0FFCF20FFF7CDFF1E
:10040000D920FFF7CAFFF120FFF7C7FFDB20FFF776
:10041000C4FF4020FFF7C1FFA420FFF7BEFFA620C6
:10042000FFF7BBFFAF20FFF7B8FFA620FFF7B5FF30
:10043000AE20FFF7B2FF2020FFF7AFFF0020FFF74D
:10044000ACFFB020FFF7A9FF4020FFF7A6FF002078
:10045000FFF7A3FF1020FFF7A0FF4FF48064013CDB
:100460000020A4B2FFF770FF002CF8D18120FFF725
:1004700094FFC820FFF791FFAF20FFF78EFF012008
:1004800010BD08B55038C0B2FFF787FF0020FFF756
:1004900084FFBDE8084010207FE710B504465039BE
:1004A000C8B2FFF77AFF04EB4400400000F00E00F2
:1004B000FFF773FF06206043BDE81040C0F3031050
:1004C00010306AE7012828BF01202DE9F04F0646C9
:1004D000734F142000FB0671724BD1F8A4421E75B5
:1004E0001C61714BD1F8B422DD69B1F8AC822A43AA
:1004F000DA61A288B1F8AEA222F44072D1F8A85213
:10050000120489B0120C4AEA0809A28003A9C5F8AE
:10051000109002228DF80E0028460193ADF80C9041
:100520008DF80F20FFF7B4FD019B00971F464FF099
:10053000080BAA6818EA020F03D10A20F7F74EFC4D
:10054000F7E70A20C5F81480F7F748FCC5F81080D3
:100550000A20F7F743FCBBF1010BEAD1C5F814A060
:100560000A20F7F73BFCC5F814800A20F7F736FCA1
:10057000C5F810800A20F7F731FC0222C5F810A058
:10058000284603A98DF80F201C228DF80E20ADF807
:100590000C90FFF77DFD454A03A894423A690BBFD2
:1005A00042F4001242F480023A613A610BBF3A69A8
:1005B0003A6922F4001222F480023A61A38823F4FB
:1005C00040731B041B0CA38023889BB243F00103E0
:1005D0002380A588FFF792F80599354B25F03F0554
:1005E000B1FBF3F32D042D0C1D43ADB2A580228881
:1005F000002522F001021204120C22802D4A03A8C9
:10060000B1FBF2F100298AB208BF012242F4004195
:100610004FF4967253434FF47A7293FBF2F3013323
:100620009BB22384A1832388009A9BB243F00103E9
:100630002380238823F4816323F002031B041B0C13
:1006400023804FF480432381142303FB062696F86E
:10065000B13201248DF80C308DF80D508DF80E500C
:100660008DF80F4002F056F896F8B0329DF80F2042
:100670008DF80C308DF80D508DF80E501AB103A87E
:1006800002F048F808E05A0903F01F039C4002F109
:100690002003094A42F8234009B0BDE8F08F00BFAB
:1006A000ECA40108C82B00200010024000540040B8
:1006B00040420F00804F120000E100E010B5134BE4
:1006C000014693F8D837012B19D1114B114C1878EA
:1006D000421CD2B21A70120644BF00221A700E4A8F
:1006E0001B7812782154934236BFC2F180029B1AC4
:1006F0009B183F2B09D9BDE81040FBF703BF074B00
:10070000BDE810401868F7F742BC10BDEC1100209E
:10071000AC2C0020AE2C0020AD2C0020082E002098
:10072000F0B5974D87B02B78023B082B00F28A81F9
:10073000DFE813F009002E004F0064007C008E00FB
:100740000A016E0179018F4B8F4C1A68636864331C
:100750009A4240F2778100268C4B8D4A1B789E424C
:100760000ADA2368884FD05C30B1FFF7A7FF3B68F7
:10077000013601333B60EFE72168834B525C002A6E
:1007800040F060811A604FF0FF325A6003231BE093
:10079000262300937F4B492003F10C020193029220
:1007A0005021A3F10A020233F9F79CFE002840F021
:1007B0004981794B4FF0FF311B6813F08002724B77
:1007C00004D083E8030004232B703BE11A605960D6
:1007D0002AE0724A022300210093019102914820ED
:1007E00002F10803F9F77EFE002840F02B81664BEA
:1007F0004FF0FF3218605A600523E5E707230093A6
:10080000674B472003F10C02019302920021A3F1F0
:1008100008020433F9F766FE002840F013815A4BB2
:100820004FF0FF3218605A600623CDE75D4A05237A
:100830000021009301910291532002F10803F9F77E
:1008400051FE002840F0FE804F4B18600723BBE7A5
:100850004D4C236813B96360012323604B4B1A7816
:1008600063681344402BA8BF4023132B636040F3FD
:10087000E980454B1B680D2B00F2EA80DFE803F0AE
:1008800060070B0E121923282D3134404B51464876
:1008900001F0C1F851E0454845493FE04548464927
:1008A000464A48E0464B474893F8D61793F8D7276F
:1008B00041E0434B0C2193F8B027434801FB02333E
:1008C00093F8B2172AE03E4B4048B3F8441125E0B4
:1008D0003B4B3F48B3F8461120E03E4B3E48196978
:1008E0001CE03E483E4B18E03E4B1B68D80404D544
:1008F000334B3D4893F87C1110E00C2323601FE03C
:100900002F4B3A4893F8801193F8812193F87F3167
:1009100001F0ECF811E03648364B198801F0E6F8A2
:100920000BE01D4B1B6819050AD5254B3248B3F85F
:100930008411B3F9822101F0D9F86368181A606054
:100940002368013323607DE02C4B1B689A0114D58A
:100950002B4B1B888BB92B4B0E201B6804A90493CF
:10096000294B1B680593F9F7A1FA284B4FF48052E5
:100970001A8009232B70F9F713FBF9F779FA61E074
:10098000FC2D0020C02D0020BC2F00206400002082
:10099000B8A7010822A801089C2D0020E0A90108A1
:1009A000F8A9010844AA0108A2C80108BFC80108A3
:1009B000C9BC0108D7C80108B4BC0108C0BC010803
:1009C000EC110020EEC8010802C901080FC9010896
:1009D00021C901085029002033C9010846C901086E
:1009E0002C000020A42F002053C9010863C901086E
:1009F0007FC90108A02F00208DC90108E410002044
:100A0000B02F0020AC2F00206C310020C42F00201C
:100A1000154B1B78002BAED0144B1B689B01AAD43E
:100A200008232B70A9E7124B1A68124B5B68C83376
:100A30009A4203D900F014FF0123C5E600F02AFF13
:100A40000028F7D100F0F6FE60B101232B7009E019
:100A500000F020FF0028F5D0074B4FF480521A8099
:100A60000923B1E607B0F0BDA82F0020E410002054
:100A7000C02D0020BC2F0020C42F002010B54B88B3
:100A8000DC0641BF2F4B14791B6853F8244044BF48
:100A90002D4B43F820404B889B0641BF294B54798E
:100AA0001B6853F8244044BF274B43F820404B8831
:100AB0001C070ED5254B0C781B78B3EB141FA1BF78
:100AC000204BD4781B6853F82440A4BF1E4B43F836
:100AD00020404B889B070ED51D4B0C781B78B3EB41
:100AE000141FDFBF174B54781B6853F82440DCBF3A
:100AF000154B43F820404B88DC070FD5154C0B787D
:100B0000247803F00F03A342DFBF0E4B14781B6859
:100B100053F82440DCBF0C4B43F820404B885B0764
:100B20000FD50B780C4903F00F0309788B42A1BF56
:100B3000044B92781B6853F82220A4BF024B43F861
:100B4000202010BDD02900208A0E0020A3220020E2
:100B5000A1220020A0220020A2220020254A00235A
:100B6000F0B515681C461A462348244903700B70DB
:100B70002E1976884EB92F5D3FB9037000230A7095
:100B80004B7007781C461A460CE0360548BF013208
:100B900004F1040403F1010348BFD2B2802CDBB29C
:100BA000E6D1EAE7E0B2B8420CD215F824000134ED
:100BB00006099E4200F00F00A8BF731C9042A8BF18
:100BC000421CEFE78A704B70C2F3470102F001024A
:100BD0000A444C1E0A490B480A70C3F3470203F04B
:100BE0000103134404700849501E084A087013702A
:100BF000F0BD00BF4022002098220020E02B002002
:100C0000A2220020A0220020A3220020A122002056
:100C1000924B2DE9F04FDA68914D1A612A6891B034
:100C2000DA60904A0295136843F0200313608E4BFC
:100C30001A78012A0CBF002201221A708B4B1A78F5
:100C4000910740F14D838A490978042940F248838D
:100C50008849097801F0040101F0FF0011B922F080
:100C600001021A701B78DB0702D408B1FBF7CCFA3B
:100C70008149CA78531C052293FBF2F202EB8202EF
:100C80009A1A7E4BCA701F7892000023DFF81082F8
:100C9000DFF8109258F82310794C91FBF9FE04F11B
:100CA000080040F823E0774844F8231000FB0E11B9
:100CB00042F2107091FBF0F004F1100680B226F8B9
:100CC00013004FF0140C04F114060CFB036C04F138
:100CD0003C0A5AF823605CF802504CF80210761B6C
:100CE000314405264AF8231091FBF6F109FB0E1159
:100CF0004434012F44F823104FEA830B444605D1B6
:100D00000238B0F5797F98BF4BF808100BB9012372
:100D1000BCE7594E029BB2461868336DC01A02F008
:100D200049FC594902F052FD029B4FF07E511B686D
:100D30000746336502F034FE08B94FF07E574B4B3F
:100D4000CAF854701B78514E13F00103504D12D065
:100D50000DAA00924F4B0EAA01920CCB94E803000F
:100D6000FBF768F90D9A6421B2FBF1F20E9B328019
:100D700093FBF1F300E033802B809AF858303E4D1E
:100D8000002B35D0696D4FF07E5002F01FFD0746F5
:100D9000EB6D2068C01A02F011FC394602F062FCCB
:100DA00002F026FE2B6E86B2606836B2C01A02F0E0
:100DB00005FC394B196802F055FC394602F052FC2B
:100DC00002F016FEB5F9662000B28118B5F964206C
:100DD0000220B31891FBF0F193FBF0F389B29BB2C0
:100DE000A5F86A10A5F86830A5F86610A5F8643073
:100DF00001238AF85830294B61681B88206803F06A
:100E000030031D4E264DCAF86010CAF85C00002B56
:100E100000F0668206F17403009306F178030193F3
:100E2000F26E336FFBF706F96B68306FC01A02F091
:100E3000C5FB194B196802F015FC02F0D9FDF36EE1
:100E40002A68C6F880009B1AF3670C4B1B78012BAD
:100E50002AD0022B00F0E68042E200BFB407002057
:100E6000C02D0020DC1900204E110020E0190020C8
:100E7000E61900208B310020E02B00201410002008
:100E8000E42B0020806967FF00007A445A1A002092
:100E90005C1A0020501100204C000020A41A0020F1
:100EA000E819002080969800D6F88430D6F8A04043
:100EB0000293D6F8943004F100400393D6F89830AA
:100EC000776D059302F094FD8146204602F090FD77
:100ED000D6F89C30BB4C0493BB4B06901B684FF07C
:100EE000000B0793B94E4FEA4B0356F82B80A6F13F
:100EF0001402404632F81B50089302F05FFB02993F
:100F000002F0B0FB02F074FD401B1FFA80FA283695
:100F100026F81BA00FFA8AFA504602F04FFB0399FD
:100F200002F0A0FB02F064FD86B20AEB080002F0BA
:100F300045FB059902F096FB394602F093FB2168C8
:100F400002F088FA02F054FD484504DB069B984203
:100F5000A8BF184600E0484602F030FB206002F0CF
:100F600047FD079B304486B2987802F023FB9849EE
:100F700002F078FB01464FF07E5002F027FC394624
:100F800002F068FA0146384602F020FC09906068D9
:100F9000D4F808A0C0EB080002F010FB394602F0BC
:100FA00015FC514602F054FA099A0146104602F027
:100FB00059FB0146504602F04DFA3135ADB2622D73
:100FC00001462061C4F80480A0600ED9049802F0A4
:100FD00049FB02F00DFD7F4AB0F5FA6FA8BF4FF450
:100FE000FA609042B8BF104600E0002040F6B832E8
:100FF000064436B29642A8BF1646774A089B9642E8
:10100000B8BF1646754A54F8140B9E52142202FBC0
:101010000BF273495050BBF1000F40F061814FF06B
:10102000010B5FE7684BB6F8A8401F68736F3D89F6
:1010300002935B089D4228BF1D4623B29D4202DCFD
:101040001FFA85F90AE06749706D02F00BFB02F0A8
:10105000CFFC20441FFA80F9A6F8A890DAF878604F
:10106000DAF8AC40341B2046FBF726F841F2931324
:101070000028D8BF40429842CCBF0020012078B35E
:10108000204602F09BFA584902F0ECFAF9F7E7FD26
:101090000446029802F08EFA0146204602F0E2FA77
:1010A00002F0A6FC40F6B83380B2AAF8B00000B255
:1010B0009842A8BF1846484B9842ACBF3018F01869
:1010C00048F6A043984203DDA0F50C40A03804E0A8
:1010D0000028BCBF00F50C40A030CAF8B40001E005
:1010E000CAF8B460DAF8B4300026C3F50C502830E2
:1010F000039302F063FA3C4902F0B4FA0446F9F7AC
:1011000021FE0F902046F9F7AAFDDAF8B830DAF898
:10111000C4400593DAF8BC300E9004F10040089307
:1011200002F066FC0490204602F062FCDAF8C0305F
:10113000DAF854802A4C09900793730048460A93C2
:1011400002F03CFA0EAB53F8261002F08BFADFF8EF
:10115000A0A005463AF9160002F030FA01462846EA
:1011600002F076F902F044FC05B2204BB5F57A7F27
:10117000A8BF4FF47A759D42B8BF1D460AF13C0ADC
:10118000A8B22AF8160000B202F018FA05998246B1
:1011900002F068FA02F02CFC089983B250460693DC
:1011A00002F060FA414602F05DFA216802F052F95D
:1011B00002F01EFC049B98421CDB099B9842A8BFCE
:1011C000184618E050100020181000205C2C002059
:1011D000DB0FC94030F8FFFF48F4FFFF221000206A
:1011E000781000200000C842D302373918FCFFFFF6
:1011F000482C0020049802F0E1F920608346B8787A
:1012000002F0D8F9384902F02DFA01464FF07E502D
:1012100002F0DCFA414602F01DF90146404602F0B8
:10122000D5FA0B906068D4F808A0281A02F0C6F925
:10123000414602F0CBFA514602F00AF9DDF82CC023
:101240000146604602F00EFA0146504602F002F9ED
:10125000656001462061A060079802F003FA02F081
:10126000C7FB069B1434034458469A4602F0C0FB61
:1012700040F6B832504400B29042A8BF10461B4A14
:101280000A9B9042B8BF1046194A1A499852142234
:10129000724342F801B00EB901264EE73B792BB1FB
:1012A000039A642392FBF3F3134A13803B88029A58
:1012B000124C9A420DD9D4F8AC30A06FC01AFAF78C
:1012C000FBFE42F2107380EAE072A2EBE0729A42F7
:1012D00006DD0B4B01221A70B4F8C820064B1A80A9
:1012E00011B0BDE8F08F00BFDB0FC94048F4FFFF2D
:1012F000221000205010002010100020E02B0020B1
:10130000141000200846FFF7D9B910B50D4C20681D
:10131000F8F7D6FB20680022047A02FB02F3193B9F
:10132000634303F6C4135343192193FBF1F30649B6
:1013300021F812300132072AEFD1BDE810400349ED
:10134000F8F776BB48110020A010002030130020D1
:101350000E4B1A78692A16D140F2DC7259889142F4
:1013600011D11A79BE2A0ED193F8D9270020EF2A7D
:101370000BD113F8012B5040054A9342F9D1B0FA32
:1013800080F04009704700207047704700F803085C
:10139000DCFF03082DE9F74FEA4C002140F2DC7234
:1013A000204605F012FFE84B04F53A721A60E74B4D
:1013B00000221A70E64B04F2B2711960692323709F
:1013C000032363714FF48073A3604FF41673A4F882
:1013D0006631FA23A4F86831BC23A4F864314FF4D1
:1013E000FA73A4F86E31012384F8623184F87E31F7
:1013F00084F88631052384F8273240F2DC53A4F8C0
:10140000983140F24C43A4F89A3140F26C73A4F83E
:101410009C3140F27533A4F89E3140F64303A4F8A2
:10142000A0312346202184F86A116E2184F87C11B2
:101430000A2184F87D112B2184F87F11212184F861
:101440008011232184F881114FF4C871A4F882110E
:10145000032ACCBF0121002102F1010283F8A2116D
:1014600014BF1E217521122A83F8A31103F1020370
:10147000EED140F27E41A4F8441140F23A71A4F852
:10148000461140F27E51A4F84C1140F2EA5140F26C
:10149000DC50A4F84E1140F2B4514FF4FA63A4F8B2
:1014A000C831A4F8CC31A4F8D031A4F8D431052344
:1014B00084F8E231C82301264FF47A774FF0320BDB
:1014C000A4F8E631DFF880924FF4C8734FF01E0A9B
:1014D0001922A4F8EA31A4F84A01A4F85011A4F89A
:1014E000C671A4F8CA71A4F8CE71A4F8D27184F8B8
:1014F000E46184F8E56184F8E861A4F84871A4F82F
:1015000052B184F895A184F8E32100920190A4F8E7
:10151000543184F8E16184F8EE61A4F856B184F89E
:10152000F161FDF793FFD9F80030009A00254FF0E4
:101530000F0E2674E673A573A58183F805E0DA71B2
:101540004FF0220E2122172183F806E05A744FF043
:101550000E0E53225975997583F810E0DA765521ED
:101560000A224FF0350E4FF02808D97083F81AE0A0
:101570002D214FF05A0E9A7400924FF0780C64228D
:1015800083F80BA083F80CA0597383F808E01A774E
:101590001D7083F8018083F80280DD7583F804B044
:1015A0009D731D76DD735D7683F8098083F80AC02C
:1015B00019754FF4FA71A3F84E103C2183F85110BD
:1015C000112183F850106349DFF8A8C19963D963EA
:1015D0006149C3F82CC099626049C3F830C0DFF894
:1015E00098C159634FF07F5A5D490198C3F820A014
:1015F000C3F824A0C3F848C04FF0000A4FF04B0CCA
:1016000059649E7783F85250C3F840A083F84CC0C9
:1016100084F8B2E7A4F8BC074FF0410E042084F828
:10162000B3E784F8B4B784F8B55784F8B95784F8A9
:10163000BA5784F8B65784F8B75784F8B85783F880
:101640005C00A3F85850A3F85A50A3F856501966F6
:10165000152183F8681043494348D966434983F804
:1016600064801967424983F86580596783F8786018
:10167000FDF716FFD9F80030009A18464FF448716C
:1016800083F8115183F8125183F8138183F81461A0
:1016900083F81851A3F8161184F8D821C82284F8C9
:1016A000D9216422A4F8DA7184F8DC51A4F8DE218F
:1016B0000E2202FB05326FF0170482F81941032451
:1016C00082F81A416FF02F0482F81B41072482F838
:1016D0001C416FF0230482F81D41052482F81E414D
:1016E00001355A2480F8204180F821416422FF24EA
:1016F000082D80F81F2180F822414FF0000100F1F1
:101700000E00D5D1C820A3F88A01142083F88C01DB
:10171000A3F890211E204FF4967283F88D01A3F850
:1017200092210120282283F8891183F88E01A3F8E1
:1017300094210B46034D5A191033C02BC2F814A044
:101740001CE000BFEC11002020110020482D0020DB
:10175000481100208FC2F53C000060406666663F7D
:101760000000A0409A99193FADCA0108F6287C3FB5
:101770003D0A773FCDCCCC3E00004040DAD105F5A4
:101780002A700021402205F020FD0023264EEA1891
:10179000995904330868382B244CC2F8A802F5D1B3
:1017A00004F50A700021802205F00FFD06F13801D2
:1017B000702204F50A7005F0FDFCFFF7CFF9D9F8A7
:1017C000006000230125314604F590604FF4CC728F
:1017D00084F8D83784F8D65784F8D75705F0EAFC50
:1017E00004F5C36031464FF4CC7205F0E3FC104BB6
:1017F0001B681A68C4F8BE275A68C4F8C2279A68DA
:10180000C4F8C6271A68C4F8CA275A68C4F8CE278D
:101810009A680223C4F8D22784F8D45484F86C362A
:1018200003B0BDE8F08F00BF6CAA0108EC110020E6
:1018300048110020074B93F8D837012B08D1064AEE
:10184000064BD0681B68834234BF002001207047DC
:1018500000207047EC1100201C000020240600200E
:1018600038B5094B93F8D85765B9084C2068F7F795
:10187000A4FF074B25601B78022B03D1BDE838403D
:10188000FDF7A3BD38BD00BFEC110020082E0020DD
:10189000042E0020064B93F8D8371BB1012B05D13D
:1018A000FAF730BE034B1868F6F765BB00207047A7
:1018B000EC110020082E0020F8B5011F0646002379
:1018C000083051F8042F02F120043F2C3BD802F1DC
:1018D00008040F2C06D80232032A04D9002B08BFB3
:1018E000012300E002238142EBD1012B30680ED0AE
:1018F000022B1AD0736800F0030003F003039B006F
:1019000043EA0010B36803F00303184317E000F044
:101910000F0040F04000FEF7D1FEB068736800F0A1
:101920000F0040EA0310C0B209E000F03F0040F0B1
:101930008000FEF7C3FE3079FEF7C0FE307ABDE8C6
:10194000F840FEF7BBBE06F10C0734463A460025C8
:1019500052F8043DAD0003F18001FF2910D903F5D1
:101960000041B1F5803F02D245F0010508E003F5E2
:101970000003B3F1807F34BF45F0020545F0030555
:10198000B242E5D165F03F00C0B2FEF797FE05F028
:101990000303022B207807D0032B0CD0012B13D18B
:1019A000FEF78CFE60780FE0FEF788FE6078FEF7A9
:1019B00085FEA07808E0FEF781FE6078FEF77EFEE7
:1019C000A078FEF77BFEE0780434FEF777FEBC4299
:1019D0004FEAA505DBD1F8BD10B50446C0B2FEF74D
:1019E0006DFEC4F30720BDE81040FEF767BE10B5DA
:1019F00004467F2C06D964F07F00C0B2FEF75EFE7D
:101A0000E409F6E7E0B2BDE81040FEF757BE430038
:101A100083EAE070EBE72DE9F047314B86B093F8AD
:101A2000D8370746012B01D004464AE005F011FCE7
:101A30000546064603A96846FAF772FC039B049A1A
:101A4000029713442B443F2B059519D90023684670
:101A500003A90322FAF790FC039B3BB9049B2BB923
:101A6000204A13705370059BABB301E0FAF740FCBA
:101A7000039B049A059E134433447F2B2BD8029F6B
:101A8000DFF860903946CA461AF8024BC4F1800864
:101A9000B04528BFB0460AEB04004444E4B24246D5
:101AA00005F088FB802C89F8004014D1C8EB0606AD
:101AB000504607EB0801324605F07CFB89F80060D0
:101AC00009E0254614F8011B21B1074B1868F6F709
:101AD0005EFAF6E7ED1B284606B0BDE8F08700BFCA
:101AE000EC110020AC2C0020082E00200FB407B50C
:101AF00004AB53F8042B054900200193F8F780FF4D
:101B000003B05DF804EB04B0704700BF0513010893
:101B1000054A08B5138801339BB21380034B18782C
:101B2000FEF7D0FC002008BDE2100020DC2B0020D6
:101B30009148F0B50368914A9C8AA4B2E1B211F0D1
:101B4000010F2ED0198821F400610904090C1980B5
:101B5000198889B241F4806119800021117051788F
:101B600099B1917811B9D178FF290ED101219170E5
:101B70001179022901BF198889B241F400611980E5
:101B8000517941F001011982E1E0517901F0FE0142
:101B90001982D378FF2B00F0DA80784BFF2119707F
:101BA000D5E08E073AD5BFF35F8F1479E4B2012CEC
:101BB00013D1517889B1917879B1198821F4806174
:101BC0000904090C1980BFF35F8F198B1988947170
:101BD00089B241F4007119801BE0198BBFF35F8F4C
:101BE00014796649022C0AD14C7844B1897831B114
:101BF000198821F480610904090C1980A1E0147985
